:020000040800F2
:10000000000001209D2300087D1600087F160008CF
:1000100081160008831600088516000800000000FD
:10002000000000000000000000000000871600082B
:1000300089160008000000008B1600088D160008C5
:10004000ED230008ED23000891160008ED230008B9
:10005000ED230008ED230008ED230008ED23000840
:10006000ED230008ED230008ED230008ED23000830
:10007000ED230008ED230008ED230008ED23000820
:10008000ED230008ED230008ED230008ED23000810
:1000900000000000ED230008ED230008ED23000818
:1000A000ED230008ED230008ED230008ED230008F0
:1000B000ED230008ED230008ED230008ED230008E0
:1000C000ED230008ED230008ED230008ED230008D0
:1000D000ED230008ED230008ED230008ED230008C0
:1000E000ED230008ED2300089D160008ED2300080D
:1000F000ED2300080000000000000000ED230008D0
:10010000ED230008ED230008A9160008ED230008E0
:10011000ED230008ED230008ED230008ED2300087F
:10012000ED230008ED230008ED230008ED2300086F
:08013000ED230008ED23000897
:1001380010B5054C237833B9044B13B10448AFF319
:1001480000800123237010BD08010020000000007A
:10015800E0EA000808B5034B1BB103490348AFF3B5
:10016800008008BD000000000C010020E0EA000843
:10017800034613F8012B002AFBD1181A01387047DF
:1001880081F0004102E000BF83F0004330B54FEA40
:1001980041044FEA430594EA050F08BF90EA020FAD
:1001A8001FBF54EA000C55EA020C7FEA645C7FEA40
:1001B800655C00F0E2804FEA5454D4EB5555B8BF63
:1001C8006D420CDD2C4480EA020281EA030382EAD4
:1001D800000083EA010180EA020281EA0303362D66
:1001E80088BF30BD11F0004F4FEA01314FF4801C39
:1001F8004CEA113102D0404261EB410113F0004F4B
:100208004FEA03334CEA133302D0524263EB430301
:1002180094EA050F00F0A780A4F10104D5F1200E9F
:100228000DDB02FA0EFC22FA05F2801841F10001FA
:1002380003FA0EF2801843FA05F359410EE0A5F1CE
:1002480020050EF1200E012A03FA0EFC28BF4CF0FF
:10025800020C43FA05F3C01851EBE37101F00045B5
:1002680007D54FF0000EDCF1000C7EEB00006EEBC2
:100278000101B1F5801F1BD3B1F5001F0CD349084C
:100288005FEA30004FEA3C0C04F101044FEA4452A3
:1002980012F5800F80F09A80BCF1004F08BF5FEA2A
:1002A800500C50F1000041EB045141EA050130BD0A
:1002B8005FEA4C0C404141EB0101013C28BFB1F51C
:1002C800801FE9D291F0000F04BF01460020B1FA67
:1002D80081F308BF2033A3F10B03B3F120020CDA3A
:1002E8000C3208DD02F1140CC2F10C0201FA0CF018
:1002F80021FA02F10CE002F11402D8BFC2F1200C7D
:1003080001FA02F120FA0CFCDCBF41EA0C01904032
:10031800E41AA2BF01EB0451294330BD6FEA04047B
:100328001F3C1CDA0C340EDC04F11404C4F1200266
:1003380020FA04F001FA02F340EA030021FA04F378
:1003480045EA030130BDC4F10C04C4F1200220FACF
:1003580002F001FA04F340EA0300294630BD21FA0D
:1003680004F0294630BD94F0000F83F4801306BFD3
:1003780081F480110134013D4EE77FEA645C18BFC7
:100388007FEA655C29D094EA050F08BF90EA020F5E
:1003980005D054EA000C04BF1946104630BD91EA56
:1003A800030F1EBF0021002030BD5FEA545C05D159
:1003B8004000494128BF41F0004130BD14F5800498
:1003C8003CBF01F5801130BD01F0004545F0FE410C
:1003D80041F470014FF0000030BD7FEA645C1ABF41
:1003E800194610467FEA655C1CBF0B46024650EA78
:1003F800013406BF52EA033591EA030F41F40021A4
:1004080030BD00BF90F0000F04BF0021704730B529
:100418004FF4806404F132044FF000054FF00001FE
:1004280050E700BF90F0000F04BF0021704730B5BF
:100438004FF4806404F1320410F0004548BF404294
:100448004FF000013EE700BF42004FEAE2014FEAE9
:1004580031014FEA02701FBF12F07F4393F07F4FC4
:1004680081F06051704732F07F4208BF704793F0C7
:100478007F4F04BF41F40021704730B54FF46074DA
:1004880001F0004521F000411CE700BF50EA0102DD
:1004980008BF704730B54FF000050AE050EA010286
:1004A80008BF704730B511F0004502D5404261EBF6
:1004B80041014FF4806404F132045FEA915C3FF437
:1004C800D8AE4FF003025FEADC0C18BF03325FEAD4
:1004D800DC0C18BF033202EBDC02C2F1200300FA85
:1004E80003FC20FA02F001FA03FE40EA0E0021FAAA
:1004F80002F11444BDE600BF4FF0FF3C06E000BF28
:100508004FF0010C02E000BF4FF0010C4DF804CD94
:100518004FEA410C7FEA6C5C4FEA430C18BF7FEA54
:100528006C5C1BD001B050EA410C0CBF52EA430C82
:1005380091EA030F02BF90EA020F0020704710F102
:10054800000F91EA030F58BF994208BF90422CBF91
:10055800D8176FEAE37040F0010070474FEA410C8A
:100568007FEA6C5C02D150EA013C07D14FEA430CA8
:100578007FEA6C5CD6D152EA033CD3D05DF8040B19
:10058800704700BF8446104662468C46194663464B
:1005980000E000BF01B5FFF7B7FF002848BF10F122
:1005A800000F01BD4DF808EDFFF7F4FF0CBF012067
:1005B80000205DF808FB00BF4DF808EDFFF7EAFFE3
:1005C80034BF012000205DF808FB00BF4DF808ED9E
:1005D800FFF7E0FF94BF012000205DF808FB00BF93
:1005E8004DF808EDFFF7CEFF94BF012000205DF81D
:1005F80008FB00BF4DF808EDFFF7C4FF34BF01202A
:1006080000205DF808FB00BF4FEA410212F5001216
:1006180015D211D56FF47873B3EB625212D94FEA41
:10062800C12343F0004343EA505311F0004F23FA2B
:1006380002F018BF404270474FF00000704750EA80
:10064800013005D111F0004008BF6FF0004070473D
:100658004FF00000704700BF80F0004002E000BF8C
:1006680081F0004142001FBF5FEA410392EA030F95
:100678007FEA226C7FEA236C6AD04FEA1262D2EBDF
:100688001363C1BFD218414048404140B8BF5B42E4
:10069800192B88BF704710F0004F40F4000020F07D
:1006A8007F4018BF404211F0004F41F4000121F093
:1006B8007F4118BF494292EA030F3FD0A2F10102DD
:1006C80041FA03FC10EB0C00C3F1200301FA03F11B
:1006D80000F0004302D5494260EB4000B0F5000F3E
:1006E80013D3B0F1807F06D340084FEA310102F1FD
:1006F8000102FE2A51D2B1F1004F40EBC25008BFAF
:1007080020F0010040EA03007047490040EB000078
:10071800013A28BFB0F5000FEDD2B0FA80FCACF179
:10072800080CB2EB0C0200FA0CF0AABF00EBC250A6
:1007380052421843BCBFD0401843704792F0000F94
:1007480081F4000106BF80F400000132013BB5E7E7
:100758004FEA41037FEA226C18BF7FEA236C21D05D
:1007680092EA030F04D092F0000F08BF08467047C2
:1007780090EA010F1CBF0020704712F07F4F04D190
:10078800400028BF40F00040704712F100723CBFA3
:1007980000F50000704700F0004343F0FE4040F4CD
:1007A800000070477FEA226216BF08467FEA23638B
:1007B8000146420206BF5FEA412390EA010F40F476
:1007C800800070474FF0000304E000BF10F00043C2
:1007D80048BF40425FEA000C08BF704743F09643A9
:1007E80001464FF000001CE050EA010208BF7047C4
:1007F8004FF000030AE000BF50EA010208BF70474B
:1008080011F0004302D5404261EB41015FEA010C5F
:1008180002BF84460146002043F0B64308BFA3F157
:100828008053A3F50003BCFA8CF2083AA3EBC25339
:1008380010DB01FA02FC634400FA02FCC2F1200258
:10084800BCF1004F20FA02F243EB020008BF20F08F
:100858000100704702F1200201FA02FCC2F12002F5
:1008680050EA4C0021FA02F243EB020008BF20EAEA
:10087800DC7070474FF0FF0C1CEAD0521EBF1CEA18
:10088800D15392EA0C0F93EA0C0F6FD01A4480EA06
:10089800010C400218BF5FEA41211ED04FF00063EF
:1008A80043EA501043EA5111A0FB01310CF000401B
:1008B800B1F5000F3EBF490041EAD3715B0040EA41
:1008C800010062F17F02FD2A1DD8B3F1004F40EB11
:1008D800C25008BF20F00100704790F0000F0CF0E4
:1008E800004C08BF49024CEA502040EA51207F3AA8
:1008F800C2BFD2F1FF0340EAC250704740F4000083
:100908004FF00003013A5DDC12F1190FDCBF00F073
:1009180000407047C2F10002410021FA02F1C2F121
:10092800200200FA02FC5FEA310040F1000053EABD
:100938004C0308BF20EADC70704792F0000F00F00B
:10094800004C02BF400010F4000F013AF9D040EA11
:100958000C0093F0000F01F0004C02BF490011F4A5
:10096800000F013BF9D041EA0C018FE70CEAD153A3
:1009780092EA0C0F18BF93EA0C0F0AD030F0004C23
:1009880018BF31F0004CD8D180EA010000F00040D7
:10099800704790F0000F17BF90F0004F084691F095
:1009A800000F91F0004F14D092EA0C0F01D14202CF
:1009B8000FD193EA0C0F03D14B0218BF084608D198
:1009C80080EA010000F0004040F0FE4040F40000E2
:1009D800704740F0FE4040F4400070474FF0FF0C75
:1009E8001CEAD0521EBF1CEAD15392EA0C0F93EABC
:1009F8000C0F69D0A2EB030280EA010C49024FEA0E
:100A0800402037D04FF0805343EA111143EA1013C6
:100A18000CF000408B4238BF5B0042F17D024FF47E
:100A2800000C8B4224BF5B1A40EA0C00B3EB510F59
:100A380024BFA3EB510340EA5C00B3EB910F24BF42
:100A4800A3EB910340EA9C00B3EBD10F24BFA3EBC7
:100A5800D10340EADC001B0118BF5FEA1C1CE0D18F
:100A6800FD2A3FF650AF8B4240EBC25008BF20F042
:100A7800010070470CF0004C4CEA50207F32C2BF96
:100A8800D2F1FF0340EAC250704740F400004FF033
:100A98000003013A37E792F0000F00F0004C02BF64
:100AA800400010F4000F013AF9D040EA0C0093F02E
:100AB800000F01F0004C02BF490011F4000F013B88
:100AC800F9D041EA0C0195E70CEAD15392EA0C0FF0
:100AD80008D142027FF47DAF93EA0C0F7FF470AF28
:100AE800084676E793EA0C0F04D14B023FF44CAF6B
:100AF80008466EE730F0004C18BF31F0004CCAD100
:100B080030F000427FF45CAF31F000437FF43CAF3B
:100B18005FE700BF4FEA4002B2F1FE4F0FD34FF03C
:100B28009E03B3EB12620DD94FEA002343F0004352
:100B380010F0004F23FA02F018BF404270474FF000
:100B48000000704712F1610F01D1420205D110F087
:100B5800004008BF6FF0004070474FF0000070473A
:100B680042000ED2B2F1FE4F0BD34FF09E03B3EB0F
:100B7800126209D44FEA002343F0004323FA02F03B
:100B880070474FF00000704712F1610F01D1420227
:100B980002D14FF0FF3070474FF00000704700BFA0
:100BA80053B94AB9002908BF00281CBF4FF0FF31CC
:100BB8004FF0FF3000F06AB9ADF1080C6DE904CED2
:100BC80000F006F8DDF804E0DDE9022304B0704720
:100BD8002DE9F047089D0C46002B4ED194468C45D4
:100BE8008646B2FA82F262D94AB1C2F12003914034
:100BF80020FA03F30CFA02FC194300FA02FE4FEA4A
:100C08001C471FFA8CF6B1FBF7F44FEA1E4307FBAB
:100C1800141143EA014304FB06F199420AD91CEB7B
:100C2800030304F1FF3080F01281994240F20F81F2
:100C3800023C6344591A1FFA8EF3B1FBF7F007FB25
:100C4800101143EA014300FB06F69E420AD91CEB49
:100C5800030300F1FF3180F0FC809E4240F2F980EE
:100C6800634402389B1B40EA044000211DB1D34075
:100C78000022C5E90032BDE8F0878B4205D90DB1E5
:100C8800C5E9000100210846F5E7B3FA83F1002918
:100C980046D1A34202D39042C0F0F080861A64EB9A
:100CA80003030120002DE6D0C5E90063E3E7002A2D
:100CB80040F09080A1EB0C044FEA1C481FFA8CF717
:100CC8000121B4FBF8F64FEA1E4308FB164443EA39
:100CD800044307FB06F0984208D91CEB030306F10E
:100CE800FF3402D2984200F2CD8026461C1A1FFA21
:100CF8008EF3B4FBF8F008FB104443EA044300FB0E
:100D080007F79F4208D91CEB030300F1FF3402D216
:100D18009F4200F2B0802046DB1B40EA0640A5E770
:100D2800C1F120068B4022FA06F71F4320FA06FC81
:100D380004FA01F343EA0C03F44000FA01F8380C12
:100D48004FEA1349B4FBF0FE1FFA87FC00FB1E4470
:100D580049EA04440EFB0CF9A14502FA01F20AD94A
:100D68003C190EF1FF3A80F08480A14540F2818061
:100D7800AEF1020E3C44A4EB09041FFA83F9B4FB5C
:100D8800F0F300FB134449EA044403FB0CFCA445BC
:100D980007D93C1903F1FF3067D2A44565D9023B56
:100DA8003C4443EA0E40A0FB0293A4EB0C049C4293
:100DB800CE469C4651D34ED055B1B8EB0E0364EBEA
:100DC8000C0404FA06F6CB401E43CC40C5E9006487
:100DD800002150E7C2F1200320FA03F10CFA02FCCB
:100DE80024FA03F394400C434FEA1C4800FA02FE2D
:100DF8001FFA8CF7B3FBF8F008FB1031230C43EA19
:100E0800014300FB07F1994208D91CEB030300F1E9
:100E1800FF362CD299422AD9023863445B1AA4B20D
:100E2800B3FBF8F108FB113344EA034401FB07F371
:100E3800A34208D91CEB040401F1FF3613D2A342E4
:100E480011D902396444E41A41EA004139E70446F9
:100E5800F0E6084606E7C845AED2B9EB020E63EBEA
:100E6800070C0138A8E73146EDE7034699E7304615
:100E7800D4E7D6467FE7634402384DE70646234663
:100E880008460FE7023E634430E700BF704700BFE3
:100E98001348144A08B54FF00043C0E90023042260
:100EA800426101220023C2614FF480510722C0E948
:100EB8000233C0E90933C0E90C1203610383837666
:100EC80080F8203080F82C30826380F83C30C3648E
:100ED80001F0C4FA18B1BDE8084000F009BB08BD2C
:100EE80024010020002401400268084B9A4282B085
:100EF8000AD14FF0B0431A6E42F400721A661B6EA4
:100F080003F400730193019B02B070470024014071
:100F18000268054B9A4201BF4FF0B042136E23F4AA
:100F280000731366704700BF0024014030B585B0D8
:100F380000240546CDE901440394FFF7A9FF1448AE
:100F480001F020FE08B100F0D3FA1148039401A97A
:100F5800CDE9015401F0E0FB08B100F0C9FA0C48F2
:100F680001F03AFD08B100F0C3FA4FF0FF3108482C
:100F780001F074FB064801F0E7FD054801F0C8FBE5
:100F88000446034801F08AFD204605B030BD00BF85
:100F980024010020014B024A1A60704724010020F6
:100FA8000024014008B50948FFF7C0FF68B1084BA5
:100FB800B3F8AA304FF6FF72934216BF40F6E442E8
:100FC800044B5343B3FBF0F398B208BD002000B4C0
:100FD8000075FF1FD8084C0013B50023ADF8063084
:100FE800FFF7E0FF04461948FFF7A0FF184BB3F8D6
:100FF800C820B3F8A8108A4204FB00F018D040F6C5
:10100800E443B0FBF3F364205B1A4343521A93FBA7
:10101800F2F31E331BB2ADF80630BDF806305BB2F2
:101028001B02ADF80630BDF8060000B202B010BDD4
:101038004FF47A7240F6FF73B0FBF3F35343A3F512
:101048003923A3F50C6340F6C412E0E7001000B0A2
:101058000075FF1F4FF0B04307B59A6C42F00402C9
:101068009A649A6C02F004020192019A9A6C42F016
:1010780001029A649B6C03F0010300930022022191
:101088000F20009B01F01CFE0F2003B05DF804EB5D
:1010980001F048BE08B501F0C9FF10B16FF00400B7
:1010A80008BD064B9A6942F040429A614CF2FA3206
:1010B8001A6101F0CDFF0028F2D0EFE70040005898
:1010C800F0B585B000230D4600930646A8B3FFF798
:1010D800E1FF044670BB01F0A9FF88BB1A481B4A10
:1010E80002230193D0F8E01506F1784302EA812142
:1010F800B3FBF1F701FB1733DB0A0293D0F8E005E5
:1011080005F178410139314402EA8022B1FBF2F05D
:1011180002FB1011C3EBD1230133694601A80393E5
:1011280002F016F820B1022814BF6FF00104012460
:1011380001F08EFF204605B0F0BD6FF00504F9E719
:101148006FF00404F6E700BF0070FF1F00FCFF0308
:10115800014B186000207047880100202DE9F04FEE
:10116800B0F1006F89B006460F469046C0F0C080C7
:10117800DFF89091644DD9F8E03505EA832303F14F
:101188000063013B984200F2B380002900F0B3806D
:1011980040EA02035B0740F0AE80FFF77BFF04469E
:1011A80090BB01F043FF002840F0A880D9F8E01573
:1011B800009705EA812106F17842B2FBF1F301FBC1
:1011C800132208F17843013B3344B3FBF1F001FBF0
:1011D8001033DB0A01334FEAD22AA3EBD222012AC9
:1011E800039388BFC6F30A050AF58037C6F10803DA
:1011F8008CBFC5F500654546FF02B3460693039BC1
:101208009A4505D301F024FF204609B0BDE8F08FC8
:10121800A6F10803069A1A4495421CD8009B049527
:101228000193CDF814B04FF00009059B09EB0301B9
:10123800049B99453DD3009BAB442B44A8EB050583
:10124800B5F5006F009328BF4FF400650AF1010A55
:1012580007F50067D3E753F8081F5A68B2F1FF3F54
:1012680008BFB1F1FF3FD5D0284B186810B96FF00F
:101278000504C7E727B14FF4006239460CF052FF66
:10128800DFF888900099D9F80030CBF30A001844A9
:10129800AAB20CF047FF4FF400613846FFF710FF81
:1012A80000BBD9F8003001934FF40063059704930D
:1012B800B9E7019B07914B4402930120D3E900232E
:1012C80001F000FF88B90799019BD1E9000259F89C
:1012D8000310029B5B689A4208BF884205D109F156
:1012E8000809A2E76FF001048CE76FF0030489E7AF
:1012F8004FF0FF3488E76FF0050485E76FF00404CA
:1013080082E700BF0070FF1F00FCFF038801002078
:10131800B1F1006F70B510D30B4BD3F8E0650B4BF0
:1013280003EA862303F10063013B994205D838B1EB
:1013380092B20CF0F7FE002070BD4FF0FF30FBE7D3
:101348006FF00500F8E700BF0070FF1F00FCFF0307
:10135800B0F1006F10B40DD3084BD3F8E045084B3B
:1013680003EA842303F10063013B984202D810BCCE
:10137800FFF7A6BE4FF0FF3010BC70470070FF1F8C
:1013880000FCFF034FF0B04382B0DA6C0243DA642A
:10139800DB6C03400193019B02B07047F0B502205B
:1013A80087B00024244ECDE90444FFF7EBFF042066
:1013B800FFF7E8FF0120FFF7E5FF03254FF6FF736E
:1013C80001A93046CDE90135039401F00FFF01A9C9
:1013D8001A4801F00BFF01A94FF0904001F006FFF9
:1013E8004FF0B0430220DA6C22F00102DA64DA6CC2
:1013F80022F00202DA64DA6C22F00402DA64FFF7FF
:10140800C1FF01271423CDE9034001A93046CDE9E6
:10141800013701F0EBFE3846FFF7B4FF01A94FF49E
:1014280000434FF09040CDE90135CDE9034501F087
:10143800DDFE07B0F0BD00BF00040048000800480A
:1014480000B59BB04822002108A80DF097FA182291
:10145800002102A80DF092FA01F0F6FF4FF0B04219
:101468000120D2F8903023F01803C2F89030D2F857
:10147800003423F4C06343F40073C2F80034D2F894
:10148800003403F4C0630193019B24230893812350
:101498000B930023CDE91003B02208A8CDE912234D
:1014A80002F04AF908B172B6FEE74F23CDE90230DF
:1014B800CDE90400CDE90600022102A802F0D6FB1E
:1014C80008B172B6FEE71BB05DF804FB08B500F082
:1014D8008BFFFFF7B5FFFFF761FF044803F0E4FA5D
:1014E80000F040FC00F045FCFCE700BF3C02002097
:1014F80072B6FEE700B58DB02C22002101A80DF0D0
:101508003DFA1748174B03601F2383604FF0804252
:101518000023C0E90433C0E9072383614FF48073D3
:10152800436202F049FE08B1FFF7E2FF0C4802F0FF
:101538006FFF08B1FFF7DCFF4FF00053002207935D
:10154800074808924FF4807301A9029206920B9300
:1015580002F092FE08B1FFF7CBFF0DB05DF804FB77
:101568008C0100200028004010B5044690B03822B5
:10157800002102A80DF002FA2268194B9A422CD1D8
:101588004FF48033029302A84FF480730F9302F054
:1015980091FC08B1FFF7ACFF4FF0B0430220D3F83D
:1015A800902042F40042C3F890209A6D42F4806281
:1015B8009A659B6D002203F4806311460193019B99
:1015C80001F07EFB022001F0ADFB00222A2011462B
:1015D80001F076FB2A2001F0A5FB10B010BD00BF7A
:1015E800002800407047000010B51448144C03F060
:1015F8005BFA00F075FB00224FF6FF714FF0904048
:1016080001F014FF20464FF6FF7101F09BFE2046C3
:1016180000224FF6FF7101F009FF0A4800224FF639
:10162800FF7101F003FF00F0F5FE074B0120BDE854
:101638001040C3F8880001F05FBF00BF3C020020E3
:1016480000040048000800480004005800F0E9BE03
:1016580008B500F0E6FEBDE80840FFF79FBE08B5F4
:1016680000F0D8FEBDE808400121002001F0F4BEDA
:1016780070477047FEE7FEE7FEE7FEE7FEE77047C4
:101688007047704770470000014802F0E7BE00BF8E
:101698008C010020014802F015BD00BF8C0100201C
:1016A800014803F004B900BFC4010020054808B58B
:1016B8000823036002F018FF18B1BDE80840FFF7DF
:1016C80017BF08BDC40100204FF0B04307B55A6EDC
:1016D80042F001025A665B6E002203F00103019397
:1016E80011463220019B01F0EBFA322003B05DF87D
:1016F80004EB01F017BB00000CB407B5054A05ABB5
:10170800102101930DF018F803B05DF804EB02B056
:10171800704700BF84EB000830B585B0044602A8C6
:101728000D460CF035FEBDF90C30064A0093102129
:10173800029B2046FFF7E0FF2046FEF719FD2880B0
:1017480005B030BD84EB00084FF0B04210B5936887
:1017580023F4004393600CF0A3FE0D4B01241C708E
:101768000CF070FB0B480CF087FB0B4B4FF400425E
:101778001A6100200CF086FBFFF70CFC00F0B4F8AF
:101788000CF07AFC21462046BDE810400CF094BCD1
:10179800D001002021170008004000580CF0A2BC1E
:1017A80008B5FFF7FFFB40F6B83398420CD8B0F500
:1017B800E16F0BD3FE23A0F5E16058434FF4966325
:1017C800B0FBF3F0C0B208BDFE20FCE70020FAE74A
:1017D8007FB5684600F06CF80198FFF79BF900B2F6
:1017E80007B05DF804FB0000194A38B5D2F8803517
:1017F800591C044619D100F01BFE054600F024FED2
:10180800054400F01BFE2B0EE3712B0CA3712B0A71
:101818006371030EE370C0F30742C0F30723257119
:10182800C0B2A2706370207038BD190AC37181718B
:10183800190C1B0E41710371D2F88435C370D2F8AC
:101848008405C0F30722C0F30743000EE9E700BF91
:101858000070FF1F38B5094BD3F88035036001339A
:10186800054609D100F0E4FD044600F0E7FD4440D8
:1018780000F0EAFD44402C6038BD00BF0070FF1F37
:10188800012102200CF002BC002102200CF0FEBB5A
:1018980000207047024B187808B100F05DB8704717
:1018A800D001002082B00190019802B000F0F0B899
:1018B80010B50446FFF790FB074BA36040F30F20D9
:1018C800FEF784FF054B064A2360064B6060C4E9B7
:1018D8000323002010BD00BF0000484200007A44E6
:1018E8000D093E00AB03050000207047014B186846
:1018F800704700BFD40100200320704708B5014697
:101908004FF47A7200238002890DFFF749F908BD68
:101918004FF47A73A0FB0303800A40EA83507047B0
:10192800034B98689A689042FBD1C043704700BF48
:101938000028004008B5FFF7F3FF014B186008BD09
:10194800D401002008B5FFF7EBFF024B1B68C01A53
:1019580008BD00BFD4010020024B187808B1FFF77A
:10196800DFBF7047D801002010B5074B074C012294
:10197800DA654FF48071204602F06AFB4FF0FF33BE
:101988002363002010BD00BF002800408C01002008
:1019980002460021014802F072BD00BF8C01002000
:1019A80002460121014802F06ABD00BF8C010020F7
:1019B80010B58CB02C220021044601A80CF0DEFFE3
:1019C800FFF7D2FF0C4B0D481B681C4400230893FB
:1019D80006934FF00053E443079301224FF48073BA
:1019E80001A902940B9302F047FC08B1FFF780FDB0
:1019F80000200CB010BD00BFD40100208C010020D5
:101A080038B50546FFF78CFF02210446074802F067
:101A18003DFDC4F309024FF47A71A2FB0121920A39
:101A2800A30A2A8043EA805038BD00BF8C010020F9
:101A38000148002102F02ABD8C0100200148012143
:101A480002F024BD8C010020F8B50F4D2E78CEB9D8
:101A58000E4C4FF0FF372763FFF74CFDFFF784FF6D
:101A68004FF48071204602F0F3FA2046276302F013
:101A7800B1FC32462046022102F001FDFFF75AFF71
:101A880001232B700020F8BDD80100208C01002014
:101A9800014610B54FF47A7200238002890DFFF7D2
:101AA8007FF80146FFF73CFF0446FFF739FF031BA9
:101AB8008B4200D310BD00BFF7E70CF0F9BD000062
:101AC80010B5064C0221204602F0E0FC0221421C1F
:101AD8002046BDE8104002F0D2BC00BF8C010020B7
:101AE8001348144A08B54FF4E133C0E90023002332
:101AF8000C22C0E90233C0E90523C0E90733C0E975
:101B08000933036103F0EBFC08B1FFF7F1FC084867
:101B1800002103F059FE08B1FFF7EAFC044803F07E
:101B280033FE18B1BDE80840FFF7E2BC08BD00BFAE
:101B38003C0200200044004070B596B006461422CE
:101B4800002103A80CF01AFF3822002108A80CF085
:101B580015FF32682C4B9A4254D10223089308A8E7
:101B68002A4B0A9302F0A6F908B1FFF7C1FC4FF01F
:101B7800B04300259A6D42F400329A659A6D02F4DA
:101B880000320292029ADA6C42F00102DA64DB6CEB
:101B980003F0010301930422019B0223CDE90323EF
:101BA8000324072303A94FF09040CDE90554079378
:101BB80001F01CFB082303A94FF09040CDE9033442
:101BC800CDE90555124C01F011FB12492562142389
:101BD800C4E900131023C4E9023520468023C4E970
:101BE8000435C4E9065501F0FDF808B1FFF780FC9B
:101BF8002520F46700220221A66201F061F8252061
:101C080001F090F816B070BD0044004004000C00CC
:101C1800DC0100205800024002680C4B9A4210B5C3
:101C2800044612D14FF0B0420C21936D23F40033D7
:101C380093654FF0904001F085FBE06F01F044F9A7
:101C4800BDE81040252001F07BB810BD00440040DD
:101C580008B50A460146024802F046FF002008BDC2
:101C68003C02002013B5114B114C18604FF40013BF
:101C7800009302AB13E90600204603F029FD236810
:101C8800DA69D103FCD4DA695202FCD59A680848AB
:101C980042F480029A6003F061FD0649044801227B
:101CA80003F0D2FC002002B010BD00BFD00200201B
:101CB8003C020020D802002008B5074B1860FFF747
:101CC800C9F9FFF70DFF054AD2F8803043F00063E9
:101CD800C2F88030002008BDD40200200008005857
:101CE80008B54FF0B04308489A6B42F400329A6343
:101CF8009A6B22F400329A63FFF78EFF0F2001F0EF
:101D08001FF8002008BD00BF3C0200200268044BF9
:101D18009A4203D1034B00201B681847704700BF45
:101D280000440040D402002002680B4B9A4210B5D0
:101D380004460FD1094B1B682BB1D0F8902012B97B
:101D480007480121984720460549BDE8104001226F
:101D580003F07ABC10BD00BF00440040D002002050
:101D6800D802002008B5FFF7EFFCBDE8084000F0F6
:101D78000BBA4FF0FF300CF019BA70477047704734
:101D8800014BD870704700BF0C000020014B18743D
:101D9800704700BF0C00002002480022042101F017
:101DA80045BB00BF00040048024800224FF4007100
:101DB80001F03CBB00040048002101200CF0BEB932
:101DC80008B50D4B1B78022B03D1002108200CF01D
:101DD800B5F90A480022042101F028FB074800222F
:101DE8004FF4007101F022FBBDE8084003480022CF
:101DF8004FF4006101F01ABB700000200004004895
:101E080010B5114C01222046102101F00FFB0122D0
:101E18002046042101F00AFB002102200CF08EF973
:101E280040F6B830FFF73EFD20460022042101F0BD
:101E3800FDFA20460022102101F0F8FABDE8104012
:101E480002480CF0E3BB00BF000400483004002047
:101E580010B5094B094C002818BF034608482360F1
:101E68000CF086FB216806480CF00AFCBDE810401F
:101E780003480CF0CBBB00BFC0D401000800002011
:101E8800300400200A460149FFF742BA00F003086F
:101E980038B514480122042101F0C8FA114801227A
:101EA8004FF4007101F0C2FA0E4801224FF40061AC
:101EB80001F0BCFA0C480CF05BFB04F0E5F860B9E3
:101EC8000A4C0B480125257003F072FF207829463B
:101ED80003F0C6FC04480CF099FBBDE838400548FF
:101EE8000CF094BB0004004830040020700000206F
:101EF8000C0000201804002004F064B92DE9F04318
:101F080087B0FFF74DFCFFF74DF8064603F0A2FD3A
:101F1800054690B1002444480CF02AFB434B424844
:101F28001B689C42214638BF19460CF0A9FB3E4865
:101F38000CF06CFB07B0BDE8F0833D4C6846FFF73A
:101F4800B7FC0223029823703A49FEF793FCFEF788
:101F580007FE87B20198FEF7DDFD37490FFA80F8D2
:101F68000098FEF787FC3349FEF738FDFEF7F8FDC9
:101F7800324A636812781A706368C0F307225A708D
:101F880063689870636883F803806368DFF8B080DB
:101F98003A0A1A7163685F7198F80030082B01D00B
:101FA800012B29D86268002393716268D371626833
:101FB800137253726423B6FBF3F60B2396726370A5
:101FC800204C637A63B103F031FD012808D1204623
:101FD8000CF0CEFA1C4800224FF4006101F026FAFA
:101FE80098F803101248002203F04AFD063091D1F8
:101FF80003F016FD04468EE7DDE90376D4F8049075
:10200800FFF7CEFB89F8060063683A14DA71636853
:102018003A121A7232149A7232125F72DA721E739C
:102028005D739D730F23CAE7300400200800002069
:1020380000000020000020410000C84224030020C6
:102048000C000020DC0200200004004810B558B144
:1020580090F9064044B906480CF08AFA0548224629
:102068004FF4006101F0E2F9BDE81040FFF746BF08
:10207800DC0200200004004802484FF4006101F02F
:10208800DAB900BF0004004808B560B1037853B15D
:10209800054801224FF4007101F0C8F9BDE8084075
:1020A80002480CF0B3BA08BD000400480C03002035
:1020B80008B503F0F2FF80B903F0B8FC01280CD191
:1020C800BFF34F8F0549064BCA6802F4E062134319
:1020D800CB60BFF34F8F00BFFDE708BD00ED00E008
:1020E8000400FA0538B504460D4679B318480122AC
:1020F800042101F09BF917480CF088FA2B782BB3D0
:1021080024B3636822780BB3022A0ED0032A1DD1A8
:102118006278012A1AD11878012802D0022800D042
:10212800A0B9BDE8384003F075BD6278012A0DD129
:102138001B78094903F001030B7003B91A46BDE87F
:10214800384003484FF4006101F070B938BD00BF52
:1021580000040048F40200202403002038B5044697
:102168000D4607484FF40061FFF7F2F830B92A46E8
:1021780021460348BDE83840FEF7F0BF38BD00BF30
:1021880000F00308704700001FB5002403A920468B
:10219800039403F067FF03A9012003F063FF2C4BAE
:1021A8002C48009422464FF4FA710CF083F92A4B1C
:1021B8002A48009422464FF4FA710CF07BF9284B18
:1021C8002848009401224FF4FA710CF073F9204664
:1021D800FEF7BEFF08B1FFF78BF9234B00940022EE
:1021E8004FF4FA6121480CF065F9214A00210120D9
:1021F8000CF060F81F4A002102200CF05BF81E4A20
:10220800002104200CF056F81C4A002108200CF08C
:1022180051F800F043F81A491A4803F0D9FE1A4851
:1022280003F0C6FD0F480CF0F1F9184B002118789F
:1022380003F016FB16490094164B0968164800224D
:102248000CF038F914480CF0E1F904B010BD00BFE7
:10225800B11D00080C030020A11D0008F402002095
:1022680081200008DC020020C91D00081804002095
:10227800BD5B0008051F0008011F0008991E000823
:1022880000000301240000200C0000207000002042
:1022980008000020091E000830040020034B00221B
:1022A800C3E902220122C3E9002270474804002042
:1022B80000487047480400204FF0B04382B0DA6C01
:1022C8000243DA64DB6C03400193019B02B0704760
:1022D8002DE9F04186B000240220154D0594FFF742
:1022E800EBFF0420FFF7E8FF124F03944FF48076CA
:1022F80001230DEB0001CDE9016328460323049374
:102308004FF4005800F072FF01A93846CDF8048058
:1023180000F06CFF22464146384601F087F828460F
:102328002246314601F082F8204606B0BDE8F08129
:102338000004004800080048032810B50ED80128FA
:1023480010D868B902460B484FF4807101F06EF856
:10235800002209484FF4005101F068F8002010BD30
:102368000122F0E7002203484FF4807101F05EF883
:102378000122EEE7000400480008004802207047E8
:102388000020704701207047002814BF16200F2036
:10239800704700000D48854600F025F80C480D49A7
:1023A8000D4A002302E0D458C4500433C4188C42A8
:1023B800F9D30A4A0A4C002301E013600432A2420E
:1023C800FBD30CF0E3FAFFF781F8FEE700000120E9
:1023D8000000002008010020ACF6000808010020D9
:1023E800B8210020FEE7704710B5032000F056FC26
:1023F80001F092F9064B18600F20FFF749FA0446DE
:1024080018B9FFF736F9204610BD0124FBE700BFD5
:10241800740000204FF0E022136923F002031361D7
:1024280070474FF0E022136943F0020313617047CD
:10243800014BD3F8900570470070FF1F014BD3F88C
:10244800940570470070FF1F014BD3F8980570473B
:102458000070FF1F8068C0F380007047F7B5002345
:1024680001930446002800F0E980856D25B9FEF740
:102478003BFDE56584F8545023689A68D00040F124
:10248800A1809A68D10000F1B480A26D42F01002D8
:10249800A265E26D42F00102E26501251846FFF7E8
:1024A800D9FFA26D02F01002024340F0C980A26D6C
:1024B800206922F4817242F00202A2659A68D2076A
:1024C8005DD4226BA67E94F82CC0003A18BF012276
:1024D8001703D4E902120A43217E42EA8132617E5F
:1024E80042EAC13242EA4632002842EA4C02B4BF0C
:1024F80020F000414FF400113A430A4394F82010A9
:10250800012903D1002E76D142F48032616A21B1CB
:10251800A66A01F4E07131430A43D968E66C21F4F4
:10252800FE3121F4FF711143D96094F83C206168B1
:10253800012A01F0404C4CEA060609D1D4E91027DB
:102548003A433243A66C324342EA0C0242F0010697
:102558001F693E4A3A4032431A6121F00042B2F103
:10256800804F0CD0B1F1004F09D0394ED6F808276A
:1025780001F4701122F470120A43C6F808275A6948
:10258800666BA16B22F0070232435A615A6922F046
:10259800700242EA01125A61002835D19A6A62F043
:1025A8000F029A625B6903F007039E423CD1002345
:1025B800E365A36D23F0030343F00103A3652846F5
:1025C80003B0F0BD9A68234922F0104222F01702A6
:1025D80042F080529A60204A1268B2FBF1F201324E
:1025E80052000192019A002A3FF44BAF019A013A36
:1025F800F7E7002552E7A16D41F02001A165E16DE3
:1026080041F00101E16581E7B0F5001FCAD19A6A7E
:10261800E269013A92006FF00F0102F01C0201FA20
:1026280002F2216E0A43BCE7A36D23F0120343F0C4
:102638001003A365E36D43F00103E3650125BEE7DD
:10264800A36D43F01003A365F8E700BF02FCFF1F6A
:1026580000200140400D030074000020F8B54569D2
:10266800082D04460E460AD00368DB68D80705D54E
:10267800A36D43F02003A3650120F8BD0425FFF7EF
:1026880009F9074623681A682A4220D0A26D42F445
:102698000072A265DA6812F4406F14D1A27E92B972
:1026A8001A6812070FD51846FFF7D4FE20BB5A68E0
:1026B80022F00C025A60A26D22F4807222F001020C
:1026C80042F00102A265227EFAB10020D5E7711C12
:1026D800D9D0FFF7DFF8C01BB04201D8002ED1D106
:1026E80023681B682B40CDD1A26D84F8543042F08A
:1026F8000402A2650320C0E7A26D42F02002A26591
:10270800E26D42F00102E265DDE70C221A60DCE7C7
:102718000368186C70470000F7B50023019390F820
:102728005430012B044600F0C0800568026901237B
:1027380080F854302846FFF78DFE002840F0AF801F
:10274800D1E90030022822F004027ED0B2F1004F15
:10275800C3F3110E35D1AA6A42EA0E02AA628A6848
:10276800686902EA032222F07C4222F0FF0220EA92
:1027780003210A43002B6A611DDA4D4A4D4DD2F8F8
:102788000817AB4201F0E07043D10D0213D4D2F820
:10279800083723F0E073034343F40003C2F8083713
:1027A800454B1A68454BB2FBF3F20C2302FB03338B
:1027B8000193019B53BB0020002384F8543003B0DD
:1027C800F0BD226E00F01F074FF00F0C0CFA07FC4B
:1027D8006FEA0C0622EA0C0CBEF1000F11D1C3F30C
:1027E8008462BA4042EA0C0222668008E26901303B
:1027F8009042B4D8A86AC3F38362BA400640324311
:10280800ACE793FAA3F2B2FA82F2EAE7019B013B42
:10281800CEE72B4DAB420BD1C901CCD4D2F8083747
:1028280023F0E073034343F08073C2F80837C2E72C
:10283800244DAB42BFD14B02BDD4D2F8083723F0A8
:10284800E073034343F48003EFE7B2F1004F01BFA5
:10285800AA6AC3F311018A43AA62002BABDA1548AE
:1028680013498342D1F8082709D1D1F8083702F073
:10287800A07223F0E0731A43C1F808279BE71048B9
:10288800834204D1D1F8083702F44002F1E70D4839
:10289800834290D1D1F8083702F0C072E9E7A26DFF
:1028A80042F02002A265184686E7022087E700BFAB
:1028B80000200140001000B074000020400D03000B
:1028C800004000B8002000B4026838B5044610463D
:1028D800FFF7C0FD08B9002038BD9368990707D4F1
:1028E800936823F0004323F0170343F01003936029
:1028F800FEF7D0FF054623689B685B07EBD5FEF71C
:10290800C9FF401B0228F6D923689B685A07F2D5ED
:10291800A36D43F01003A365E36D43F00103E36582
:102928000120D9E773B50023026801939368DD0796
:10293800044602D5002002B070BD9168214B1942AF
:1029480009D0A36D43F01003A365E36D43F00103C1
:10295800E3650120EFE7936823F0004323F01703B2
:1029680043F001039360184BD3F8083718021CD4BE
:10297800637E012BDED0FEF78DFF144E05462268DC
:102988001368DB07D6D49368D9075FBF93683340D1
:1029980043F001039360FEF77DFF401B0228EED948
:1029A80023681B68DA07EAD4CBE7094B094A1B6896
:1029B800B3FBF2F301330193019B002BD8D0019BA9
:1029C800013BF8E71700008000200140E8FFFF7F87
:1029D80074000020400D030038B504460068FFF776
:1029E80039FD054620BB94F85430012B20D0012333
:1029F80084F854302046FFF795FFB0B9A36D2268DC
:102A080023F4706323F0010343F48073A3651C234C
:102A1800E065136084F85400936823F0004323F0C2
:102A2800170343F00403936038BD84F85450FBE760
:102A38000220F9E7026838B5936891680446C80728
:102A480001D4002038BD9907FBD4936803F005032F
:102A5800012B19D1936823F0004323F0170343F0A7
:102A68000203936003231360FEF714FF05462368EF
:102A78009B68DB07E5D5FEF70DFF401B0228F6D95A
:102A880023689B68DA07F2D5A36D43F01003A365AA
:102A9800E36D43F00103E3650120D3E770B5044615
:102AA80000284BD0836D43F002038365FFF70CFFCA
:102AB800054668B92046FFF7BDFF054608B901235A
:102AC800A3652268936823F0104323F017039360EB
:102AD80023685A6822F4677222F003025A6040F2AF
:102AE8009F321A60D968164A0A40DA601A6922F0D9
:102AF80040421A615A6922F007025A611A6A02F0C2
:102B0800F0221A625A6A02F0F0225A62DA6A02F075
:102B1800F022DA629A6A0B4A00269E62D2F80837D7
:102B280023F0FE73C2F808372046FEF7F1F9E66590
:102B38002666A66584F85460284670BD0125FBE723
:102B480000023E830020014010B590F85430012B5C
:102B5800044615D0012380F85430FFF7B5FE58B964
:102B68002046FFF767FF38B9A36D23F4807323F07D
:102B7800010343F00103A365002384F8543010BD1A
:102B88000220FCE7F7B50023019390F85430012B9D
:102B980004467FD0012380F85430FFF74BFF2368A9
:102BA8009A6812F00102054607D0A36D43F010039E
:102BB800A365002384F854302DE0A16D364F21F42D
:102BC800817141F00201A165DE68D96826F4FF46EB
:102BD80026F07C0621F40041360421F00301360C6E
:102BE800D96008209968394041F000419960996896
:102BF800002913DA0199013101910199B1F52E3FAC
:102C0800F5D3A36D23F0120343F01003A36500234B
:102C180084F854300125284603B0F0BDD3F8B41029
:102C2800013801F07F010A44DCD199681A48014053
:102C380041F001019960D3F8B41021F07F0141EA15
:102C4800D202C3F8B4209A68024042F002029A60A5
:102C5800FEF720FE074623689A68D20708D4DA6888
:102C68003243DA60A36D23F0030343F001039FE7C7
:102C7800FEF710FEC01B0228EDD923689B68D90710
:102C8800E9D5A36D43F01003A365E36D43F0010399
:102C9800E365BFE70225BEE7E8FFFF7F0749CA688B
:102CA80022F4E0620302120403F4E063120C1343FB
:102CB80043F0BF6343F40033CB60704700ED00E09E
:102CC800164B30B5DC68C4F30224C4F10703251D94
:102CD800042B28BF0423062D4FF0FF358CBF033C7F
:102CE800002405FA03F321EA0303A54022EA0502BA
:102CF800A340002843EA0203ACBF00F16040084A41
:102D08004FEA0313B8BF00F00F00DBB2AABF00F50B
:102D18006140135480F8003330BD00BF00ED00E07F
:102D280014ED00E0002807DB044A4109012300F004
:102D38001F00834042F82130704700BF00E100E0E7
:102D480000280CDB4309064900F01F00203301224C
:102D5800824041F82320BFF34F8FBFF36F8F704736
:102D680000E100E070B5D0E913456560446D14B129
:102D7800D0E916456560D0E9105404F01C0601241A
:102D8800B4406C60046863608368102B0BBFA2605A
:102D9800A160E160E26070BD0268416CD3B210B519
:102DA800083B1424B3FBF4F30B4CA24288BF0B4A34
:102DB80021F0030199BF01F1804202F50232521855
:102DC80007338264064AC26403F01F03012202FA31
:102DD80003F3036510BD00BF070402401C0802404E
:102DE8008008024038B500285CD002682E4B9A4211
:102DF8004FF014014AD82D4B1344B3FBF1F32C497F
:102E08009B00C0E91013022380F825301368056978
:102E180023F4FF4323F070031360D0E902432343F4
:102E28002B43456911682B4385692B43C5692B439F
:102E3800056A2B430B431360FFF7AEFFB4F5804FD1
:102E480004BF002343604368816C03F07F020A607B
:102E5800D0E91314013B032B4C601ED8154B1649BF
:102E6800816513449B000121013A01FA02F2002115
:102E78004365C2651960114B5A6400230122C3637C
:102E880080F8243080F82520184638BD0C4B1344B0
:102E9800B3FBF1F30B499B00B3E70023C0E91533FB
:102EA800C365EAE70120F0E707040240F8FFFDBF29
:102EB800000002403F820010400902400009024021
:102EC800F8FBFDBF0004024038B5002841D0026875
:102ED800136823F0010313601F4B9A424FF014014B
:102EE80030D81E4B1344B3FBF1F31D499B00C0E9D6
:102EF8001013012403F01C0304FA03F300251560E2
:102F08004B60FFF749FF836C41681D60D0E91332BD
:102F18005A604A1E032A06D8124B0B449B00944061
:102F28001D60114B5C640023C363C0E91533C0E91D
:102F38000B33C0E90D33C36580F8253080F82430A1
:102F4800184638BD094B1344B3FBF1F308499B00FD
:102F5800CDE70120F5E700BF07040240F8FFFDBFF9
:102F6800000002403F82001000090240F8FBFDBF4C
:102F78000004024070B590F82450012D04463BD05F
:102F880090F825600125AE4280F824504FF00006E5
:102F98002CD1022580F825500568C6632E6826F0D6
:102FA80001062E60FFF7DEFE036BBBB12B6843F012
:102FB8000E032B60A36C1A68D20342BF1A6842F44E
:102FC80080721A60636D1BB11A6842F480721A60CD
:102FD8002B6843F001032B60002070BD2B6823F0A1
:102FE80004032B602B6843F00A03E2E78023C363E2
:102FF80080F824602846F0E70220EEE70A4A536981
:1030080043F4802330B55361EFF3108472B6002384
:10301800CD58C5500433B3F5807FF9D11369DB036C
:10302800FCD484F3108830BD00400058064B5A6920
:10303800002ABFBF054A9A6002F188329A60BABF77
:103048005869C00F002070470040005823016745A9
:10305800044B5A6942F000425A615869C043C00F94
:10306800704700BF0040005870B50546FEF712FCD7
:10307800124E04463369D90313D43369DA0744BFBF
:10308800012232614CF2FA32134011D10B4E3069F1
:1030980010F480200BD0FEF7FDFB001BA842F6D3EE
:1030A80004E0FEF7F7FB001BA842E3D3032070BD42
:1030B800024A1361024A01205360F8E700400058B1
:1030C800580400202DE9F041184D98462B78012B23
:1030D80006460C46174626D001232B704FF47A700B
:1030E80000236B60FFF7C0FFA0B9012E16D1104A6C
:1030F800536943F0010353612760BFF36F8FC4F82E
:1031080004804FF47A70FFF7AFFF094A536923EA46
:103118000603536100232B70BDE8F0813946204631
:10312800FFF76CFFEDE70220F6E700BF5804002028
:1031380000400058054A536923F47E7343EAC000EF
:1031480040F4803040F00200506170470040005861
:103158002DE9F041234F3B78012B054688463FD0A7
:1031680001233B704FF47A7000237B60FFF77CFFEC
:10317800044688B92B68042B13D11B4A536943F4BE
:10318800803343F0040353614FF47A70FFF76CFF08
:103198000446154B1A681B6800233B702046BDE89F
:1031A800F0814FF0FF33C8F800306E68D5E901327E
:1031B8001344B3420AD93046FFF7BCFF4FF47A7084
:1031C800FFF752FF50B1C8F800600446064A536939
:1031D80023F47E7323F002035361DAE70136E5E74F
:1031E8000224DBE758040020004000582DE9F04F86
:1031F800524C00234FF00F090A6832FA03F501D147
:10320800BDE8F08F012505FA03F818EA020200F07C
:103218008E804E68032706F003054FEA430E07FA2F
:103228000EFC6F1E012F6FEA0C0C32D8876807EA74
:103238000C0ACF6807FA0EF747EA0A07876047685B
:1032480027EA0808C6F300179F4047EA08074760BF
:10325800C76807EA0C088F6807FA0EF747EA0807F5
:10326800022DC76017D14FEAD30800EB880803F096
:10327800070AD8F820704FEA8A0A09FA0AFB27EAEF
:103288000B0B0F6907FA0AF747EA0B07C8F8207013
:1032980001E0032DDCD1076805FA0EF507EA0C07F3
:1032A8003D4316F4403F056041D023F0030707F182
:1032B800804707F5803703F0030CBD684FEA8C0C94
:1032C8004FF0070E0EFA0CFEB0F1904F25EA0E0EE5
:1032D8002FD01B4DA8422ED005F58065A84214BFFB
:1032E8000725022505FA0CF545EA0E05BD60256897
:1032F800D74316F4801F0CBF3D4015432560656811
:1033080016F4001F0CBF3D4015436560D4F880508B
:1033180016F4803F0CBF3D401543C4F88050D4F8E4
:103328008450B60354BF3D401543C4F8845001335C
:1033380062E70025D6E70125D4E700BF000800585A
:1033480000040048374A2DE9F04F00234FF0010AE6
:103358004FF0070B4FF00F0931FA03F401D1BDE824
:10336800F08F0AFA03FC1CEA010654D023F0030488
:1033780004F1804404F5803403F00307A568BF0016
:103388000BFA07F8B0F1904F08EA050E45D0264D24
:10339800A84244D005F58065A8420CBF0225072540
:1033A800BD40754517D1D2F8805025EA0605C2F808
:1033B8008050D2F8845025EA0605C2F88450156872
:1033C80025EA06051560556825EA06055560A568CD
:1033D80025EA0805A560056803265C0006FA04F4DA
:1033E80023FA06F6254300EB8606056003F0070579
:1033F800376AAD0009FA05F527EA050737628568D7
:1034080025EA04058560456825EA0C054560C56818
:1034180025EA0404C46001339EE70025C0E70125BE
:10342800BEE700BF00080058000400480AB18161E7
:10343800704781627047436901EA030221EA030188
:1034480041EA024181617047024A136843F480737C
:1034580013607047000400580D4B10B55B690C46AB
:1034680028B99A0507D500F027F820B110BD9B05AB
:1034780001D400F019F8074A1369012C23F004035A
:10348800136101D130BFF1E740BF20BF20BFEDE796
:103498000004005800ED00E0024B186800F4C0601A
:1034A800704700BF00040058024A136843F4804381
:1034B80013607047000400580C4A136823F48043D3
:1034C80013600B4B1B6832214B430A49B3FBF1F3E2
:1034D8005169890500D533B9536913F4007F14BFC6
:1034E800032000207047013BF2E700BF00040058AA
:1034F8007400002040420F000B4A136823F00703B2
:1035080043F002031360094B1A69012842F00402D0
:103518001A6105D130BF1A6922F004021A61704796
:1035280040BF20BF20BFF6E70004005800ED00E0D0
:103538004FF0B0431868C0F3404070474FF0B043B5
:103548001868C0F3400070474FF0B042536823F446
:103558007F4343EA0023536070474FF0B043186835
:10356800C0F34060704700007FB54FF0B0432C4A6D
:10357800D3F80831C0F3031003F00F0352F82040CA
:10358800284A52F82330B4FBF3F4FFF785FF264BA3
:10359800054693E80700B5F5007F04AB03E907008B
:1035A80010D0224B9C4218D303F5B70303F67F5380
:1035B8009C4229D903F5741303F510639C4225D85E
:1035C80002230BE01A4B9C4207D91A4B9C421BD989
:1035D80003F5370303F5D853F0E7002304AA02EBF9
:1035E800830353F80C4C144D2B6823F00703234333
:1035F8002B60FEF74FF906462B6803F007039C4241
:1036080006D1002004B070BD0123E7E70024EAE7F3
:10361800FEF740F9801B0228EED90320F2E700BF2D
:10362800E0EB000840EC0008F8EA0008C0CF6A00A8
:10363800BFEA21013F933402004000584FF0B043E5
:1036480010B59A68D96812F00C0205D00C2A4AD134
:1036580001F00303012B51D14FF0B0412B480B6807
:1036680013F0080306D00B6813F0080337D1D1F81C
:10367800941007E00C68240756BFD1F89430096805
:10368800C3F3032350F82330002A0CBF1846002048
:103698004FF0B0418A6802F00C020C2A1ED1CA68A9
:1036A80002F00302022A2ED0032A06D10B68184A18
:1036B80013F4801F174B18BF13464FF0B042D06861
:1036C800D168D268C0F306205843C1F3021301330E
:1036D800B0FBF3F0530F0133B0FBF3F010BD0B68F0
:1036E800C3F30313CEE7042A05D0082A06D11B68C2
:1036F80013F4801305D006480023C9E700231846B1
:10370800C6E70448C4E7024BD7E700BFE0EB000870
:103718000024F4000048E80108B5FFF78FFF4FF0D8
:10372800B043044A9B68C3F3031352F82330B0FB39
:10373800F3F008BD40EC00082DE9F04104460028EC
:1037480053D04FF0B0439D68DE6803689B0605F0D0
:103758000C0506F0030668D5026A1DB10C2D46D18A
:10376800012E44D1002A40D04FF0B043A16A1A6814
:10377800170756BFD3F894301B681B0903F0F003F2
:1037880099421FD90846FFF7EFFE00282DD14FF0C8
:10379800B042136843F0080313601368A16A23F06A
:1037A800F0030B431360606AFFF7CEFEFFF7B4FF28
:1037B800AB4B1860AB4B1868FEF76AF8002834D09A
:1037C800BDE8F0814FF0B042136843F0080313607E
:1037D800136823F0F0030B431360606AFFF7B4FE2D
:1037E8000846FFF7C1FE0028E0D00120E8E74FF0C7
:1037F800B043002A54D01A6842F001021A60FEF75A
:1038080049F80746FFF79AFE002842D04FF0B04229
:10381800136843F0080313601368A16A23F0F003E8
:103828000B431360606AFFF78FFE2368D80748D4FC
:103838002368990700F18C8023681E0740F1FA80FD
:10384800A3694FF0B046002B00F0E180D6F8943021
:10385800E16903F01002914200F0C48003F0030212
:10386800022AC2D0D80740F1B380D6F8943023F0AA
:103878000103C6F89430FEF70DF80746D6F89430E1
:10388800990740F1A580FEF705F8C31B112BF5D960
:1038980004E0FDF7FFFFC01B0228B3D903208FE720
:1038A8001A6822F001021A60FDF7F4FF0746FFF7D5
:1038B80045FE0028B9D0FDF7EDFFC01B0228F6D958
:1038C800ECE7082D03D00C2D05D1032E03D1636836
:1038D800002BADD189E74FF0B043A1681A6822F4F4
:1038E80080120A431A606268B2F5803F10D11A68E4
:1038F80042F480321A60FDF7CDFF0746FFF718FE45
:10390800002895D1FDF7C6FFC01B6428F6D9C5E786
:10391800B2F5041F04D11A6842F400121A60E6E7EF
:10392800196821F480311960196821F400111960AF
:10393800002AE0D1FDF7AEFF0746FFF7F9FD0028A2
:103948003FF476AFFDF7A6FFC01B6428F5D9A5E7BD
:10395800042D236903D00C2D0ED1022E0CD1002B7F
:103968003FF443AF4FF0B0426169536823F0FE4320
:1039780043EA016353605FE74FF0B046BBB1336879
:1039880043F480733360FDF785FF074633685A05B3
:1039980005D4FDF77FFFC31B022BF7D97EE77368B9
:1039A800626923F0FE4343EA0263736044E73368C5
:1039B80023F480733360FDF76DFF074633685B05BA
:1039C8007FF53AAFFDF766FFC31B022BF6D965E713
:1039D8004FF0B042E169D2F8943023F010030B4362
:1039E800C2F894304FF0B047D7F8943043F0010351
:1039F800C7F89430FDF74EFF0646D7F894309A077B
:103A080018D4FDF747FF831B112BF6D946E7D6F8E4
:103A1800943023F00103C6F89430FDF73BFF0746C6
:103A2800D6F894309B0705D5FDF734FFC31B112B3F
:103A3800F6D933E72368580754D50B4F3B68D905A7
:103A480014D4FFF701FDFDF725FF06463B68DA05AC
:103A58000CD4FDF71FFF831B022BF7D91EE700BF0D
:103A6800740000207800002000040058E3684FF03C
:103A7800B046002B58D023F08003052B02BFD6F8A0
:103A8800903043F00403C6F890304FF0B046FDF78D
:103A980001FFD6F8903043F001030746C6F890308E
:103AA80041F28838D6F890309B0705D4FDF7F2FE2E
:103AB800C31B4345F6D9F1E6E36823F00403812BE1
:103AC8001BD1FDF7E7FED6F8903043F08003C6F827
:103AD800903007464FF0B04641F28838D6F890301B
:103AE800180504D5E36A002B4AD1002068E6FDF7E3
:103AF800D1FEC01B4045F1D9D0E6FDF7CBFED6F884
:103B0800903023F08003C6F8903007464FF0B04657
:103B180041F28838D6F890301905E3D5FDF7BAFE9A
:103B2800C01B4045F6D9B9E6FDF7B4FED6F890308B
:103B380023F080030746C6F8903041F28838D6F85B
:103B480090301A0516D4FDF7A5FED6F8903023F06C
:103B58000103C6F8903007464FF0B04841F2883666
:103B6800D8F890309B07BDD5FDF794FEC31BB34230
:103B7800F6D993E6FDF78EFEC01B4045DFD98DE6EA
:103B88000C2D4ED0022B4FF0B0431A6822F08072F1
:103B98001A6033D1FDF77EFE0546FFF7DEFC38BB21
:103BA800D4E90C314FF0B0420B43D0682D490140A5
:103BB8000B43E16B0B43216C0B43616C0B43A16B13
:103BC80043EA0123D360136843F080731360D3681A
:103BD80043F08053D360FDF75DFE0446FFF7BDFC5C
:103BE800002882D1FDF756FE001B0A28F6D955E6B3
:103BF800FDF750FE401B0A28CFD94FE6FDF74AFED5
:103C08000446FFF7AAFC30B94FF0B042164BD16812
:103C18000B40D36069E7FDF73DFE001B0A28F0D989
:103C28003CE6012B3FF4E1AD4FF0B043D868236B7D
:103C380000F003029A427FF4D8AD626B00F0700383
:103C480093427FF4D2ADA26B00F4FE43B3EB022F94
:103C58007FF4CBAD636C00F06040C01A18BF012040
:103C6800AEE500BF8C80C111FCFFFEEE2DE9F041EE
:103C78000D46044610B90120BDE8F081684E33684E
:103C880003F007038B4216D323689A0727D54FF012
:103C9800B047A268BB6823F0F0031343BB60FDF78D
:103CA800F9FD0646BB68DB0319D4FDF7F3FD831B5A
:103CB800022BF7D911E0336823F007030B43336075
:103CC800FDF7E8FD0746336803F00703AB42DBD096
:103CD800FDF7E0FDC01B0228F5D90320CCE72368D7
:103CE800580617D54FF0B0476269D7F8083123F066
:103CF8000F0343EA1213C7F80831FDF7CBFD064658
:103D0800D7F80831D90305D4FDF7C4FD831B022B6E
:103D1800F6D9E2E723685A0713D54FF0B047E268AF
:103D2800BB6823F4E0631343BB60FDF7B3FD0646AD
:103D3800BB689B0305D4FDF7ADFD831B022BF7D9A8
:103D4800CBE72368180714D54FF0B0472269BB6842
:103D580023F4605343EAC203BB60FDF79BFD0646AC
:103D6800BB68590305D4FDF795FD831B022BF7D9D2
:103D7800B3E72368DA070FD4294C236803F0070355
:103D8800AB4239D8FFF7C8FC264B1860264BBDE874
:103D9800F0411868FDF77CBD6268022A1DD1FFF763
:103DA800C7FB00283FF467AF4FF0B04641F28838B0
:103DB800B36823F003031343B360FDF76BFD0746B5
:103DC800B368626803F00C03B3EB820FD4D0FDF73D
:103DD80061FDC01B4045F3D97FE7032A02D1FFF7F5
:103DE800BCFBDEE712B9FFF7A9FBDAE74FF0B043F7
:103DF8001B685B05D8D43EE7236823F007032B43F1
:103E08002360FDF747FD0646236803F00703AB422E
:103E1800B8D0FDF73FFD801B0228F5D95DE700BF4C
:103E280000400058740000207800002008B5FFF713
:103E380073FC4FF0B043044A9B68C3F3022352F863
:103E48002330D84008BD00BF20EC000808B5FFF7B4
:103E580063FC4FF0B043044A9B68C3F3C22352F893
:103E68002330D84008BD00BF20EC00084FF0B04315
:103E7800D3F89000C0F3400070474FF0B0410209FA
:103E8800D1F8883002F47F22000123EA020300F40B
:103E98007F200343C1F8883070474FF0B041020CCF
:103EA800D1F88830120423EA020343EA0040C1F83B
:103EB800880070470368DA0370B5044639D5FFF700
:103EC800C3FAFDF7E7FC614E05463368DB0532D5DA
:103ED8004FF0B043616BD3F8902002F440729142E6
:103EE8001DD0D3F89010D3F8902042F48032C3F854
:103EF8009020D3F8902021F4407022F480328D076E
:103F0800C3F89020C3F8900009D5FDF7C3FC41F22F
:103F180088360546FFF7AAFF012840F090804FF049
:103F2800B042616BD2F8903023F440730B43C2F86F
:103F38009030002605E0FDF7ADFC401B0228C4D9EF
:103F480003262568E8070AD54FF0B0416268D1F822
:103F5800883023EA124392B21343C1F88830A90784
:103F68000AD54FF0B041A268D1F8883023EA12434D
:103F780092B21343C1F88830AA0609D54FF0B0426F
:103F88002169D2F8883023F440630B43C2F88830A3
:103F9800AB0502D5206AFFF780FF680502D5606A85
:103FA800FFF77BFF290502D5A06AFFF776FF6A06AF
:103FB80002D56069FFF761FF2B0602D5A069FFF7FC
:103FC8005CFFE80502D5E069FFF757FFE90610D561
:103FD8004FF0B042E168D2F8883023F440730B43C5
:103FE800C2F88830B1F5807F02BFD36843F0807390
:103FF800D3602A040ED54FF0B042216BD2F8883036
:1040080023F040430B43C2F8883019B9D36843F012
:104018008073D3606B0410D54FF0B042E16AD2F8D8
:10402800883023F040530B43B1F1005FC2F8883069
:1040380003D1D36843F48033D360304670BDFDF7B5
:1040480029FC401BB0427FF665AF79E700040058B1
:1040580030B590F82C30012B02464FF0020022D0E8
:10406800174B82F82D00CA24012582F82C505C6277
:1040780053245C62B1F5807F146B996914D121F4E3
:1040880088519961596C24F0010421F00041596468
:104098001463DD650A4BFF2159620020012382F871
:1040A8002D3082F82C0030BD21F408519961D96C6B
:1040B80024F0020421F00041D9641463D865E9E7CB
:1040C8000028004070B50B4E036B756D1D40EA0764
:1040D800044603D50123F365FDF7EFFCAB0704D5D0
:1040E8000223F365204600F0C9F9012384F82D3036
:1040F80070BD00BF0028004038B50A4CE36823F0C3
:104108002003E360FDF7C6FB0546E3689B0601D57F
:10411800002038BDFDF7BEFB401BB0F57A7FF4D90F
:104128000320F6E700280040F8B5114DEC6814F0BC
:10413800400406461AD1EB6843F08003EB60FDF7B4
:10414800A9FB23460746EC6814F0400401D1032B71
:1041580001D11846F8BDFDF79DFBC01BB0F57A7F6D
:10416800234684BF032386F82D30ECE70023F0E7CD
:104178000028004038B50F4CE36823F08003E36063
:10418800A3699B06054606D4FFF7B6FF10B10320C6
:1041980085F82D0038BDA36923F02003A361FFF73C
:1041A800ABFF10B1032085F82D00A36943F020036D
:1041B800A361EFE70028004038B5044600284BD03B
:1041C80090F82D3003F0FF021BB980F82C20FDF782
:1041D800CBF90223214D84F82D30EB68DB0636D469
:1041E800CA236B6253236B622046FFF79DFF10B111
:1041F800FF236B6238BDAB6923F08E6323F0400365
:10420800AB6121696368AA690B431343A26913432D
:10421800AB61D4E9022343EA02432B61D4E90931B3
:10422800EA680B4322F4F8521343EB602046FFF789
:10423800A1FF0028DCD1D4E90713AA690B4322F0B7
:104248006042134362691343AB61FF236B6201232E
:1042580084F82D300020CDE70120CBE7002800406E
:104268000023092803D840EA0310C0B270470A386F
:104278000133C0B2F5E700002DE9F04790F82C3083
:10428800012B05464FF0020069D0012385F82C3038
:104298004E4B85F82D00DE6806F44076B6F5807F33
:1042A80078D04C69087891F8019091F802A091F8BB
:1042B8002470002A55D19B6913F0400308BFCB70C6
:1042C800FFF7CEFF80464846FFF7CAFF0246504632
:1042D800FFF7C6FF81463846FFF7C2FF0B6ACF7863
:1042E800234343EA875343EA090343EA084343EA7B
:1042F800022343EA0063354ACA20506253205062C1
:104308008C6A8869B4F5807F946945D124F488540F
:1043180094610124D465B6F5807F09BFCB69136425
:104328000343536418BF5064284B4A681A672A6BC2
:1043380042F001022A639A6942F488529A61244A37
:10434800D2F8803043F40033C2F880301F4BFF228C
:104358005A620020012385F82D3085F82C00BDE82D
:10436800F087B4F1803F07D0B4F5000F04D09B6903
:1043780013F0400308BFCB700B6ACA781C4344EAA9
:104388000A0444EA004343EA092343EA825343EA1E
:104398000763B0E70023AEE724F4085494610224CD
:1043A800D465B6F5807F09BFCB6993640343D364B2
:1043B80018BFD064054B4A685A672A6B42F002025C
:1043C8002A639A6942F40852B8E700BF00280040FF
:1043D8000008005890F82C20012A03464FF00200EC
:1043E80012D00A4A83F82D00CA2151625321516222
:1043F800916941F020019161FF2151620020012261
:1044080083F82D2083F82C00704700BF0028004057
:1044180090F82C20012A03464FF0020019D00D4ACB
:1044280083F82D00CA2151625321516291690A48CB
:1044380041F080019161D0F8801041F48021C0F8EA
:104448008010FF2151620020012283F82D2083F87B
:104458002C0070470028004000080058064B5A6D91
:10446800520610B5044603D54022DA65FDF728FB4D
:10447800012384F82D3010BD0028004070478900C2
:1044880001F1804101F531410A607047890001F16D
:10449800804101F53141086870470000034AD2F8AD
:1044A800903043F40043C2F890307047000400583D
:1044B800034AD2F8903023F40043C2F89030704792
:1044C80000040058074B1A6822F040021A6040F4B2
:1044D80041704FF4B85218605A601A6842F04002AE
:1044E8001A6070470000015837B5054600284ED0BD
:1044F800837903F0FF046BB1032C0BD0254B4FF4E9
:1045080000629A612868FFF7DDFF002401232B7100
:10451800AC602FE000236B712846FDF7D5F81E4AE2
:10452800D2F8903043F48053C2F89030002CE5D193
:1045380002234FF0B042AB71D2F8943023F4004319
:10454800C2F89430154B1B681C214B43DB0C6421CB
:104558004B430193019B93B90124AC60FFF79EFF85
:104568000C4B9A6842F400629A604FF400629A61B8
:10457800002CC7D00123AB71204603B030BD019B8E
:10458800013B0193D2F894305B04E3D4E6E70124BD
:10459800F2E700BF0004005800080058740000202B
:1045A80037B5174D2B6802461C204343DB0C6420AB
:1045B800434314480193019B93B901209060114C27
:1045C80021732B681C214B43DB0C64214B43019363
:1045D800019B6BB9012090600A4BDB6803B030BDCA
:1045E800019B013B019383689C07E4D50020E6E723
:1045F800019B013B0193A368DB07E9D5ECE700BF0A
:10460800740000200000015837B5184D2B68024689
:104618001C204343DB0C6420434315480193019B52
:10462800A3B901209060124CFF2323732B681C252B
:104638006B43DB0C64256B430193019B73B9012029
:1046480090600B4BDB680B7003B030BD019B013BE6
:10465800019383689C07E2D50020E4E7019B013BB6
:104668000193A368DB07E8D5EBE700BF74000020DF
:10467800000001580E4B0F491B681822534382B0A3
:104688001B0D6422534301934B69019AC3F38003C2
:1046980022B902238360012002B07047019A013ACF
:1046A80001924A69920701D5002BEDD10020F3E76A
:1046B800740000200004005807B50379012B0FD1BE
:1046C8000A4B1B68182253431B0C0193FFF7F0FE9B
:1046D800019B013B0193019B002BF9D1FFF7DEFE03
:1046E80003B05DF804EBFFF7C5BF00BF74000020FE
:1046F800F8B51E468379012B154604460F46DAB2F3
:104708002DD14379012B2AD0022342718371FFF7FF
:10471800D3FF0D212046FFF7CBFEFFF741FF390AF3
:104728002046FFF73DFFF9B22046FFF739FF2E4438
:10473800B5420ED12046FFF7B1FEFFF79BFFA068F8
:1047480001230038A3714FF0000318BF01206371E3
:10475800F8BD15F8011B2046FFF722FFE8E7022005
:10476800F6E7F8B51E468379012B154604460F4631
:10477800DAB22FD14379012B2CD04271FFF79CFF7D
:104788001D212046FFF794FEFFF70AFF390A20464D
:10479800FFF706FFF9B22046FFF702FF0021204687
:1047A800FFF7FEFE2E44B5420ED12046FFF776FEF7
:1047B800FFF760FFA06801230038A3714FF00003E2
:1047C80018BF01206371F8BD29462046FFF71CFF7A
:1047D8000135E8E70220F6E7F8B51F468379012B93
:1047E800154604460E46DAB22CD14379012B29D05E
:1047F8004271FFF761FF06F0EF03A3F18402534211
:104808005341237131462046FFF752FEFFF7C8FE99
:104818002F44AF4210D1FFF741FE842E02D020462C
:10482800FFF728FFA06801230038A3714FF00003A9
:1048380018BF01206371F8BD15F8011B2046FFF76A
:10484800AFFEE6E70220F6E7F8B51E468379012BAE
:10485800154604460F46DAB227D14379012B24D0F6
:104868004271FFF729FF39462046FFF721FEFFF77F
:1048780097FE00212046FFF793FE2E44B5420ED145
:104888002046FFF70BFEFFF7F5FEA068012300386E
:10489800A3714FF0000318BF01206371F8BD2946CA
:1048A8002046FFF7B1FE0135E8E70220F6E737B505
:1048B8000023ADF8043001AA022312210546FFF7B0
:1048C800C3FFBDF80440022364BA01AAA4B2194682
:1048D8002846FFF781FFE20702D5284609F0B4F918
:1048E800A30702D5284609F0B5F9600702D528467E
:1048F80009F0DAF9210702D5284609F0DBF9E206C2
:1049080002D5284609F0DCF9A30602D5284609F0A5
:10491800C5F9600602D5284609F0A2F9210606D590
:1049280014F4807118BF0121284609F09FF9A205E7
:1049380002D5284609F0AAF9630402D5284609F0E9
:10494800C5F903B030BDF8B51E468379012B15466D
:1049580004460F46DAB227D14379012B24D042719D
:10496800FFF7AAFE0E212046FFF7A2FDFFF718FE6B
:1049780039462046FFF714FE2E44B5420ED1204694
:10498800FFF78CFDFFF776FEA06801230038A371BE
:104998004FF0000318BF01206371F8BD15F8011B23
:1049A8002046FFF7FDFDE8E70220F6E7F8B51E46CA
:1049B8008379012B154604460F46DAB22BD1437989
:1049C800012B28D04271FFF777FE1E212046FFF702
:1049D8006FFDFFF7E5FD39462046FFF7E1FD0021B1
:1049E8002046FFF7DDFD2E44B5420ED12046FFF7E5
:1049F80055FDFFF73FFEA06801230038A3714FF073
:104A0800000318BF01206371F8BD29462046FFF74F
:104A1800FBFD0135E8E70220F6E7026852E8003FAF
:104A280023F0C00342E8003102680029F5D102F101
:104A3800080353E8003F23F4000302F1080C4CE894
:104A480000310029F3D12023C0F8883070470000D6
:104A580010B5026852E8003F23F4907342E8003131
:104A680002680029F5D10F4C02F1080353E8003F12
:104A7800234002F1080C4CE800310029F4D1C36E40
:104A8800012B07D152E8003F23F0100342E8003120
:104A98000029F7D12023C0F88C300023C366436770
:104AA80010BD00BFFEFFFFEF38B50546C8B124238F
:104AB800C0F8883003681A68002422F001021A60DE
:104AC8001C605C609C60FDF7A7F8C5F8904085F80D
:104AD8008440C5F888402046C5F88C40EC662C67B1
:104AE80038BD0120FCE70000F8B504461346D4F8A9
:104AF8008850202D32D1F1B1EAB1E06FA4F85620E8
:104B0800A4F8542000262122C4F890602165C4F836
:104B18008820226888B1124FC762124F0763124F6C
:104B28002832C0E90D76FEF725FA30B11023C4F813
:104B38009030C4F888500120F8BD236840221A62DA
:104B4800226802F1080353E8003F43F0800302F1B2
:104B5800080141E800300028F3D1EDE70220EBE737
:104B6800754B0008BD4B0008C94B000808B5034643
:104B7800806A1B681B6813F0200317D1A0F8563011
:104B8800026802F1080353E8003F23F0800308326B
:104B980042E8003102680029F2D152E8003F43F0B0
:104BA800400342E800310029F7D108BDFDF7AEF80F
:104BB800FBE7704708B5806AFFF7FBFF08BD704741
:104BC800806A38B50468D0F88830D0F88C50A2686C
:104BD800120606D5212B04D10023A0F85630FFF782
:104BE8001CFFA3685B0606D5222D04D10023A0F87C
:104BF8005E30FFF72DFFD0F8903043F01003C0F877
:104C08009030FFF7DCFF38BD70470000D0F88C20EB
:104C1800B0F86010222A08B5036855D15B6A826D26
:104C28000B401370836D01338365B0F85E30013B30
:104C38009BB2A0F85E30B0F85E309BB2002B42D138
:104C4800026852E8003F23F4907342E80031036899
:104C58000029F5D103F1080252E8002F22F00102E1
:104C680003F1080C4CE800210029F3D12022C0F8F8
:104C78008C20184A41679342016705D1C26E012A08
:104C88000ED0FDF751F81EE05A681102F6D553E828
:104C9800002F22F0806243E800210029F7D1EDE7D8
:104CA8000022C26653E8002F22F0100243E80021D8
:104CB8000029F7D1DA69B0F85C10D20644BF102297
:104CC8001A62FFF7A1FF08BD9A6942F008029A61CB
:104CD800F9E700BF00800040D0F88C20B0F86010E1
:104CE800222A08B5036852D15A6A1140826D22F807
:104CF800021B8265B0F85E20013A92B2A0F85E20ED
:104D0800B0F85E2092B2002A40D153E8002F22F476
:104D1800907243E800210029F7D103F1080252E814
:104D2800002F22F0010203F1080C4CE800210029B1
:104D3800F3D12022C0F88C20174A416793420167BB
:104D480005D1C26E012A0ED0FCF7EEFF1EE05A68AC
:104D58001102F6D553E8002F22F0806243E80021C3
:104D68000029F7D1EDE70022C26653E8002F22F0B0
:104D7800100243E800210029F7D1DA69B0F85C1085
:104D8800D20644BF10221A62FFF73EFF08BD9A6997
:104D980042F008029A61F9E7008000402DE9F84FD7
:104DA8000368B0F86060D3F81CB01F689D68D0F83D
:104DB8008C20222A044640F0B980B0F8683043B10C
:104DC800DFF87491DFF874A14FF000081BF0200F92
:104DD80020D1B4F85E309BB2D3B1B4F868209A42BF
:104DE80016D9226802F1080353E8003F23F08053E4
:104DF800083242E8003122680029F2D1504B63673B
:104E080052E8003F43F0200342E800310029F7D17F
:104E1800BDE8F88F2368A26D5B6A33401370A36DF9
:104E28000133A365B4F85E30013B9BB2A4F85E3051
:104E38002368D3F81CB01BF0070F2ED01BF0010F0E
:104E480009D0F90507D501221A62D4F8902042F05A
:104E58000102C4F890201BF0020F09D0EA0707D519
:104E680002221A62D4F8902042F00402C4F890207A
:104E78001BF0040F09D0E80707D504221A62D4F8FA
:104E8800903043F00203C4F89030D4F8903023B146
:104E98002046FFF794FEC4F89080B4F85E309BB2C9
:104EA800002B93D1226852E8003F23F4807342E834
:104EB800003123680029F5D103F1080252E8002FD8
:104EC80002EA090203F1080040E800210029F3D1B1
:104ED80020225345C4F88C20616721670AD05A689C
:104EE800110207D553E8002F22F0806243E8002121
:104EF8000029F7D1E26E012A14D10022E26653E8B4
:104F0800002F22F0100243E800210029F7D1DA69C6
:104F1800B4F85C10D20644BF10221A622046FFF78C
:104F280073FE53E72046FCF7FFFE4FE79A6942F00D
:104F380008029A616CE700BFFEFFFFEF00800040A7
:104F4800154C00082DE9F84F0368B0F86060D3F8F5
:104F58001CB01F689D68D0F88C20222A044640F0B7
:104F6800B780B0F8683043B1DFF87091DFF870A10E
:104F78004FF000081BF0200F20D1B4F85E309BB230
:104F8800D3B1B4F868209A4216D9226802F108030E
:104F980053E8003F23F08053083242E8003122688A
:104FA8000029F2D14F4B636752E8003F43F02003DA
:104FB80042E800310029F7D1BDE8F88F2368A26DD7
:104FC800596A314022F8021BA265B4F85E20013A02
:104FD80092B2A4F85E20D3F81CB01BF0070F2ED0B5
:104FE8001BF0010F09D0F90507D501221A62D4F880
:104FF800902042F00102C4F890201BF0020F09D063
:10500800EA0707D502221A62D4F8902042F0040277
:10501800C4F890201BF0040F09D0E80707D5042234
:105028001A62D4F8903043F00203C4F89030D4F8F0
:10503800903023B12046FFF7C2FDC4F89080B4F841
:105048005E309BB2002B95D1226852E8003F23F4D2
:10505800807342E8003123680029F5D103F1080282
:1050680052E8002F02EA090203F1080040E8002193
:105078000029F3D120225345C4F88C2061672167A9
:105088000AD05A68110207D553E8002F22F080622F
:1050980043E800210029F7D1E26E012A14D1002249
:1050A800E26653E8002F22F0100243E800210029AD
:1050B800F7D1DA69B4F85C10D20644BF10221A623C
:1050C8002046FFF7A1FD55E72046FCF72DFE51E7E6
:1050D8009A6942F008029A616EE700BFFEFFFFEF8F
:1050E80000800040E14C000838B504460368216997
:1050F800A2681D68C0690A4361690A437749024387
:1051080029400A431A605A68E16822F440520A4367
:105118005A60734AA16993421CBF226A11439A6874
:1051280022F06E4222F430620A439A60DA6A616AB7
:1051380022F00F020A43DA626A4A934219D14FF009
:10514800B043694AD3F8883003F0030343F440338B
:10515800934200F0B480B3F1031F24D0013A934284
:1051680040F0B580B0F5004F40F08F80FEF766FA4A
:105178006EE05E4A93421CD14FF0B0435C49D3F8CD
:10518800883003F00C0343F440228A4200F09780F1
:1051980006D8002B7CD0574B9A42E3D0012026E05A
:1051A800B2F10C1FFAD1B0F5004F53D04FF40040C4
:1051B80075E04B4A9342F1D14FF0B043D3F88830B1
:1051C80003F44063B3F5006F18D006D85BB1B3F5AC
:1051D800806FE3D1FEF732FA07E0B3F5406FDDD117
:1051E8004FF400400BE0FEF721FE40B900204FF0DD
:1051F8000113A3660023C4E91D3338BD3E48656822
:105208003E4B626A05EB450133F81220B0FBF2F31E
:105218009942C3D8B3EB053FC0D800231946FBF722
:10522800BFFC090241EA10616B080002C0182A4657
:105238004FF0000341F10001FBF7B2FC304BA0F541
:1052480040729A42AAD82368D860CFE7FEF7EEFDED
:105258000028CBD06168294B626A33F81220B0FB72
:10526800F2F24B0803EB42034FF6EF72B3FBF1F394
:10527800A3F11001914291D823F00F02216892B254
:10528800C3F342031343CB60B0E7FEF7D7F904E05A
:10529800B0F5004FDAD0FEF7C9FD0028A6D0636844
:1052A800616A164A32F81120B0FBF2F000EB5300A5
:1052B800B0FBF3F04FF6EF73A0F11002C1E7B0F5C1
:1052C800004F0D48EBD1C5E7FEF7C0FDC0E7B0F5CC
:1052D800004FF9D0FEF7BAFDDFE700BFF369FFCF53
:1052E80000800040003801400200030000440040F4
:1052F80008000C0004000C000024F40080EC0008F6
:10530800FFFC0F00836ADA0710B506D50168C46A86
:105318004A6822F4003222434A609C0706D5016895
:10532800046B4A6822F4803222434A60590706D542
:105338000168446B4A6822F4802222434A601A07B3
:1053480006D50168846B4A6822F4004222434A6009
:10535800DC0606D50168C46B8A6822F480522243B1
:105368008A60990606D50168046C8A6822F400529E
:1053780022438A605A060FD50168446C4A6822F4B1
:1053880080122243B4F5801F4A6005D14A68846CB4
:1053980022F4C00222434A601B0606D50268C16C8B
:1053A800536823F400230B43536010BD2DE9F843E1
:1053B800DDF8209005460F46164698462A68D369B8
:1053C80037EA03030CBF01230023B34201D00020B6
:1053D80029E0B9F1FF3FF2D0FCF75CFAA0EB080036
:1053E80048452C6802D8B9F1000F1ED154E8003F97
:1053F80023F4D07344E80032002AF7D104F10803FB
:1054080053E8003F23F0010304F1080141E80032AA
:10541800002AF3D12023C5F88830C5F88C30002342
:1054280085F884300320BDE8F88323685A07C5D57A
:10543800E3691B05C2D54FF40063236254E8003FBB
:1054480023F4D07344E80032002AF7D104F10803AA
:1054580053E8003F23F0010304F1080141E800325A
:10546800002AF3D12023C5F88830C5F88C30C5F858
:105478009030D4E773B504460026C0F89060FCF776
:1054880009FA23681B681A07054619D423681B689C
:105498005B070AD56FF07E43009300222B464FF43A
:1054A80080012046FFF782FFB0B900202023C4F80E
:1054B800883084F88400C4F88C30E06620670CE0FB
:1054C8006FF07E430093324603464FF400112046A6
:1054D800FFF76CFF0028D9D0032002B070BD10B5CB
:1054E800044650B3D0F888301BB980F88430FCF7F4
:1054F80023FB22682423C4F88830136823F00103AF
:1055080013602046FFF7F0FD012816D0A36A13B1F7
:105518002046FFF7F7FE23685A6822F490425A6043
:105528009A6822F02A029A601A6842F0010220461C
:105538001A60BDE81040FFF79DBF012010BD0000B4
:1055480030B581658168A0F85C200023B1F5805FE3
:10555800A0F85E20436735D10369002B40F2FF13A2
:1055680018BFFF23A0F860300023C0F89030222332
:10557800C0F88C30016801F1080353E8003F43F09C
:105588000103083141E800340368002CF2D1456E6C
:1055980084680169B5F1005F32D1B0F8685095426E
:1055A8002ED8B4F5805F244A03D1244C002908BFC3
:1055B80022464267B1B153E8002F42F4807243E8B3
:1055C8000021F7E729B90369002B14BF7F23FF23C4
:1055D800C8E7B1F1805FC5D10369002B14BF3F2331
:1055E8007F23BFE703F1080252E8002F42F0805200
:1055F80003F1080040E800210029F3D1002030BD64
:10560800B4F5805F0E4A03D10E4C002908BF22462C
:10561800426741B153E8002F42F4907243E80021F9
:105628000029F7D1EAE753E8002F42F0200243E8C7
:1056380000210029F7D1E1E7A54D00084D4F0008EA
:10564800154C0008E14C0008D0F88C30202B30B401
:1056580015D1B9B1B2B100230468C3660A4B9C42A4
:105668000AD063681B0207D554E8003F43F0806303
:1056780044E80035002DF7D130BCFFF761BF0220A8
:1056880030BC70470120FBE700800040436E30B516
:105698002BB90123A0F86A30A0F8683030BD036840
:1056A800094D9A689968094C490FC2F342626B5CCC
:1056B800615CDB00B3FBF1F3A0F86A30AB5CA25C81
:1056C800DB00B3FBF2F3E7E7A0EC000898EC000876
:1056D8001FB504AB03E9060090F88430012B04469B
:1056E8003AD0012380F884302423C0F88830036836
:1056F8001A6822F001021A609A6822F440120A43DA
:105708009A6071B95A68BDF80C009DF80E1022F025
:10571800100202435A605A6822F07F4242EA01624C
:105728005A601A6842F001021A60FCF7B3F86FF089
:105738007E42034600924FF4800100222046FFF784
:1057480035FE38B92023C4F88830002384F8843023
:1057580004B010BD0320F8E70220F9E790F8843080
:10576800012B0FD0012380F88430016851E8002F05
:1057780042F0020241E80023002BF6D180F8843081
:10578800184670470220704710B590F88430012BF6
:10579800044617D02423C0F8883003681A681968AB
:1057A80021F00101196042F000524FF000514166AA
:1057B8001A60FFF76BFF2023C0F88830002084F8B8
:1057C800840010BD0220FCE770B590F88430012BEE
:1057D800044617D005682423C0F888302E682B6843
:1057E80023F001032B60AB6823F060431943A960E1
:1057F800FFF74CFF20232E60C0F88830002084F883
:10580800840070BD0220FCE738B5084D052455F822
:10581800043B2BB9013C14F0FF04F8D1204638BDF5
:10582800DB6898470028F5D0F9E700BFAC050020F1
:10583800034BD870034B1B681B6C03B118477047A8
:105848009405002090050020034B1874034B1B6837
:105858005B6C03B118477047940500209005002041
:10586800F0B5314D314B95F90420314E91B00C46CD
:10587800012795F905108DF8047002288DF8092084
:105888008DF80A1010D18DF80800D8711C7202F03A
:1058980063FD337803B114B101A803F0C1F9254BB6
:1058A800059A1A6011B0F0BD59714FF480711A71E0
:1058B800D9801C7233788DF8087053BB1F2306A853
:1058C8008DF81C208DF8183002F024FF20238DF865
:1058D800183006A82B798DF81C3002F01BFF222304
:1058E8008DF8183006A86B798DF81C3002F012FF7D
:1058F80021238DF8183006A86B798DF81C3002F03A
:1059080009FF29238DF8183006A80B4B079302F0DE
:1059180001FF02F021FD012306A88DF818308DF84B
:105928001C3002F0F7FEB4E794050020AC0000201C
:105938007004002064050020000400017FB50923DD
:1059480001A88DF8043003F06BF90038044B059A70
:105958001A6018BF0120404207B05DF804FB00BF81
:105968006405002070B504460B46144962784A70F5
:105978000020A2780A7208701A884A729A788A7285
:10598800DB780B746368CB600D4B1B68DA6A2AB14D
:10599800237803F0FB030A2B00D09047094E00251B
:1059A80056F8043B1BB15B6A0BB12046984701359A
:1059B800EBB2052B6DB2F3D170BD00BF7C000020A7
:1059C80090050020AC05002070B50446114801235D
:1059D800037063784370A3788372E368C360E378E5
:1059E800037623694376237943720B4B1B689B6AC2
:1059F80003B19847094E002556F8043B1BB19B6933
:105A08000BB1204698470135EBB2052B6DB2F3D1A7
:105A180070BD00BF9000002090050020AC0500205C
:105A2800014B1868704700BF6405002000B58BB0B3
:105A3800012368468DF8003002F046FD38B99DF81C
:105A48000400003818BF01200BB05DF804FB0020EB
:105A5800FAE7000008B501F037FE40B9FFF7E6FFA6
:105A6800012806D0054B197AD879FFF7F9FE0120ED
:105A780008BDBDE80840FFF7C7BE00BFAC00002066
:105A88002DE9F04186B005460E46174601F01CFE8A
:105A9800002873D101F030FE044640B9FFF7C6FF75
:105AA80001280AD03D4B197AD879FFF7D9FE6FF053
:105AB8000204204606B0BDE8F081DFF8E48088F8EB
:105AC8000860003E18BF01268DF80460354E6878DE
:105AD80033798DF81230694602F094FC00283FD0E3
:105AE8008DF804400394ADF810406FF0060495E873
:105AF80003002D4B83E80300337988F80A303946D0
:105B080001A803F091F9294B059A1A6011283FD88A
:105B180001A353F820F000BF8B5B0008855B0008E9
:105B2800995B0008995B0008995B0008995B00087D
:105B3800995B0008B75A0008995B0008995B000850
:105B4800995B00087F5B0008995B0008995B000877
:105B5800855B0008855B0008855B00089F5B000883
:105B68002B788DF808306B78ADF810306B6803939C
:105B78004FF0FF34BBE76FF005049AE76FF00104BC
:105B880097E70B4B00221A70E31D18BF144690E7E5
:105B98004FF0FF348DE76FF004048AE7AC00002073
:105BA8009000002094050020A0000020640500203B
:105BB8006305002037B501F0A9FD134D052455F8FC
:105BC800043B4BB11A693AB19B682BB1984718B19D
:105BD80055F8043C1B699847013C14F0FF04EED1CA
:105BE800FFF712FE68B9094D2B7853B1084BADF891
:105BF8000040D978019422466846FFF741FF00B972
:105C08002C7003B030BD00BFAC0500206305002038
:105C18009405002030B58BB0044601F055FD0546CB
:105C2800002835D1FFF702FF012834D168468DF8E6
:105C3800005002F049FC40BB9DF80430A34204D058
:105C4800012C22D0022C12D014B100200BB030BD90
:105C5800002BFAD068468DF8044002F05BFDA0B92D
:105C68000E4B1B681B6B002BEFD09847EDE763B911
:105C780068468DF8044002F04DFD30B9074B1B68AB
:105C88001B6B002BE1D02046EFE74FF0FF30DDE73C
:105C98006FF00100DAE76FF00200D7E79005002007
:105CA80010B504468AB018B94FF0FF300AB010BDDD
:105CB800002368468DF8003002F006FC0028F3D176
:105CC8009DF804302370F1E77FB500220B46204988
:105CD8008DF8072001220A7042784A700446002A8B
:105CE80033D102790A721A884A729A788A72DB78F2
:105CF8000B740369CB60C378164D8DF80830037BAD
:105D08008DF80930836803932B68DB6A0BB102A80E
:105D180098472B689B6B13B1227E02B198470E4EB1
:105D2800052556F8043B1BB1DB690BB120469847A3
:105D3800013D15F0FF05F4D10DF10700FFF7B0FFA5
:105D4800637913B1054B01221A7004B070BD00BF0E
:105D58007C00002090050020AC0500206305002091
:105D680010B504468AB018B94FF0FF300AB010BD1C
:105D7800202368468DF8003002F0A6FB0028F3D1F6
:105D8800024A9DF9043023701371EFE7940500204F
:105D980000B58BB02323019068468DF8003002F0DF
:105DA800B9FC003818BF012040420BB05DF804FB75
:105DB80070B5654C01468EB01822204606F0C0F832
:105DC800624B00221A70FCF773FA237840680122AC
:105DD80002FA03F1014004D15D4B084608F09CF833
:105DE800FEE75C495C481A4602F0F8F818B14FF033
:105DF800FF300EB070BD272304A88DF8103002F0D4
:105E080089FC564E564D002870D1012333702B68FB
:105E1800DB690BB100209847272304A88DF81030C0
:105E280002F052FB059B93F84820227093F8182142
:105E380093F81A316270A370464BD3E9020105F05A
:105E48006FFF05460028D2D1464E062304A88DF8D8
:105E5800103002F039FB059B736104A802F05AFC6C
:105E6800022304A88DF81030059602F02DFB0836A1
:105E7800032304A88DF81030059602F025FB0F26A1
:105E880006F014F8012304A88DF814308DF810607A
:105E980002F040FC10230DEB03008DF810308DF854
:105EA800145002F037FC04238DF8103004A8A378AE
:105EB8008DF8143002F02EFC3A238DF8103004A827
:105EC8006369059302F026FC02A920788DF8086022
:105ED80004F09CF8003818BF0120E0711420FFF787
:105EE80057FFE07903F062F9284682E728238DF806
:105EF80010302B681B6943B104A802F0E5FA2B683F
:105F080005981B6940F2C4519847272304A88DF8C7
:105F1800103002F0FFFB50B9012304A88DF81030AF
:105F280002F0D2FA9DF81430002B7FF46EAF33786C
:105F3800002B7FF46CAF052204A88DF81020059380
:105F480002F0E8FB78E700BF940500206305002015
:105F5800A8EC0008680500208005002070040020D7
:105F680090050020D005002037B500230D46019389
:105F78000446D0B900F0A8FB0190019BD3B10F4AA9
:105F880042F824300E4A9A620E4A1268916B1963DD
:105F9800916C596392690C49D9625A6128465B68C9
:105FA8000A49F2229847002006E001A900F092FB76
:105FB8000028E2D04FF0FF3003B030BDAC05002020
:105FC8006958000890050020455900087104002010
:105FD800194B07B51860194B194A1A60194A5A60C3
:105FE800194A9A60194ADA60194B02681A604268BD
:105FF8005A6082689A60C268DA60164A1A618269D1
:106008005A61154BC26B5A60144A019119609A6023
:106018001946134ADA600020FFF7A6FF48B901A81D
:1060280000F056FB003818BF0120404203B05DF86D
:1060380004FB4FF0FF30F9E79005002080050020B1
:10604800D1590008D15C0008E56000086D590008C6
:1060580068050020C59F0008C005002039580008C1
:106068005158000849B118B1012804D000207047E0
:10607800034B0B60FAE7034BFBE74FF0FF30704729
:10608800000400010100010208B503F0ABF8002884
:1060980014BF6FF00100002008BD08B502F084F9B4
:1060A800002814BF6FF00100002008BD10B5044699
:1060B8008AB018B94FF0FF300AB010BD21236846E6
:1060C8008DF8003002F000FA0028F3D1024A9DF959
:1060D800043023705371EFE7940500202DE9F04157
:1060E8002F4D304F00232B7043786B703B689B6AB1
:1060F8008AB004460BB128469847DFF8AC800026E2
:1061080058F8043B1BB11B6A0BB12046984701366F
:10611800F3B2052B76B2F3D12378052B2FD00B2BB6
:1061280035D0012B25D1214C062368468DF8003047
:1061380002F0CAF90199E07905F038FE10B91C4B54
:10614800019A5A611B48FFF70BFE1B48FFF7AEFF89
:106158006B788BB9A371194B5878FFF75BFD3B68D7
:106168005B6A0BB1114898476B7813B9E07905F071
:10617800AFFE0AB0BDE8F081FF23A371EFE7104B33
:1061880001225A74227A9A74627ADA74F1E763788F
:10619800002BEED00AB0BDE8F041FFF7CFBB00BF3F
:1061A8009000002090050020AC050020AC000020E5
:1061B800D0050020B0000020B10000209405002088
:1061C8007C00002030B58BB0FFF767FF0446F0B9BC
:1061D80003F0FCFE831C1DD0F8B9134D2B685B69D6
:1061E800DBB1272368468DF8003002F06DF92B6883
:1061F80001985B694FF4B961984703F0F9FE78B9E3
:106208002CB9094B1B68DB690BB101209847204664
:106218000BB030BD6FF00704EFE74FF0FF34ECE749
:106228004FF0FF34F3E700BF90050020014B1878CA
:10623800704700BF04060020014B5878704700BF24
:106248000406002070470000044B9A7A0AB1012224
:106258005A70034B5B6903B1184770470406002066
:10626800B800002073B5224C6378002B33D008F0B7
:106278003BF966680546FFF7D3FB0644AE4214D2E5
:10628800A37A93B1E0228DF800208DF80130217AAD
:10629800E368019301226846FFF7F2FB08B1073073
:1062A80010D100236370A372656094F83430EBB1A9
:1062B800002384F834300F4B5B6BBBB102B0BDE8F0
:1062C8007040184740F2DC510B4808F0D9F90A48E9
:1062D80008F09CF9E8E794F83520002AE5D094F80E
:1062E800360084F83530FFF795FCDEE702B070BD64
:1062F80004060020B8000020E805002037B5104D3E
:10630800104CC8B1C1B16272012300222860E1605B
:1063180023700D480D4B00924FF0FF3108F0CAF87A
:1063280000250B4825822022294605F01DFE6570B0
:10633800A574A58603B030BD00232B602370EFE75A
:106348000006002004060020E8050020516200082D
:10635800180600202DE9F0478E4C23788CB0002BCE
:1063680056D0C2780AB9837B13B1238A01332382BA
:10637800437B002B4CD0E02A4AD10023A3728768C4
:1063880097F80080B8F1220F27D8B8F1220F30D83B
:10639800DFE818F04100FB0052005A0061006E006F
:1063A80075008E009D00B400C7002F002F002F003D
:1063B8002F002F002F002F002F002F002F002F005D
:1063C8002F002F002F002F002F002F002F002F004D
:1063D8002F002F00C900D000D400B8F17E0F00F0C4
:1063E800CC80B8F17F0F00F0DF80B8F17D0F00F0AE
:1063F800AB80A57A002D00F05B81674C637A3BB9CE
:106408004FF47A71204608F03BF9204608F0FEF870
:106418000CB0BDE8F087E36801220021A272197070
:10642800A37AE1689818A0720620C854A37AE16894
:106438009818A072CA54DCE7584B9B6A002BD8D036
:10644800012102209847D4E77B7884F8363001236D
:1064580084F83530CDE704238DF804307B78003B91
:1064680018BF012301A88DF8083002F053F9C0E7DE
:106478007878003818BF012002F098FEB9E7484E36
:106488000FCE01AD0FC50FCE0FC596E8070085E802
:1064980007007B780A2BACD8424A12685268002A57
:1064A800A7D00CA901EB830353F82C0C9047A0E765
:1064B8007878431E012B9CD83A4B01381B6818BFCB
:1064C800012020729B68002B93D0984791E7E268DF
:1064D80001230821A3721170627A057BA17AAA426E
:1064E80028BF2A46934284D285685A1CEB5CE5682B
:1064F80001334E1CA6726B54D3B2EDE7E368012258
:10650800A27209221A70A37AE268218A581CA07222
:10651800D154A27A238AE1681B0A501CA0728B54BA
:1065280067E7238265E705238DF8043001A802F0A8
:1065380077FB5EE7194BDB6A98475AE7194B78787F
:106548001B686075DB68BEE7037B072B7FF451AFE0
:1065580006238DF80430B7F80130ADF808307B79A0
:106568003A791B0443EA0223FA781343642253431B
:106578000393BB798DF81030D8E73B2201A88DF83A
:1065880004208DF8083002F0C5F8012384F834306F
:106598002FE700BF04060020E8050020B80000200F
:1065A80004EB0008000600202A2301A88DF8043017
:1065B80001F08AFF94F80A90E6689DF808009DF8B3
:1065C80009509DF80A709DF80BC09DF80D309DF894
:1065D8000E209DF80F109DF80CE009F1010A84F8CF
:1065E8000AA006F80980354E94F80A903668D4F85F
:1065F8000C8009F1010A84F80AA096F803A008F8AB
:1066080009A094F80A90D4F80C8009F1010A84F8DA
:106618000AA096F802A008F809A094F80A90D4F8FD
:106628000C8009F1010A84F80AA096F801A008F87C
:1066380009A094F80A9009F1010A84F80AA096F8CA
:106648000080E66806F8098094F80A80E66808F190
:10665800010984F80A9006F808C094F80AC0E668A8
:106668000CF1010884F80A8006F80C70A77AE6682D
:1066780007F1010C84F80AC0F555A57AE6686F1C85
:10668800A7727055A07AE568461CA6722954A17AAB
:10669800E0684D1CA5724254A27AE168501CA072B1
:1066A8008B54A37AE268591CA17202F803E0A0E6B1
:1066B800034807F05DFF6570AAE600BF00060020EA
:1066C800E80500207047000000487047B800002027
:1066D800002070474FF0FF3070470000044B054A18
:1066E80093F81831022B18BF062382F890347047AC
:1066F800A80C00206C120020034BD3F8483313B1C8
:106708005B6903B1184770476C120020034A13787D
:1067180043F004031370FFF7EFBF00BF50060020DB
:106728001FB50A4B8DF8090093F87C208DF80A20D4
:1067380093F88C2093F848000D3202A98DF80820B0
:1067480003F064FCC0B205B05DF804FBA80C00209F
:1067580008B5074807F00CFF064B93F81A2412B146
:10676800012283F81924BDE80840FFF7C5BF00BF20
:106778006C1600206C12002010B50C4CD4F8403375
:1067880043F08003C4F8403394F81A3413B100205E
:10679800FFF7DEFF94F8913423F0120343F012035D
:1067A80084F89134BDE81040FFF798BF6C120020C0
:1067B8002DE9F041DFF8AC8098F81831022B064635
:1067C8000D4602D0284BDB6A984702F0A6FD044626
:1067D80028B1022002F097FD002002F099FD98F8F8
:1067E8001831012B17D102F09AFD074630B100206D
:1067F80002F08AFD002002F08CFD3C4602F091FD7B
:1068080048B1002002F081FD002002F083FDBDE8C0
:10681800F041FFF763BF002CF9D1144C94F8902491
:1068280094F81A34BAB90BB184F84164304602F0CE
:1068380017FFD8F82C0007F061FED4F8B43398425B
:10684800E5D30B4807F094FE94F8913443F0100315
:1068580084F89134DBE70BB184F84154284602F000
:10686800FFFEF1E7A80C002024F400086C120020B9
:1068780004160020074A10B5137843F0020313707A
:10688800FFF73AFFBDE81040034B01220021022028
:1068980007F042BB50060020F1EC0008074A10B58B
:1068A800137843F008031370FFF726FFBDE8104084
:1068B800034B01220021022007F02EBB50060020C6
:1068C80001ED00082DE9F0410F4616461D468046A9
:1068D80007F00AFE0B4A0C4C1378278123F01103AA
:1068E80043F01103C4E90008137066812573FFF7AC
:1068F80003FFBDE8F041054B01220021022007F00B
:106908000BBB00BF500600203C06002011ED00081C
:1069180013B507F0E9FD0D4B6C461860204607F0EB
:1069280037FD94E803000A4A0A4B83E8030013780A
:1069380043F020031370FFF7DFFE074B012200210D
:10694800022002B0BDE8104007F0E6BA4C0600206D
:1069580050060020A41500201EED00082DE9F04186
:1069680092B0064602F0D9FC002840F05881AD4D9F
:1069780095F81831012B09D02B6BAB4C93B194F8D7
:106988000431BBB1042B6FD0032003E002F0C7FC35
:1069980018B10F2012B0BDE8F08102F0C2FC002847
:1069A800EAD0F6E7B5F82031D4F81C24013B53436C
:1069B8002B63E4E79D4803F060FA002840F0128159
:1069C80094F80C3123802B6B0C930DF1180895F873
:1069D80039308DF83830404695F81C318DF83A300A
:1069E80007F0FCFCD5F82831009302AF98E80600C0
:1069F800D5F82431384607F088FC97E803000FAB38
:106A080083E80300EB6A0D9300238DF84430238854
:106A1800ADF8463095F8303101228DF839201BB990
:106A28008DF844208DF83930814B0093814B95F8CF
:106A38004800A3F179020CA903F05DFBC0B10B2853
:106A4800A8D1D4F8941499B1002EA3D0D4F8403327
:106A5800794843F02003C4F8403307F011FE764824
:106A680007F0D4FD002095E7704803F03AFAA4E750
:106A780095F8487095F9693095F9392095F87D10A1
:106A88006E4E384603F044FB009641B2EB6C95F825
:106A980050203846183603F0DFFA0096EB6C95F86C
:106AA800502095F9701095F8480003F0D5FAD4F8FD
:106AB800C413AB6DD4F8DC230B44C4F8B033EB6DCE
:106AC8001344C4F8B43394F80431042B07D02B6E64
:106AD8000B44C4F8B0336B6E1344C4F8B4330023CA
:106AE800089395F83031002B40D100238DF81330EE
:106AF80095F839308DF8213095F838308DF82230F6
:106B0800D5F880300993D5F884300A932388ADF8F6
:106B18002C3095F8303194F81B648DF82E3095F8A8
:106B28004800474B8DF820600DF1130208A903F0C7
:106B3800A7FA012384F8413495F8393084F84234AF
:106B48009DF8133084F84334D4F81C34C4F85064E6
:106B5800C4F84834C4F8583402F0E5FBC8B1D4F896
:106B68001C0402F0F2FBA0B1102013E708A802F001
:106B7800A7FC60B995F9390094F837629DF8207040
:106B8800FFF7CEFD3E44B042AFD2082002E7132003
:106B980000E795F81831012B01D102F0D8FB02F07B
:106BA800C5FB0023059394F8043195F9395094F8FE
:106BB8001B649BB1042B7FF4E7AE05A802F0B4FE7A
:106BC80058BB94F8183413B1059B013B0593174B38
:106BD80005983246E9B202F00DFF02E0134802F0D0
:106BE800DDFE08B11120D5E6D4F8403394F80C1135
:106BF800218043F00203C4F8403394F81834114854
:106C08000133DBB284F8183484F845340E4B002580
:106C18009B6AC4F89854984724E71220BAE60E20D5
:106C2800B8E600BFA80C00206C12002074130020E6
:106C3800D80C002000170020D415002024160020AE
:106C4800881600206E12002024F4000873B5134D36
:106C5800134E0096EB6C95F8502095F9781095F83E
:106C6800480003F0F9F995F83031337595F8480084
:106C780040F2012306F13C023146738203F0F8F931
:106C880050B196F83C3086F88230064B00205B6B9A
:106C98009847F37C86F8A83002B070BDA80C002095
:106CA8005416002024F40008F8B5324C94F8183132
:106CB800012B05460ED0022B4ED0002B57D138B9E8
:106CC800D4E91B0104F1740383E803000020F8BD34
:106CD800012806D102F02CFB0028F8D184F81851BD
:106CE800F5E7022843D1244E84F8180106F5747C90
:106CF800BCE80F0006F57A770FC79CE8030094F804
:106D0800E92094F8003187E8030086F8FB53D2B1F4
:106D1800022B18D1D4F804316367C6F8EC3394F821
:106D28007D3094F8082186F8F83394F88C3084F88C
:106D3800782086F8F93396F81B2486F8E82340F281
:106D48000133A6F8FA33002386F81A340B4BDB6AB2
:106D58009847FFF77BFFB9E748B9074B84F8180154
:106D6800062283F89024054BDB6A9847AEE7032098
:106D7800ADE700BFA80C00206C12002024F4000826
:106D8800F0B5504C504EB4F8DC202287D4E92D01E0
:106D980094F8B12084F8692004F16C0282E80300B9
:106DA800D4E92F0104F1740282E80300B4F8C42086
:106DB800A4F87C2091B0D4F8CC20D4F8C810C4F83A
:106DC80084200025D4F8D020C4F888200123A4F812
:106DD8002031C4F8801084F83051A56284F81B5122
:106DE80084F83A5084F81D5184F81E51C4F834517F
:106DF800C6F89854A6F8185486F81A54A4F83851C6
:106E08008DF8183004F50973039304F50A7394F8A0
:106E18004800049303A92D4B84F84551C4E94F5504
:106E2800A4F84651059303F0FFF8E36EC6F8D4338F
:106E380094F87D3086F8E03394F88C3086F8E133A6
:106E48004FF48073A6F8E23386F8D05394F83031C3
:106E580086F8E43306F574770FCF06F57A740FC415
:106E680097E8030040F2012384E80300A6F8FA3308
:106E7800D6F8483386F81B54CDE901551BB15A683A
:106E88005B6901920293124B0793A3F1480208929F
:106E9800A3F1140209920F4A0B9229330A93A2F123
:106EA8009C030C93A2F198030D93131D0E9301A953
:106EB80002F14C0307A802F599620F9302F022FA37
:106EC80011B0F0BDA80C00206C1200205406002060
:106ED800D41600208C0D0020F8B50D4F0D4E0C4631
:106EE80007F046FB3B6B98470B4A96F8480021464B
:106EF80003F0BEF850B1094D706D95F8243485F84B
:106F08006A347B6B9847E37C85F89034F8BD00BF02
:106F180024F40008A80C0020901600206C12002011
:106F28000F4890F81B3480F8B8330E4B93F869205B
:106F380080F8BB2393F87D2080F8C82393F88C2031
:106F480080F8C92393F8303180F8CC330022A0F8B8
:106F5800CA2300F56E7100F56070FFF7BDBF00BF72
:106F68006C120020A80C0020114890F89034EBB166
:106F780090F81B3480F8D0330E4BDA6EC0F8D42367
:106F880093F87D2080F8E02393F88C2080F8E123A3
:106F980093F8303180F8E4334FF48072A0F8E2239C
:106FA80000F5747100F56670FFF796BF704700BF73
:106FB8006C120020A80C002070B5344C2421204607
:106FC80004F0D4FF636A984218BF60624FF01C0156
:106FD8002F4814BF0125002504F0C8FF636C9842B0
:106FE80018BF60644FF480712A4818BF45F0020545
:106FF80004F0BCFFD4F84831984218BFC4F84801DF
:107008004FF0D401244818BF45F0040504F0AEFF42
:10701800D4F82032984218BFC4F820024FF000017B
:107028001E4818BF45F0080504F0A0FFD4F8243224
:10703800984218BFC4F824024FF46071184818BF6A
:1070480045F0100504F092FFD4F8A835984218BF0F
:10705800C4F8A8054FF01401124818BF45F02005E0
:1070680004F084FFD4F8C03598420F4B18BFC4F819
:10707800C005D3F8483318BF45F040052BB11B694C
:107088001BB12846BDE87040184770BDA80C002009
:10709800D00C0020F00C0020F40D0020CC0E0020B5
:1070A800D00E0020541200206C1200202DE9F04F61
:1070B8008FB04FF00009012B06460F4690468DF819
:1070C8000D90ADF8109002D84C46BC4202D30FB0D8
:1070D800BDE8F08F305D02F033FA2044B842F6DCA8
:1070E800335D651C023BEDB2112BF0D801A252F8BA
:1070F80023F000BF457100086F7100086D72000829
:107108009572000813730008397300089F7300080C
:10711800C77300084D740008D7700008D7700008BE
:10712800A1740008D7700008D770000849750008D6
:1071380071750008A9750008DD750008052002F0C2
:10714800A7FA70B10521002002F068FA725DBA4B07
:10715800E51C0234E4B283F85C24325D83F85D24D4
:10716800EDB22C46B1E700238DF80E308DF80F30C4
:107178008DF814308DF81830B9F1000F6DD1AF4C7F
:107188004FF0050994F87C208DF831206B1E94F897
:1071980039208DF83320334494F838200B938DF838
:1071A800342094F81A3194F868208DF83520D4F8F2
:1071B8002C218DF832300A9273B37B1C5B1BDBB237
:1071C8008DF8303006AB019305AB009394F8480076
:1071D8000DF10F030DF10E020AA902F05DFF8DF803
:1071E8000D0000F00700072813D194F939209DF904
:1071F8000E3084F839309A429DF80F3084F83830D0
:10720800B8BF01229DF81430B8BF84F81D2184F856
:1072180068304FF0000A09E00523D1E701220DF19B
:107228000D01032002F0A4F80AF1010A5FFA8AF2BC
:107238009DF81830B3FBF9F19142EFD82B44DDB239
:107248006B1EDBB29F420BD9F25C032A9AD0AF4285
:1072580088BF1D464FF0010983E70534E5B2F9E719
:107268001D46F7E7735D754903F00F03012281F8A6
:107278001B31023402FA03F3A1F82031E4B20022F0
:1072880004A9042002F074F825466AE707238DF85C
:107298000D30735DC3F3021203F00F038DF828302D
:1072A800E31CDBB28DF82920F25C231DDBB2651DDF
:1072B800F35C0234E4B21B0443EA0223325D5F4C00
:1072C80013436422534394F848000B930AA902F02D
:1072D800F2FE00F00703072BEDB28DF80D000CD17C
:1072E8009DF8283084F8703084F878300B9BE3667A
:1072F80063679DF8293084F869308DF81000012201
:1073080004A9052002F034F82BE74B4BD3F8483397
:1073180063B11B6853B1984708F03F038DF810001C
:107328008DF81130022204A90620EBE7FF20F3E7CD
:1073380003238DF80D30735D8DF81C300AAB06936E
:10734800E31CDBB2A51DF25C231DDBB206A9F35CCE
:107358001B0443EA0223A21CD2B20534B25C1343D5
:1073680064225343E4B20A9300230B93335D8DF8F0
:107378003030324B93F8480002F0A3FEC3B2002825
:10738800EDB28DF80D30FFF6ECAE8DF8103001221D
:1073980004A90720B6E7735D03F00F03012B4FF430
:1073A8007A7238BF01235343244A0234936503F5A4
:1073B8007A73D365E4B2002204A9082062E7735DFA
:1073C8001E4DC3F340128DF8152095F84800C3F3FD
:1073D800001205A903F00F038DF814208DF816305C
:1073E80002F075FE02340130E4B23FF44DAFBDF84F
:1073F8001430134AA5F87C309DF816309DF814A077
:10740800D05CF9F7DFF90223C5F880000AA995F8DE
:1074180048008DF828308DF82AA002F0F7FD95F97C
:107428003930069040B29842B8BF184685F83900FE
:10743800002204A9092025E76C120020A80C0020CE
:107448002BED000803238DF80D30735D8DF828307F
:10745800E31CDBB2651DF25C231DDBB20234F35C76
:10746800E4B21B0443EA0223325D1343642253430C
:107478000B93644B0AA993F8480002F02EFEC3B29E
:107488000028EDB28DF80D30FFF66BAE8DF8103098
:10749800012204A90A2035E7092002F0F9F8DFF8EB
:1074A80068B1002849D00921002002F0B7F800236C
:1074B800ADF81E30A31CDBB2F25CE31CDBB216F89D
:1074C80003A0735D4FEA0A4A4AEA022A4AEA030A13
:1074D800231DDBB2A51D0534F35CE4B24AEA036A56
:1074E800335D4FF47A7253430AAC1B122046ADF851
:1074F8001C3006F04DFF454B53440693DBF83C33F4
:1075080000930DF1180A9AE80600DBF8383308A84A
:1075180006F0FBFE099B009394E80600089B504682
:1075280006F0D8FE9AE8030006F00AFF01F00AFF09
:107538000123EDB28BF8383413E68BF8380410E6E3
:107548000C2002F0A5F800283FF40BAE0C21002017
:1075580002F064F82C4B93F89034043B012B7FF62F
:1075680000AE01F0EBFEFCE5A31CDBB2725DF15C42
:10757800E31CDBB2651DF35C0434E4B21B04305D2C
:1075880043EA012313436421594300F00F0001F03B
:10759800D6FEEDB28DF81000012204A91120B1E643
:1075A8000D2002F075F800283FF4DBAD0D21002016
:1075B80002F034F8A31CDBB2154AF05C735D126864
:1075C800251D0334E4B243EA0020315DEDB201F039
:1075D800B8FEC6E5725DA31C251D0334DBB2E4B218
:1075E800F15C335D1B0443EA0123134364205843D1
:1075F80001F0A9FEEDB28DF81000012204A91320B4
:1076080080E600BFA80C00206C120020803DD51237
:107618003C0600200E4B93F89124920703D593F86B
:107628008F24012A08D90B4991F81A2122B18A6AB4
:10763800501C18BF01328A620022A3F8182483F86C
:107648001A24D3F8402322F00202C3F840237047DB
:107658006C120020A80C002070B5184C1848194D61
:1076680006F086FFD4F84033D4F89804D5F8906033
:1076780023F02003C4F8403338B106F03FFF8642B8
:1076880003D2002385F83A3070BD0120FFF766F970
:107698000028F9D00B28F7D095F8393084F842340F
:1076A800092094F8183484F8453484F8410401F02A
:1076B800D7FFBDE87040FFF7ADBF00BF6C120020D8
:1076C800D4150020A80C0020094BD3F84023012A28
:1076D8000AD008490978C90708D43AB993F8920436
:1076E800013818BF012070470020704701207047FB
:1076F8006C12002050060020034BD3F84003431EB1
:1077080058425841704700BF6C1200202DE9F04FD5
:10771800A9B0EFF3108272B6DFF8F0B20021DBF8FF
:107728000030CBF8001082F31088B94C002B00F021
:10773800E180DAB29B06039264D5B64D95F818310C
:10774800022B02D0B44BDB6A9847EFF3108872B66D
:10775800B24F06F0C9FE3E68D4F8B013361A314469
:10776800AF4806F08DFFAE4806F050FFD4F8B413CA
:10777800AC48314406F084FFAA4806F047FF88F376
:10778800108894F81A34002B00F06B81152312A985
:1077980095F848008DF8483002F038FCD4F8B41356
:1077A8000F900144A04806F06BFF9F4806F02EFF9B
:1077B8003B6894F81B24EB620DAF38468DF87020B7
:1077C8001D9306F00BFED5F82831009306AE97E816
:1077D8000600D5F82431304606F097FD96E80300F8
:1077E8001FAB83E80300D4F81C341E9395F830319E
:1077F80095F84800003B18BF01231CA98DF871308B
:1078080002F00DFC039BDF0648D5824DDFF81CA271
:10781800D5F8E42004929BF80020BAF90A809AF976
:107828000C90A4F88C84002363F300020A9384F874
:107838004434A4F8223484F82534C4F82834A4F84D
:107848002C3484F82E34C4F8303484F82034C4F846
:10785800343484F83834C4F83C346F4B8BF8002047
:1078680094F89024DB6A84F88E9484F88F24DAF8EC
:107878000470BAF80860984794F88F3413B96948C7
:1078880006F076FE3146384601F045FD834600286D
:1078980000F0EA80A4F87E8484F88094039B19079A
:1078A8001AD55C4B93F81831022B02D05A4BDB6A7D
:1078B80098470220FEF712FF84F8410401F0D0FE39
:1078C80094F81A3413B1012384F8193494F89134D4
:1078D80043F0100384F89134039B5A0703D506211B
:1078E8000520FEF765FF039B9B0703D504210320B2
:1078F800FEF75EFF01F02DFD94F89124D7065FD5C1
:10790800002384F89234D4F840331E0644BF23F091
:107918008203C4F8403312F0050F00F0FB820B20FD
:1079280001F0B6FE002800F0F58294F89134DD07E6
:1079380000F1F082580740F10783D4F8403323F070
:107948000203C4F84033D4F8402382BB94F891541E
:1079580015F001011EBF2B4662F3000384F8913431
:1079680094F891345E0744BF6FF3820384F891342E
:10797800012384F8923421B1D4F844332C481B688D
:1079880098476D070BD52B4801F08EFE01F0BCFE21
:1079980028B194F8913443F0040384F8913401F049
:1079A800C6FC94F891346FF3041384F891340123DE
:1079B80084F8923494F8913443F0200384F8913495
:1079C80094F8913418070AD56FF3C3031A4984F859
:1079D8009134D4F84433A1F12400DB68984794F833
:1079E800913499070AD56FF34103134984F8913408
:1079F800D4F84433A1F16C005B68984794F890344C
:107A0800022B1BD1FFF722F918E000BF5006002017
:107A18006C120020A80C002024F400084C0600205A
:107A2800EC150020041600206C1600203C060020EF
:107A3800AC160020C0160020F816002094F89134E7
:107A48009A0640F1C4826FF3451384F89134D4F850
:107A58004033002B40F0BB8229B0BDE8F04FFFF760
:107A6800ABBA84F84134A3E695F81831012B0CD150
:107A780001F055FC804668B1584601F045FC58466F
:107A880001F047FC042384F88F347EB9012384F87D
:107A980021344FE101F045FC0028F6D0404601F0C2
:107AA80034FC404601F036FC0523ECE73B780593AF
:107AB8005B09013B062B00F21782DFE813F0070091
:107AC800150295001502920015020602102EDDD946
:107AD80095F830311297F6B28DF84C60002BD5D15D
:107AE8001CA804F055F912AA1CA9FF2002F09EF860
:107AF8009DF85830C3F3030307468DF82C3095F8EA
:107B0800480095F87D308DF82D3007220BA902F03A
:107B180090FA002F5DD100285BD09DF853309DF876
:107B280052201599C5F8E4101B0443EA02239DF876
:107B3800512002201343C5F8E03004F037F99DF8CE
:107B4800583095F8480085F82E71C3F30212C3F334
:107B5800030385F8703085F878309DF8593085F83A
:107B68006920012B38BF01234FF47A725343AB6568
:107B78001344EB650DF15A034FF001081093113EC1
:107B880094F81B348DF83C300FA985F868808DF87F
:107B9800446002F056FA0223404685F8303101F07D
:107BA80077FD18B14146384601F038FD94F88F3416
:107BB800012B00F2A78194F81A34002B40F09A8127
:107BC80094F8913443F0100384F89134FEF786FD5D
:107BD80064E6012001F05CFD0028E7D001210720C0
:107BE800E2E7012384F8203495F87D308DF82E30B3
:107BF80094F824348DF82D3095F88C3095F8480099
:107C08000D330BA98DF82C3002F000FAA6F10D0304
:107C18001BB2099023EAE37300B283423FF736AF01
:107C28000B2E7FF633AFBA4B25931CA8FF231C9766
:107C38008DF874608DF8983002F0C4F80746002873
:107C48007FF424AF95F81831012B13D101F067FBAD
:107C5800002872D0384601F057FB384601F059FB2E
:107C680004239DF87C101E9884F88F34C1F300110A
:107C780001F06EFB9DF87C301E99C4F8341413F0A3
:107C88000F0203D09DF89000002862D19DF898005B
:107C9800002861D0002A7FF4F9AE9DF89020002AD0
:107CA80014BF4FF003084FF0020800220A92D5F8DB
:107CB800EC2095F8E900914251D100284FD0D5F831
:107CC8000C1195F8EAB009680A9195F8181102297B
:107CD80002D1032184F88F14B8F1030F7FF4D6AED4
:107CE80013F0600F7FF4D2AE0492012795F82E317D
:107CF800BBF1000F36D0BBF1010F13D1012B33D1EB
:107D08006FF0090646FA08F606F00106C6F1020603
:107D1800F6B2BDF87E100AAA304601F011FE38B35B
:107D2800072823D0012384F821340A9BC4F830346F
:107D3800C4F86C34FEF720FDB0E501F0F2FA002833
:107D480098D0384601F0E1FA384601F0E3FA052305
:107D580087E74FF00008A8E74FF00108A5E74FF0C4
:107D6800010BC3E70426D4E70326D2E70823DAE7A2
:107D78001CAB009304990A9B3246584601F0A2FEB8
:107D880020B1022814BF0B230A2380E60A9BC4F8FB
:107D98003034C4F86C349DF87C3084F82104C3F383
:107DA800401384F82E3484F8443494F88F3484F8DB
:107DB8002274012B9EBF0122A86285F81E21012F83
:107DC800C4F8280484F82C0484F8410438D1022229
:107DD80084F8202495F83A20002A4AD19DF87C207E
:107DE800D60646D4012B94F840149DF87C2005D87B
:107DF800012901D1900601D501F04CFBB8F1020F21
:107E080094F88F3443D0B8F1030F0AD09DF87C1052
:107E1800B8F1010F4A4601F00F0120A83BD0FFF747
:107E280045F99DF8903084F82334259BC4F828340C
:107E38009DF8983084F82C34012384F82D3430E0F0
:107E4800059A02F0E002A02A1BD195F82E11012212
:107E580085F83A2009B927996963012B84F8202409
:107E680007D9D5F89020C4F83C24DAF80020C4F8E3
:107E7800982495F81821002AB4D1012284F82524E1
:107E8800B0E7002285F83A2084F82024A6E79DF878
:107E9800981025984A46FFF709F99DF8903084F81C
:107EA80023349DF89020E02A08D195F81F312BB98A
:107EB80084F82324C4F82834A4F82C3494F8913492
:107EC80043F0020384F8913470E6114D013EB2B2DA
:107ED800791C284604F034F80323A4F82034C4F8A5
:107EE800285484F82C64E9E7012384F82134FEF748
:107EF80043FC5BE694F84434002B3FF461AE002069
:107F0800FEF726FC94F88F34022B3FF45FAE57E659
:107F1800A414002094F89134590715D5012001F0D4
:107F2800B7FB60B1012001F08BFB08B984F8180495
:107F3800D4F8403323F00203C4F8403304E00620A9
:107F480001F0A6FB0028F3D194F89134DA077FF505
:107F5800FAAC94F840240AB1032A18D11D4A94F8BF
:107F6800181492F86820914205D29B0723D594F8FB
:107F78008F34012B1FD8184806F0FAFAD4F840338A
:107F880023F02003C4F84033FFF744FBDBE4012A65
:107F980011D194F81924002A3FF4D5AC0D4A94F86D
:107FA800181492F868209142E5D29F0703D594F8F7
:107FB8004434002BDFD194F8913400206FF304137C
:107FC80084F8913484F81904FFF746FBBBE429B020
:107FD800BDE8F08FA80C0020D41500202DE9F04F43
:107FE80089468DB090460746002800F08F81002909
:107FF80000F08C810368002B00F088814368002B17
:1080080000F084818368002B00F08081C368002B16
:1080180000F07C81104601F0F5FF002800F078811F
:10802800BD4CBE4D384601F0AFFA40F2C4520021B3
:10803800204603F099FF40F21C520021284603F025
:1080480093FFB74BC4F82C3104F50973089304F572
:108058000A7300264046099308A9B24B84F8488061
:108068000A9384F8186184F88C608DF82C6001F00C
:10807800DBFF0F2306A994F848008DF8183001F0AB
:10808800C5FF801B18BF01204FF00A0B84F81C01A4
:1080980006A994F848008DF818B001F0B7FF4FF022
:1080A800060A84F8DC0006A994F848008DF818A0A0
:1080B80001F0ACFF102384F8DD0006A994F848000D
:1080C8008DF8183001F0A2FF1123C4F89C0006A90E
:1080D80094F848008DF8183001F098FF1223C4F87E
:1080E800A00006A994F848008DF8183001F08EFF1A
:1080F8001323C4F8A40006A994F848008DF8183092
:1081080001F084FF1423C4F8A80006A994F84800D5
:108118008DF8183001F07AFF1623C4F8AC0006A9D0
:1081280094F848008DF8183001F070FF172384F890
:10813800B10006A994F848008DF8183001F066FFE0
:1081480018230DEB0301C4F8B400C4F8BC0094F87C
:1081580048008DF8183001F059FFC0B21D2384F88B
:10816800B80084F8C00006A994F848008DF81830C3
:1081780001F04CFF1E2384F8C40006A994F84800B7
:108188008DF8183001F042FF1F2384F8C50006A9B6
:1081980094F848008DF8183001F038FF2023C4F80F
:1081A800C80006A994F848008DF8183001F02EFF91
:1081B8000B23C4F8CC0006A994F848008DF81830B1
:1081C80001F024FF0C2306A9A4F8D00094F8480075
:1081D8008DF8183001F01AFFD4F89C306365D4F894
:1081E800A030A365D4F8A430E365D4F8A83023669A
:1081F8004FF00108D4F8AC300590A4F8D2006366BB
:1082080084F8B080C4F894B084F898A0C4F84CB04E
:1082180084F850A084F8688084F81F81C5F84893D2
:10822800FEF7AEFDC5F84473C4E90B663E4B84F80F
:10823800198185F89164C5F8408332464FF0FF31C3
:10824800009605F55A7006F035F9384B0096324617
:108258004FF0FF3105F5607006F02CF9344B0096AD
:1082680032464FF0FF3105F5667006F023F902AF8C
:10827800304B009632464FF0FF3105F5806006F02E
:1082880019F9384606F0AAF897E8030004F592733E
:1082980083E80300284B294F1E60294BC5F84C334F
:1082A800284BC5F85433284BC5F85C33274BC5F821
:1082B8005033274BC5F8583305F553703B6898473A
:1082C80004F5A67003F080FB20B1112630460DB0EE
:1082D800BDE8F08F204601F003FB0028F5D101F03E
:1082E80039F8B8B91B4801F04DFB06460028ECD117
:1082F8007B69984703F002FEBB6D94F81901984713
:10830800FB6A9847012385F89234DFE70326DDE707
:108318000926DBE71326D9E7A80C00206C120020F9
:10832800000400015406002061760008296F000847
:10833800716F0008596700085006002024F40008EF
:1083480019690008CD68000815670008A5680008C5
:108358007D680008900D002008B5034B0020C3F885
:108368004003FEF7BBF908BD6C12002010B5FFF7FB
:10837800ABF90A4C60B90A4B93F81831022B02D1B9
:10838800084BDB6A98470123C4F84033002010BD2E
:10839800D4F84003013818BF0120F8E76C12002018
:1083A800A80C002024F4000838B5124C204606F02A
:1083B800DFF804F1180006F0DBF804F1300006F0ED
:1083C800D7F804F1980006F0D3F800F0AFFF0A4B95
:1083D8000025DB6A984744F8285CFEF7EDFD07495D
:1083E800074840F2C45203F0ABFD012344F8283C8F
:1083F800284638BDD415002024F40008A80C002015
:10840800E406002070B52E4B8AB0054693F8DD00CF
:108418008DF8090093F8DC008DF80A0029489A6A5B
:1084280090F81804039200268DF80B0004960C4669
:10843800002940D00692D3F8882007921A8F93F823
:108448001A118DF8151052BAADF8202093F87C2037
:1084580093F848308DF8243003AB8DF822008DF85E
:10846800232000930DF10A020DF10B030DF1090110
:1084780005A88DF8146000F0D7FE9DF90900FEF7F5
:108488004FF9607004A801F01BF8B0B9049A0F2ADC
:108498000DD863789A420AD81544AB42A3EB02017F
:1084A8002CBF002001202170C0000AB070BD00233D
:1084B80023700820F9E70320F7E71320F5E700BF4A
:1084C800A80C00206C1200201FB50446002800F0FC
:1084D80010810378412B00F20781DFE813F0420096
:1084E80049004D005100550059005E000501050185
:1084F8000501050105010501050105016500690082
:108508006D0078007F00820085008A0088008C005A
:1085180090009300960099009C009F00AE00B20066
:10852800BA00B600BE00C100C500CE00CA00CC002B
:108538000501D20005010501050105010501050137
:1085480005010501050105010501050105010501F3
:108558000501DA00DE00E200E700EB00EF00F300BF
:10856800FC00664B93F818312371002004B010BD4D
:10857800624B93F83031F7E7406803F0C3FBF4E748
:10858800406803F005FCF0E75C4B93F81A31EBE721
:108598005A4BD3F8E0306360E7E7584B011D93F876
:1085A800300103F00DFCE0E7544B93F81931DBE799
:1085B800524B93F88C30D7E71C238DF808304F4B7B
:1085C80002A993F8480001F021FD6060CDE74C4B0B
:1085D800043493E8030084E80300C6E7494B0434F5
:1085E800F7E7494B0434F4E7484B0434F1E71A231E
:1085F800E3E71923E1E7414B93F86830B4E73F4BD1
:108608005B6DC8E73D4B9B6DC5E73C4BDB6DC2E737
:108618003A4B1B6EBFE7394B5B6EBCE702238DF804
:108628000830364B02A993F87C2093F848008DF85F
:108638000A2001F0EBFC207197E7304B93F8DD300E
:1086480092E72E4B93F839308EE72C4B93F8DC30B9
:108658008AE72A4B93F8383086E7284BDB6C9AE791
:10866800264B93F850307FE7244BD3F8843063606F
:108678007BE7224B8FE7264B8DE7204BD3F8CC3096
:10868800F5E71E4BD3F82C31436001F04DFDA06097
:108698006BE71A4BD3F890307DE7184B93F81F31EE
:1086A80062E7164BB3F88830A3805EE7134BB3F844
:1086B8008A30F9E7114BB3F8D030F5E70F4BB3F830
:1086C800D230F1E70D4B93F848200AB1062A12D1AF
:1086D800B3F8A035E8E7094B93F848200AB1062A11
:1086E80009D1D3F8A43556E704B0BDE8104000F02E
:1086F80021BE03203AE7182038E700BFA80C002065
:10870800140D00205C0D00201C0D0020640D0020BD
:10871800E40600207FB5044610B9032004B070BDFC
:10872800A34DD5F840339A0700F16F820278412AA9
:1087380000F26882DFE812F04200470055005B0053
:108748005F00640069007600810087008D00930057
:1087580099009F00A500AB00B5006602BA00DC00D6
:10876800EF0016013801290142014B014F01530165
:1087780057015B0166025F01710199018701AB0135
:10878800B101B801BD01C201660228026602660293
:108798006602660266026602660266026602660291
:1087A80066026602660266026602660234023902E0
:1087B8003E02430248024D0252025C020079FEF773
:1087C80073FA30B1AAE70379022BA6D0794A82F866
:1087D800303195F8913443F0200385F89134002026
:1087E8009CE7406803F080FA0028F2D095E74068DB
:1087F80003F0BEFAF8E76F4B027983F81A21E8E72D
:108808006C4B4268C3F8E020E3E76A4E416896F88B
:10881800300103F0CBFA00287FF47FAF6368C6F815
:10882800E430D6E7416800293FF477AF002001F033
:10883800DDF90028CDD0112070E7416800293FF408
:108848006CAF0120F3E7416800293FF466AF0820C8
:10885800EDE7416800293FF460AF0920E7E7416888
:1088680000293FF45AAF0C20E1E7416800293FF4A2
:1088780054AF0D20DBE7416800293FF44EAF0E20CE
:10888800D5E7416800293FF448AF0F20CFE74A4CAD
:10889800484B007983F81901A36D9847E36A984714
:1088A80097E7444B027983F88C2092E7414E037A8C
:1088B8008DF8043096F8480096F87D308DF805302C
:1088C800072201A901F0B5FB00283FF426AF636831
:1088D80096F848000193002201A901F0AAFB00289C
:1088E8003FF41BAF6C36D4E9010186E8030070E75A
:1088F800304E037A8DF8043096F8480096F87D30AB
:108908008DF80530072201A901F093FB00283FF4F8
:1089180004AFB436E7E7274E037A8DF8043096F8AB
:10892800480096F87D308DF80530072201A901F03E
:1089380080FB00283FF4F1AED4E9010106F174038D
:1089480083E8030096F81831022B7FF442AF96F8BB
:108958003031002B3FF43DAF174BDB6A9847FEF7E9
:1089680075F936E7134E037A8DF8043096F8480007
:1089780096F87D308DF80530072201A901F059FBE2
:1089880000283FF4CAAEBC36ADE743680293012322
:108998008DF80C30074B02A993F8480001F056FBFC
:1089A80000287FF416AFB8E6436802930023EFE788
:1089B8006C120020A80C002024F4000803795A1E29
:1089C8000E2A3FF6AAAE934A82F8683001E7914B27
:1089D80042685A65FDE68F4B42689A65F9E68D4B09
:1089E8004268DA65F5E68B4B42681A66F1E6894B10
:1089F80042685A66EDE6874C037994F848008DF88A
:108A08000430062201A901F014FB00283FF485AECA
:108A18009DF8043084F8DD30DBE67E4C03798DF870
:108A2800043094F8480094F87C308DF8063005221C
:108A380001A901F0FEFA00283FF46FAE9DF804305A
:108A480084F83930C5E6734C037994F848008DF8FA
:108A580004300A2201A901F0ECFA00283FF45DAEC7
:108A68009DF8043084F8DC30B3E66A4C037994F856
:108A780048008DF80430092201A901F0DAFA00282B
:108A88003FF44BAE9DF8043084F83830A1E6614BD2
:108A98004268C3F89420DA649BE65E4B027983F857
:108AA800982083F8502094E65A4B4268C3F88420F3
:108AB8008FE6584B4268C3F8CC208AE6012B40F079
:108AC800A480554C2421204603F050FA636A98424A
:108AD80001D0172022E61C2104F1280003F046FAF1
:108AE800636C9842F5D14FF4807104F1480003F0AB
:108AF8003DFAD4F848319842EBD1D42104F5A67058
:108B080003F034FAD4F820329842E2D1002104F577
:108B1800097003F02BFAD4F824329842D9D14FF4D3
:108B2800607104F50A7003F021FAD4F8A835984268
:108B3800CFD1142104F2AC5003F018FAD4F8C035A0
:108B48009842C6D1334E2146304640F2C45203F013
:108B5800F7F9204640F2C452002103F005FA95F8CF
:108B68001B3485F8E833736FC5F8EC3396F87D301D
:108B780085F8F83340F20123A5F8FA33274B96F825
:108B880019019B6D984724E68379012B3FF6C5AD03
:108B9800204B42684068C3F82C2100F0BDFE48E62F
:108BA8001C4B4268C3F8902013E61A4B027983F8ED
:108BB8001F210EE6174B8288A3F8882009E6154B7B
:108BC8008288A3F88A2004E6124B8288A3F8D02072
:108BD800FFE5104B8288A3F8D220FAE50D4B93F8F5
:108BE80048200AB1062A12D1A288A3F8A025F0E5E8
:108BF800084B93F848200AB1062A08D16268C3F8DE
:108C0800A425E6E500F098FBDBE5012086E51820C1
:108C180084E500BFA80C0020E406002024F4000826
:108C28002DE9F04387B00023ADF800300646002850
:108C380000F0EE800361FEF747FD20B101242046D5
:108C480007B0BDE8F08300F065FD0028F6D100F01C
:108C58005BFD014618B96F48142203F085F96E4D83
:108C680095F89134012243F0040385F8552485F8DA
:108C7800913433788DF804300021013B8DF80520BC
:108C8800ADF806100C2B00F2BB80DFE803F007B943
:108C9800B9B97982B9B990B9AD9AA900D5F8407334
:108CA80017F02007CAD196F80480B8F1020F46D110
:108CB800DFF868815A4CFEF763F896F9051098F8C2
:108CC80048003A4601F00FFA88F83900B37988F875
:108CD8003830384607238DF80530FDF7E5FFFF23C8
:108CE80004F58670A5F80C31C5F8084185F80471BB
:108CF80003F04EF804F58A7003F004F83846FDF7DF
:108D08002DFE0446002839D096F9051098F8480039
:108D1800012201F0E8F988F83900D5F89434336174
:108D2800002C71D000F0F0FC002888D195F891341F
:108D380085F81A0460F3820385F891347FE7B8F167
:108D4800010F4FF00204E8D1DFF8D0908DF81440FD
:108D580099F8480089F81D7102A901F065F933797D
:108D680089F830318DF805708DF80680FDF7C4FC60
:108D780095F8913443F0100385F891340024CCE73A
:108D880000226946022000F0F3FA0028F6D01324E6
:108D9800C3E7244BB288DB6B96F90C10B068984790
:108DA800D5F8403343F00203C5F84033E6E702A99B
:108DB8000D2000F053FB0028E0D0002269460D206A
:108DC800E1E7164B93F81831D3B9347904F007006A
:108DD80000F0ABFA8DF80040012269461020D2E776
:108DE800002269461220CEE78DF8072000F08EFA9F
:108DF800044638B900F087FA204600F089FABDE742
:108E080002248AE7012488E701A800F0D1FB16E7CD
:108E1800032414E7C01600206C120020A80C0020C0
:108E28006E12002024F400082DE9F04F99B0804616
:108E3800059118B9032019B0BDE8F08F002303612C
:108E4800FEF742FC0446002840F0A58046460FCEB7
:108E58000EAD0FC51422524898F800A0B8F80C704F
:108E680098F90EB04F4E214603F07EF84E4B012282
:108E780083F8412496F83021022A25460BD196F82A
:108E88001821022A07D196F81E2122B9BAF1010F3A
:108E980038BF4FF0010ABAF1010F2BD0BAF1030F16
:108EA8002AD0BAF1000F33D102229DF83C30DDF808
:108EB8004090029362F34715012496F87C108DF8D0
:108EC800321002220CA996F848008DF8302001F0E3
:108ED8009DF896F81A3196F830C196F81D1140B2EF
:108EE800002B63D0BCF1010F57D1002955D1002CBC
:108EF80061D153E00422D8E70023DDF83C90BDF8A7
:108F080040709DF942B0029365F01F050124D4E733
:108F18004FF0000BD946CDF808B0CEE74FF001006E
:108F280084F81A04D2E005F29A420BA900F0D4FAA8
:108F3800002800F015811320049B33871A4B002268
:108F480083F81A2423E105F29A452A460BA900F072
:108F5800C3FA0028EFD10B9B84F82801C4F82C51E0
:108F680084F83031FCE0B9F1000F00F0F980002AF4
:108F780000F0F6804946E01C02F0E2FF94F8373230
:108F880001332380ECE01220D6E70220D4E7072043
:108F9800D4E71320D2E701204DE7FCB90220F6E020
:108FA800AC160020A80C00206C120020002CF5D074
:108FB8005845B8BF584696F87C308DF820000522F1
:108FC80096F848008DF8223008A901F032F80028F8
:108FD8003FF430AF9DF8203086F839306F4A704B37
:108FE800D2F89804D3F8904038B105F087FA6C4B62
:108FF80084423CBF002283F83A20198F1A8F93F8D5
:1090080030010491996A099152BA0028BFD093F8A7
:109018001B0100B9186393F81801ADF858200138FE
:1090280093F87C2093F81A411491D0F1000BD3F8EF
:1090380088108DF85B204BEB000B93F8482093F8D1
:109048003A0093F868308DF85A3009AB0093554BC5
:1090580003904FF001008DF84C0015918DF85C20BD
:10906800A3F12F01A3F1300213A88DF84D4000F0B1
:10907800DBF8039B4FEA0B1B4BEA431B00264BEA2A
:10908800801B4BEAC413B145444C039308BF3746D1
:109098003A46494604F59C70CDE90A669B46268007
:1090A80084F81A6402F04CFFE9B2A570C5F34215C2
:1090B800FAB2042D3A4E039B84F837223FF42EAFC0
:1090C800072D3FF450AF022D7FF45FAF364D84F883
:1090D8000D110420029984F80401FF2084F80C0182
:1090E80084F8281184F81431D6F8E410C4F808512B
:1090F80005F59B730AA8C4F8101184F83021C4F848
:109108002C3100F011FC00287FF43DAF0A9BA4F835
:1091180044040BA8A4F81631C4F84C3400F0D0F974
:1091280000287FF408AF0B9BD3B196F93900FDF7FF
:10913800F7FA94F83732002B3FF405AF0B9B0F2B4F
:109148003FF6F1AE05F58B720BA90F2000F0C4F9BC
:1091580000287FF4F0AE0B9B63F3030B84F814B183
:109168000598FDF7FBFB00287FF4E6AE099B86F81F
:109178003A00B36200F080F900287FF40AAF94F84F
:10918800913484F840A443F0010384F89134034BEC
:10919800D3F89434C8F810304DE600BF6C120020A4
:1091A800A80C0020100D00206E12002037B50B4DC2
:1091B8008DF8040004460F2295F8480001A900F034
:1091C80038FF40B1064A85F81C4192F8913443F0C3
:1091D800200382F8913403B030BD00BFA80C0020F2
:1091E8006C12002010B5FFF7C1F8044688B90A4888
:1091F80005F0BEF9094805F0BBF9094805F0B8F9CA
:1092080000F094F8FDF7BCFD064BDB6A9847204652
:1092180010BD0124FBE700BFD4150020EC15002089
:109228000416002024F400082DE9F04F8BB047788D
:109238000093149B90F90C8090F90D6090F80EB093
:109248008A464168196004469146002F58D0022387
:109258008DF8103004A9C37B007C8DF8123000F023
:10926800D5FEB4F808C0618943B2606898454546A0
:109278006144B8BF1D46604534BF002701278842B6
:1092880009D30A218DF81010207C019304A900F05D
:10929800BDFE019B46B2B4F808C0608961680CEB5A
:1092A800400E714519D3A1EB0C01B1FBF0FC00FB9A
:1092B8001C1191B9984503DC2378CBB94FF0010B09
:1092C80021238DF81030207CE37B8DF8115004A900
:1092D8008DF8123000F09AFE45B2009B8AF80050D3
:1092E800384689F8006083F800B00BB0BDE8F08F0D
:1092F8000223207C8DF8243006A900F095FEDDE7D6
:109308004546EAE770477047704770470020704746
:109318007047704770470020704700207047002052
:1093280070470020704700207047704770477047AB
:1093380002207047022070470220704770470020C3
:10934800704770477047002070470020704770478B
:109358007047704710B5054C4FF403722046002142
:1093680002F002FE0020C4E9000010BD88170020AA
:109378002DE9F8438146904600293CD01F4C202314
:10938800224604F1100012F8017F6FBB8242FAD125
:109398001B4E3368013403B93460736803B11C6031
:1093A80000252560C4F8088074601FFA88F284F8E4
:1093B8000490601D02F0C4FDB9F1110F4FF00003D5
:1093C80098BF104D6373D6F8083298BF25FA09F58F
:1093D80003F1010398BF05F0010543442573C6F85E
:1093E80008323846BDE8F883013B13F0FF03044612
:1093F800C6D10227F5E70127F3E700BF8F17002042
:10940800881700202007020010B518B3124A136805
:10941800984204D103681360002305E00B46002B33
:10942800FAD019688842F9D15168884208BF536058
:109438000BB101681960D2F808328168013B002439
:109448005B1A04602146C2F80832102202F08CFD33
:10945800204610BD0120FCE788170020054B1B683B
:1094680013B11A798242FAD1002B0B600CBF03208A
:10947800002070478817002010B5054B186800B900
:1094880010BD037B04680BB9FFF7BEFF2046F6E763
:109498008817002038B5084B084C186800B938BD43
:1094A80003790568112B05D824FA03F3DB0701D5E6
:1094B800FFF7AAFF2846F1E78817002020070200D7
:1094C80028B1044BD3F8083203600020704701200C
:1094D800704700BF881700202DE9F04107460E4667
:1094E800154642B339B3154B1C6800232CB93046D6
:1094F800FFF7E6FF0020BDE8F081A268F91A013203
:10950800914215D32279EA54581C22895FFA80F8CF
:10951800611D55FA80F002F013FDA3682468984491
:109528005FFA88F3E2E720462568FFF76DFF2C46CF
:10953800002CF8D1DBE70120DDE700BF8817002009
:109548000238C0B211289ABF014B185C002070473E
:109558003BED000830B50B4B93F820200446084635
:1095680072B100211C330578A54208D00131984218
:10957800CDB214BF04301038AA42F4D8002030BD50
:109588001046FCE79419002010B5084C0023206011
:10959800142204F10C00FF2184F82030C4E90100F2
:1095A80002F0E2FC012384F8213010BD9419002058
:1095B80010B50E4A92F82010042915D8936804783B
:1095C8001C7044785C70C478807898700131DC70C5
:1095D80082F8201002F11C018B4214BF043302F1FF
:1095E8000C039360012010BD0020FCE794190020B3
:1095F800094B93F8200068B15A6803F11C018A42AC
:1096080000F1FF3014BF043203F10C0283F820008C
:109618005A600120704700BF9419002010B5074B0D
:1096280093F820200446084632B15968FFF792FFA4
:1096380010B101234470837010BD00BF941900203D
:1096480008B5064B93F820202AB15968FFF782FF26
:1096580008B1407808BD0120FCE700BF941900203C
:1096680030B50A4A92F82010536882F8210061B197
:10967800916801241C32DD78587005B99C709342BA
:1096880014BF0433103B9942F5D130BD9419002022
:1096980008B5044B5968FFF75DFF003818BF012073
:1096A80008BD00BF94190020F7B50422154E0446E2
:1096B80000210DEB020096F8207002F055FC002501
:1096C800EBB29F4201D803B0F0BD736819782170DE
:1096D8005A786270987838B1336820469B68984702
:1096E800FFF786FF0135EBE7DB788DF804108DF87E
:1096F80005208DF80730FFF77BFF01A8FFF758FF1B
:10970800F0E700BF94190020014B93F82000704740
:1097180094190020034B93F82000042894BF0020DC
:1097280001207047941900201FB50024CDE9024498
:10973800C41F8DF800408DF801100C0AADF8042004
:10974800090C120C8DF803108DF806208DF80730DF
:1097580002461B0A012168468DF802408DF8083040
:1097680002F05DFA002818BF0E2004B010BD2DE9E4
:10977800F04188B090460D460F9A0746002847D01A
:1097880000240121CDE904448DF810109DF838100B
:109798008DF81510ADF81630190CCDE900441B0EE4
:1097A800CDE902448DF81930ADF81A20130C120EC9
:1097B80007948DF818108DF81C308DF81D20E3B231
:1097C8001E01002DF6B203DC002008B0BDE8F081D0
:1097D800013310218DF81F3042466B460DEB010016
:1097E80002F0B3F90346A8B9102D28463E44A8BF95
:1097F80010206946327811F801CB013382EA0C0255
:10980800984206F8012BF5DC103D2DB20134D6E75D
:109818000920DAE70E20D8E70138032815D8DFE851
:1098280000F002080C100A4B1B681B690B60002033
:109838007047074B1B685B69F8E7054B1B689B691A
:10984800F4E7034B1B68DB69F0E70520704700BFAE
:10985800B81900202DE9F041C4B00C464A9E1746BD
:109868001D468046B8B3B1F5807F36D84FF488726C
:109878000021684602F078FB492300934FF4807377
:10988800ADF804302B0C8DF80830330CADF80650C9
:10989800ADF80A608DF80C3022460023414604A832
:1098A8002D0E360E8DF80E308DF809508DF80D609E
:1098B8008DF80F4002F044FB04F110014B9A3B462F
:1098C80089B2684602F02BF910B1012818BF0E20A2
:1098D80044B0BDE8F0810920FAE70D20F8E7000060
:1098E80010B590B10A4C28220021206002F03CFB00
:1098F8002368084A1A6000204FF0FF32C3E90302C8
:10990800C3E90522C3E9072210BD0820FCE700BF10
:10991800B819002000010101024B1B6818600020E3
:10992800704700BFB819002030B1044B1B68DB68D2
:10993800013303600020704709207047B8190020E0
:1099480013B500230C460193CAB101A9FFF764FFC0
:1099580018B9019B591C02D1146002B010BD99B20C
:10996800611A002901DD5C18F6E702D113600720AF
:10997800F3E71B0C1B0403F580331C44ECE70920B8
:10998800EBE7000028B1044B1B681C33436200203E
:1099980070470920704700BFB81900201FB504465A
:1099A80000B3002303A8039302F090F9104ABDF80E
:1099B8000C30126820469380E38200F05EFA98B972
:1099C80004F11803009321680123132202F09CF884
:1099D80060B9204600F051FA003818BF0120000194
:1099E80004B010BD0920FBE71020F9E70E20F7E7C7
:1099F800B8190020F0B5054687B01C4613B90920F0
:109A080007B0F0BD2E4E3368DB68834255D894F812
:109A18002020002A0CBF08220922834205D32046B1
:109A280000F05FFA68B11020EAE700230190009384
:109A3800A36894F82810606AFFF799FE0028EED012
:109A4800DEE723792168B4F808C0A768043B9AB216
:109A58000029D4D0B2F5807F2DD8ADF80EC08DF88E
:109A680017304FEA174C04F12C033F0E8DF8117094
:109A780000932F0C08234FF0490EADF80C008DF819
:109A880014708DF816002F0E0DEB0300CDF808E0CA
:109A98008DF810C0ADF812508DF8157002F034F83A
:109AA80008B10E20ACE7204600F01BFA0028BAD116
:109AB8003368DD60A4E70D20A2E70620A0E700BF19
:109AC800B81900202DE9FF410A9D80460F46164629
:109AD8001C46002D5AD0002303A910460393FFF714
:109AE8009BFE18B1062004B0BDE8F081039B9C42A0
:109AF80001D80133F6D1284600F064F9002847D18F
:109B0800264B1A78424503D01A79424542D10120A2
:109B1800AA68BA4240D103EB8002EB6A92F801804E
:109B28002979CDE900430439927828683B4689B2FF
:109B3800FFF790FE0028D6D195F820300194002B2D
:109B48004FF00103009314BF4246082295F82810ED
:109B5800686A3B46FFF70BFE0028C4D1013E032E7E
:109B6800C1D8DFE806F002070B0F0D4B1B681C611C
:109B78001C62B8E70A4B1B685C61F9E7084B1B6875
:109B88009C61F5E7064B1B68DC61ACE70920AAE796
:109B98000F20A8E70B20A6E70220A4E7F00000208A
:109BA800B81900201FB50B294FF00003CDE9003389
:109BB800CDE902330A4607D00C2914D00A2910D05F
:109BC8000A2005B05DF804FB012802D120238DF896
:109BD80000300021684602F022F8002818BF0E2045
:109BE800EFE73023F3E70B21F4E7000038B505462B
:109BF80002F010F8044610B10E24204638BD002D9E
:109C0800FBD1094B1B680B219878FFF7CBFF002885
:109C1800F2D10C21FFF7C6FF0028EDD10A21FFF78A
:109C2800C1FF0028E9D0E7E7B81900202DE9F04383
:109C380080468FB00C461746002A6BD0002969D0A1
:109C4800002529461D2206A8059504F097FE8DF8E3
:109C58001350344D2B680DF114099E88CDF80490EB
:109C68000DF1130302933B7900933B68324621467A
:109C7800404601F0F0FF00284ED138683A7949464D
:109C880002F05EF9384600F04FF8002846D13C7AD9
:109C9800FA79BB79240444EA02241C432B689A68A5
:109CA80094423DD99C609DF813000B21FFF77AFF81
:109CB800034658BB0C21FFF775FF034630BB0A214A
:109CC800FFF770FF034608BB7B7ABA7AFF7A3F0436
:109CD80047EA02271F433A46334621460920FFF741
:109CE80023FD034690B933463A4621460820FFF73C
:109CF8001BFD034650B92A689DF813109170002186
:109D0800D1604FF0FF31C2E90411916118460FB0DC
:109D1800BDE8F0830923F9E70E23F7E70F23F5E7FA
:109D28000323F3E7B819002010B50446002845D0EE
:109D38000168002942D011F8013B43710322063023
:109D480002F0FEF82046032250F8091B043102F005
:109D5800F7F82168CB79E3600A7A43EA0223E360E3
:109D68004A7A43EA0243E3608A7A43EA0263E36099
:109D7800CB7A23740B7B63742379212B1AD110229D
:109D88000D3104F1120002F0DBF81D222168501C8D
:109D98008B5C6362085C43EA0023901C6362085C86
:109DA800033243EA004363628A5C43EA0263636204
:109DB800002010BD112B03DC0D22E7E70220F8E795
:109DC8000120F6E710B50446002854D001680029A0
:109DD80051D00B7843714B7883608A7843EA022329
:109DE8008360CA7843EA024383600A7943EA0263DC
:109DF80083604B7903738B79C381CA7943EA022361
:109E0800027BC38102F00F020831103002F098F88B
:109E1800237B002203F00F0384F8202084F82820F5
:109E2800227903F10800111A04290DDD216809338C
:109E3800043AD21A085C84F82000D2B2606A84F826
:109E48002820194402F07CF8237922681A4400205B
:109E580012F8043CE36212F8031C43EA0123E362AC
:109E680012F8021C43EA0143E36212F8012C43EAA8
:109E78000263E36210BD0220FCE710B5044660B33C
:109E8800036853B30279162A29D942791A70014610
:109E9800082251F8060B013002F05CF8214608222E
:109EA80051F80E0B093002F055F82368E28A5A740B
:109EB800E38A22681B0A93742368A269DA74A36987
:109EC80022681B0A13752368628B5A752368E27E21
:109ED8009A7517232371002010BD0120FCE702208A
:109EE800FAE738B50446002863D00168002960D035
:109EF800037B90F8282003F00F03002A57D108337A
:109F0800207904321344984255D363790B7023683F
:109F1800A2685A70A36822681B0A93702368628932
:109F2800DA702368E27A1A712368227B5A712368EF
:109F3800E2899A71E38922681B0A2146D371227B40
:109F480051F8100B02F00F02083001F0F9FF237BE3
:109F580094F8282003F00F0303F108052AB12268BA
:109F680094F82010515503F10905206894F8282029
:109F7800616A284401F0E4FF94F828302268E16A15
:109F88002B44D1545A1CE16A206892B2090A8154C0
:109F98009A1C2168E08D92B28854DA1C216894F8E2
:109FA8002F0092B2043388542371002038BD09333E
:109FB800A6E70120FAE70220F8E70000024B1A881A
:109FC80010431880704700BFBC19002008B5074B24
:109FD8001B883BB1FEF7CAF9002814BF6FF00200D6
:109FE800002008BD6FF00100FBE700BFBC1900208E
:109FF80010B5034B00241C80FEF7AEF9204610BDB7
:10A00800BC190020B0FA80F04009704782B018B936
:10A01800084602B000F0CAB8002002B0704710B974
:10A02800084600F077B9704710B9084600F08EB9B5
:10A0380070470346084611460BB900F0E5B9002001
:10A04800704710B9084600F06DBD704710B9084652
:10A0580000F006BA0020704710B4044608461146BE
:10A068001A46019B14B910BC00F014BA10BC704712
:10A078000346084611460BB900F03EBA0020704767
:10A0880010B40446084611461A4614B910BC00F02C
:10A09800ABBA002010BC704730B4054608461146DC
:10A0A8001A46DDE902341DB9029430BC00F02ABB1F
:10A0B800002030BC704710B9084600F0DBBB002018
:10A0C800704710B9084600F06BBD0020704710B902
:10A0D800084600F0EABB0020704710B9084600F0B7
:10A0E800E7BB002070470346084611460BB900F04D
:10A0F80001BC0020704710B40446084611461A46B1
:10A10800019B14B910BC00F0F7BB092010BC7047C4
:10A1180010B40446084611461A4614B910BC00F09B
:10A1280061BDC8B210BC7047004870470100010209
:10A13800064B10B51B6A0446984730B10448054BD6
:10A14800204498428CBF0020012010BD24F4000850
:10A1580040C220C980B92A00F0B5114B85B00C4621
:10A1680010491F56054601F04BF80F4BE4B25E6AE2
:10A17800072D4FF00103CDE9024301460AD105221C
:10A188000023CDE900234FF47A727A431846B0478A
:10A1980005B0F0BD08220020CDE900203A46F5E7D9
:10A1A80008EE0008E8ED000824F400081FB50023B5
:10A1B80000930378013B372B21D8DFE803F01C24F8
:10A1C8002020201E202020204143454E2055585B4A
:10A1D8005E6164206C1E6E73787A20207D81262053
:10A1E80020202020202020202020202083858A2035
:10A1F80020838A208C90C3780BB1022300930098A7
:10A2080005B05DF804FB8378F6E743788DF80430F1
:10A2180005238DF805308378003B18BF01235B00C8
:10A228008DF8063010238DF80730304B1B6801A8D5
:10A2380003F55872CDE9022300F0C2FF0090DEE773
:10A248004023DBE72023D9E7827890F9013012B95F
:10A25800274AD35CD2E7274AFBE7827890F9013096
:10A26800002AF8D1244AF4E740F6B833C6E74FF499
:10A278007A73C3E74FF4FA63C0E741F28833BDE766
:10A2880041F27073BAE71D484FF47A7101F03CFE51
:10A2980000F5FA60D2E71A4BB0E7144B1B6803F5D8
:10A2A8005873ABE7114B1B6803F55B73A6E71023E4
:10A2B800A4E70E4B1B68A1E74FF0834300939EE78A
:10A2C800104BFBE7104B99E740F21113ADF8003043
:10A2D80095E7032392E790F901300C4AB9E70C4956
:10A2E80090F9010000F08CFFA8E700BFC419002016
:10A2F800DDED0008CDED0008D5ED000818FCFFFFE6
:10A3080000EA06379A99094040F7093708EE00082D
:10A31800E8ED000837B50B4B02781B680C2101FBF0
:10A3280002335B7A03EB4304074B1D680369009310
:10A33800C3684278816805EBC40000F0DDFC03B017
:10A3480030BD00BFC4190020C019002070B586B008
:10A35800027B6423ADF80030012A4FF00003CDE9F9
:10A368000133CDE903338DF802308DF8143030D045
:10A37800022A39D05ABB03684BB343683BB31F4D1D
:10A3880080682B601E4B18226946186001F0D8FDC2
:10A398001C4B2C6893E807000C3384E8070093E80B
:10A3A800070004F10C06032386E80700A4F86C33C1
:10A3B800012204F55B7104F5587000F08EFC2B68DF
:10A3C8004FF6B072A3F878230522C3F87C2306B0B1
:10A3D80070BD0A4908684360036100F55B7100F5C8
:10A3E800587000F07AFCF2E7044B1B68B3F860235E
:10A3F800B3F86C130A43A3F86023E8E7C4190020F4
:10A40800C019002030EB000808B503460A2924D8F3
:10A41800DFE801F006232323230B161B2321210049
:10A42800BDE808400068FFF783BE90F900009978FE
:10A43800052271B900F011FC003818BF012008BDD1
:10A44800052293F900000021F4E790F900005978FB
:10A45800EEE70221EEE70722F3E70020EFE700002E
:10A4680008B502791AB1012A0BD0002008BD084BA3
:10A4780001681B68012203F5587000F02EFC0120CA
:10A48800F4E7034B01681B6803F55B70F5E700BF51
:10A49800C4190020F7B50528144D1C46A8BF05208F
:10A4A80058700E462946174600F0AAFE94F9013066
:10A4B800A070072B13D1322000F0A2FD0C4BDB6DEE
:10A4C8000546984704F10C020834034601920094AB
:10A4D8003A463146284600F098FD03B0F0BD054ADB
:10A4E80055F82310D05C00F083FDE7E7E8ED00089D
:10A4F80024F4000808EE00082DE9F04F344F90F9D5
:10A5080001607B68D0F804908BB004468846984771
:10A518000546002859D1E37C73B92E4A237812687E
:10A5280003EB4303990002EB8303D3F80490B9F1DA
:10A53800000F01D152F80190274B484613F906B095
:10A54800FB689847A37C2289D7F818A00993072E9F
:10A5580028D100230121CDE90223204A0693CDE921
:10A568000431CDE907330521CDE900214FF47A7292
:10A5780002FB0BF24CF250311846D047637C13B300
:10A58800174B995D7B6D0D31C9B228469847E07C21
:10A598003246494600F046FE88F8006001200BB0BC
:10A5A800BDE8F08F002101250823CDE90013CDE98E
:10A5B8000715CDE90511CDE903110292A1782B46C3
:10A5C8005A462846D9E7074BDBE70020E7E700BFF4
:10A5D80024F40008C419002008EE0008854501008D
:10A5E800D5ED0008DDED00082DE9F04F8DB090F9AC
:10A5F8000130DFF8FCA0DFF8FC90CDE90A123E4AF2
:10A6080012F903B00278DAF800300C2505FB0233A2
:10A618003A4A5B7A126803EB430302EBC30304462E
:10A6280093F9021090F9020000F0E5FD344906465E
:10A6380094F9010000F0E4FDA268616880463046A4
:10A6480000F00BFD2178DAF80020D9F80C306943C6
:10A65800074650589847D9F81C309C4694F9013061
:10A668000025072B4FF47A63CDE90753CDE905554B
:10A678002DD10123CDE903530523CDE901534FF42F
:10A688007A7303FB0BF300933946434646F2A8124C
:10A6980028466746B8472378DAF800200C214B4350
:10A6A80094F90110D05800F0DFFDA18994F9010058
:10A6B800FFF752FD0B9B217B1860D9F854302846D0
:10A6C80098470A9B01201E700DB0BDE8F08F01204D
:10A6D8000823CDE90350CDE901032A46CDF800B09F
:10A6E800654643463946A84701200546D3E700BFDB
:10A6F800C419002024F4000808EE0008C01900203E
:10A70800E8ED00082DE9F04F8FB0002405468A4691
:10A71800914698460494ADF81440ADF802400726D7
:10A728004FF0010B2B7AA34206D9686804A920448C
:10A7380000F0F6FB00285ED102238DF8083002A84D
:10A748006B7A8DF80A30FFF731FDAB7A8DF81D3042
:10A758009DF811308DF81E309DF812308DF81F309D
:10A768009DF810308DF82030EB7A8DF821302B7B56
:10A778008DF822306B7B8DF8233010238DF81C6008
:10A788008DF824303A4E8DF82C000DF102030A930F
:10A7980005238DF82D3033680C930723ADF834303A
:10A7A8002B6806930DF1120204AB0DF1110106A8F6
:10A7B80000F0D0FB072805460BD130680C22002199
:10A7C80000F5587001F0D0FB3368BDF80220A3F8FB
:10A7D80060239DF811308AF800309DF8123089F80E
:10A7E80000309DF8103088F80030189B28461C70FF
:10A7F8000FB0BDE8F08F9DF81330BDF81470ADF8B8
:10A8080002702044C4B2F3B917B3194A0020116882
:10A81800072602464FF00C0C062B1BD10CFB00FE42
:10A8280051F80EE0BEF1000F04D00BFA00F23A43E3
:10A8380097B2012201301028EED1002A3FF472AFFE
:10A84800ADF802706EE75A1E042A01D9062BDCD037
:10A85800062667E747FA00FE1EF0010FEAD00CFB58
:10A8680000FE51F80EE0BEF1000F08BF0626E1E732
:10A87800C419002038B505464068FFF759FC052281
:10A88800841D002195F90000E4B200F0E6F908B94A
:10A8980004F0FD0495F901000722002100F0DDF91C
:10A8A80008B904F0FB04204638BD002070470000BA
:10A8B80010B503780F2B044618D84068FFF738FC0A
:10A8C80022780B4902EB42020968831C01EB8200E3
:10A8D80051F82220DBB21AB903F0FD0358B210BDBB
:10A8E800032B06BF626842600223F7E70020F6E701
:10A8F800C4190020022070472DE9F04FDFF8388195
:10A908000446D8F8000099B08946174600211E462B
:10A918000122032300F55870CDE90611CDE908118D
:10A928008DF814108DF81510ADF8163000F0B7F941
:10A9380038B9D8F80020B2F8603343F00303A2F81E
:10A948006033D8F80020637A8DF8283002F5587102
:10A95800CDE90B12394A94F9083012680D920DF1BD
:10A9680016020F922268109262681192D4E90301CC
:10A97800A27A8DF8482001228DF8492013AA82E88E
:10A9880003001025227DE18A8DF8293018468DF8BC
:10A998005420ADF83850FFF7DFFB0AAB17930DF1E1
:10A9A8001503169000933146019705AB06AA10A827
:10A9B80000F0C2FB064698BB9DF81410204F0139E1
:10A9C80001F0A2FA1F4B1B690393C4B24FF00C0BA2
:10A9D80004F160036B44D8F8000013F848AC9DF804
:10A9E80014300BFB0AFC01343946B4FBF3F203FBC9
:10A9F8001244D0F87C33B0F9782350F80C00DDF815
:10AA08000CC0E4B2E04728B189F800A0304619B07C
:10AA1800BDE8F08F013D15F0FF05D9D10D26F5E70A
:10AA28000C2801BFD8F80020B2F8603343F00303C4
:10AA3800A2F86033EAE700BFC4190020C01900205B
:10AA4800400D030024F40008F8B50679012E0546E8
:10AA580048D90F2E48D80368187A40F30300052216
:10AA6800002140B200F0F9F82B680446187A40F348
:10AA780003100522002140B200F0EFF8B8B1B4FA93
:10AA880084F4640929680B7A086843F3030243F3E2
:10AA980003135BB252B29A42C8BF0124FFF748FBC6
:10AAA80080F00103DBB224B10533D8B2F8BD01242C
:10AAB800E8E7DBB90E4F29683B6806EB460003EB75
:10AAC80080000C2201F03CFA3A680C2303FB0623B1
:10AAD80020465C72B2F860130123B3400B43A2F81E
:10AAE8006033E3E70620E1E70320DFE70420DDE742
:10AAF800C419002010B4017801290ED9084B186830
:10AB08000C234B43C4180022C250C4E9012200F5AB
:10AB1800587010BC102200F0A9B8002010BC704773
:10AB2800C41900202DE9F04186B050238DF8143067
:10AB3800037A102B074630D14368DD7B6DBB0224B6
:10AB4800A8466426062C14D87A68535D03932A44D1
:10AB5800517843EA01230393927843EA024373430B
:10AB6800CDE9033863B968468DF80040FFF7C2FFA6
:10AB78000DE0CDF80C808DF81480CDF81080F2E748
:10AB880003AB01A801938DF80840FFF75DFF01347E
:10AB9800E4B2102C05F10305D4D106B0BDE8F0816C
:10ABA8001FB502680379116849B901A88DF8043006
:10ABB800FFF7A0FF78B1032005B05DF804FB02A8F9
:10ABC80002928DF80C30FFF73FFF042805D00528C6
:10ABD80005D00028EFD00020EEE70220ECE70120A6
:10ABE800EAE70000C90020B9034B0B449856C0B2ED
:10ABF8007047024BF9E700BF8DED00084DED0008E6
:10AC0800F0B59A42069D03DB9DF914309A4220DD87
:10AC18000020F0BD03EB430331F814C005EB8303B8
:10AC280000264CFA06F7FF0707D51F7A07F00F0E24
:10AC3800964502DCB2EB171F0DDD0136102E03F12D
:10AC48000C03EED10134E4B22301DBB29842E1D81F
:10AC5800DEE70024F8E70120DBE7884204DB9042C6
:10AC6800CCBF0020012070470020704710B51409A0
:10AC7800B4EB111F03464FEA11100ED391420CD2C8
:10AC880002B201F00F0133F81240012000FA01F17D
:10AC980024EA010123F8121010BD0020FCE7F0B5EA
:10ACA80028B100EB410501270020914200D3F0BDF7
:10ACB800002435F802CB234607FA04F636EA0C06D8
:10ACC80008BF013304F1010408BFDBB2102CF3D133
:10ACD80018440131C0B2C9B2E7E710B500B149B9AB
:10ACE80010BD31F8134020F813400133DCB2A24202
:10ACF800F7D8F5E70023F9E782B030B50488049364
:10AD0800D2B9B3F5616F15D349F6AF2542F2107287
:10AD1800AB4298BF4FF47A72944238BF14466143ED
:10AD2800BDE83040C3688B428CBF5B1A0023C36008
:10AD380002B070476422EFE7012C38BF0124EEE728
:10AD48002DE9F04F8FB01546199F03939DF8603099
:10AD580007930C46804603F0C7FB6A4A0590A7F59F
:10AD6800F633303BB3FBF2F3534303F5F63B04935E
:10AD7800182313FB05430BF1300B069300254FF006
:10AD8800FF3A069B9C4207D1002D14BF50464FF056
:10AD9800FF300FB0BDE8F08FBDF96830ADF8243052
:10ADA800099919973846089703F02EFB2688B8F1B9
:10ADB800000F5FD1B7F5616F5AD349F6AF2242F25F
:10ADC8001073974298BF4FF47A739E4238BF1E465D
:10ADD800642E59D1DFF83091A060A1680CA803F067
:10ADE80035FB0D9B0093DDE908120C9B0AA803F0C4
:10ADF8008CFA039A0A9B0AB9079A2AB122694A452A
:10AE080002D1424A93420ED9414BC4F80C909F425A
:10AE180009D90023ADF82C300B99CDF828B0584645
:10AE280003F0F2FAA060606808B9C4F80C90C4F89E
:10AE38001090B8F1000F04D003F060FBE3680344FE
:10AE4800E360D4E903329342059B88BFE260636004
:10AE58001B9BE1687343994204D20398E8B9B8F19F
:10AE6800000F1AD001231D442375EDB2183488E76A
:10AE78006423AAE7039B0BB9234BE360012EDFF899
:10AE8800889038BF0126CEE7B6F57A7F0ABFDFF88B
:10AE98008490DFF88490A0609FE70020934220759B
:10AEA80006D85B1A9A4505F1010528BF9A46EDB206
:10AEB800B8F1000FDAD1642E184AADF82C801DD0F5
:10AEC80049F6B023B6F57A7F18BF1346974281BF7B
:10AED800049A02F5A83202F5C0729B180A931A9BCD
:10AEE80000930AAE96E80600199B304603F00DFA67
:10AEF80096E8030003F088FA8246B7E74FF46163E7
:10AF0800E4E700BF8051010040771B007F5101003A
:10AF18002FEC010080A81201002E930230EC0100F2
:10AF28000378032B14D1437803F00F021B098A70AE
:10AF38004B7083788B80C27843EA02238B80037935
:10AF4800C3F3021203F00F03CA700B700520704799
:10AF5800002070472DE9F3479A464379057990F91F
:10AF680007609146044690F906208846D3B190F9C7
:10AF78000870002D37D00F2A1BD194F909200F2E05
:10AF880027D194F90A00072D02D1002F08BF012705
:10AF980088F8002089F8000028468AF8007002B076
:10AFA800BDE8F08790F90B7090F9092090F90A60D4
:10AFB800DFE7A369019394F91530009394F91430ED
:10AFC8002169207BFFF71CFE0028D8D105F0FD057C
:10AFD800D5E794F91D00B042D5DC94F91C30B34292
:10AFE80003DA05F0FB053046D2E73046CBE7000030
:10AFF800024B03FA00F0B0FBF1F0704740420F003B
:10B008004FF4FA53B3FBF0F0704730B54FF47A754C
:10B018000C1F6A4300FB042252001EBF00F1FF34DC
:10B028001219B2FBF0F2914238BF1146039A11602F
:10B03800820048431CBF013040084FF47A71121A4D
:10B0480001FB1323002BCABF03F2E73393FBF1F193
:10B05800B3FBF1F1049B196030BD38B540001446CC
:10B068000D46F5F7AFFB01462846F5F7F9FA2146F4
:10B07800F5F7F6FAF5F7E8F903F0AEFCF5F7C4FAD8
:10B0880040B238BD2DE9F74F019300239C469E46F8
:10B09800048A1E01F6B2B44246D906EB46054FEAC9
:10B0A8004309AD000024476837F809702741FF07B6
:10B0B80029D5876807EB050A7F5927B3077837B979
:10B0C800476927B137F809702741FF071BD59AF858
:10B0D800087090F901B047F303084FFA88F8D8458B
:10B0E80011DC47F303177FB25F450CDB9AF8097050
:10B0F80007EB4708C76807EBC8073F7D5FB90CF146
:10B10800010C5FFA8CFC0134102C05F10C05CAD136
:10B118000133DBB2BCE70EF1010706EB040801F8C6
:10B128000E805FFA87FEEEE7019B82F800E083F865
:10B1380000C003B0BDE8F08F2DE9FF470446406822
:10B14800DDE90C671D468A46914603F0D7F9236866
:10B158001B1A3B604FF000080123337085F800800C
:10B16800636813B12368834224D8D4F81CC0CAF892
:10B178000080A3699CF800E00393D4E9030101ABC4
:10B1880083E80300237D0093DCF80C10237A627AAD
:10B198007046FFF7D5FD334638602A46E0694946D0
:10B1A800FFF770FF2B782BB1C7F80080002004B0A0
:10B1B800BDE8F0873378002B0CBF0C200B20F6E796
:10B1C80037B590F9002090F90250954204460FD007
:10B1D800013A52B295420BD0A368019394F9013019
:10B1E80000936168E0782B46FFF70AFD0028EFD04E
:10B1F800104603B030BD8842B8BF0846704700000B
:10B2080051F82000054B984205D0054BC31A584207
:10B218005841400070470120704700BF90D003009C
:10B2280020A1070005281FB50ED80C4B53F8203075
:10B238000093CDE901120A4B01220021022002F0FD
:10B248006BFE05B05DF804FBCDE90012054B012249
:10B258000021022002F060FEF3E700BF7CEE000848
:10B2680010EE00082FEE000807B5054BCDE90001E8
:10B2780001220021022002F04FFE03B05DF804FB1A
:10B288004BEE000810B5102204460021F13000F002
:10B298006BFE0021C4F814112046F022BDE81040CE
:10B2A80000F062BE02460846102100F0A5B92DE95B
:10B2B800F0430446D0F8140185B00E46154604F252
:10B2C800011988B3C0F110089045474628BF1746B2
:10B2D800BAB2484400F034FED4F814313B440F2B82
:10B2E800C4F814312DD9A8452BD204F1F00304F584
:10B2F800807113F8012F187C8B4282EA00021A70C1
:10B30800F7D104F1F10810224146684600F018FE12
:10B3180022466946684600F0F1F91022694640461F
:10B3280000F00EFE3E44ED1B04F5807804F1F107B1
:10B33800102D09D8AAB23146484600F001FEC4F8DB
:10B34800145105B0BDE8F08304F1F003711E13F841
:10B35800012F11F8010F434582EA00021A70F6D155
:10B3680010223946684600F0EBFD224669466846D9
:10B3780000F0C4F910226946384600F0E1FD1036A5
:10B38800103DD5E7F0B589B00C46102200210546DE
:10B39800684600F0E9FD22466946684600F0AEF9C5
:10B3A8009DF90030002B6A464FF0000143DA13780C
:10B3B80012F8010F01315B0043EAD0130F2902F89C
:10B3C800013CF4D19DF80F305B0083F08703D4F87B
:10B3D8001401DBB210288DF80F303BD104F58073CF
:10B3E800694604F5887013F8016F11F8012B98422B
:10B3F80082EA06021A70F6D104F1F00304F58071AE
:10B4080013F8012F187C8B4282EA00021A70F7D1D8
:10B4180010220DEB020004F1F10100F091FD22462B
:10B42800294604A800F06AF910220021684600F0B5
:10B438009BFD09B0F0BD137812F8010F01315B00D4
:10B4480043EAD0130F2902F8013CF4D19DF80F30DC
:10B458005B00BCE79DF90030002B6A464FF0000105
:10B4680037DA137812F8016F01315B0043EAD6131B
:10B478000F2902F8013CF4D19DF80F305B0083F0EE
:10B488008703471CDBB28DF80F30102F04EB000345
:10B49800C0F10F064FF0800288BF002600F58170CA
:10B4A80083F801210021324620443E4403F066FA25
:10B4B800C4F8146104F58073694604F5887013F8BC
:10B4C800016F11F8012B984282EA06021A70F6D130
:10B4D80092E7137812F8016F01315B0043EAD61343
:10B4E8000F2902F8013CF4D19DF80F305B00C8E742
:10B4F8000A780378534003704A784378534043707E
:10B508008A78837853408370CA78C3785340C3706D
:10B518000A790379534003714A7943795340437157
:10B528008A79837953408371CA79C3795340C37147
:10B538000A7A037A534003724A7A437A5340437231
:10B548008A7A837A53408372CA7AC37A5340C37221
:10B558000A7B037B534003734A7B437B534043730B
:10B568008A7B837B53408373CA7BC37B5340C373FB
:10B57800704710B50B7814786340037054784B7893
:10B588006340437094788B7863408370D478CB7829
:10B598006340C37014790B796340037154794B7914
:10B5A8006340437194798B7963408371D479CB7903
:10B5B8006340C371147A0B7A63400372547A4B7AEE
:10B5C800634043728B7A947A63408372D47ACB7ADD
:10B5D8006340C372147B0B7B63400373547B4B7BC8
:10B5E80063404373947B8B7B63408373CB7BD27BB9
:10B5F8005340C37310BD0000A1F11003DBB2102B40
:10B608002DE9F047044604D83A4820FA03F3DB074B
:10B6180005D4002382F8F030FF20BDE8F087561EDD
:10B62800254615F8013B06F8013F631B0B4413F050
:10B63800FF00F6D101F11C039B005FFA83FCC3F302
:10B648000313013BDFF8B09082F8F03088465318B6
:10B658004FF0010EB8FBF1FA01FB1A8A1AF0FF0A43
:10B6680013F8047C13F8036C13F8025C13F8014C0C
:10B6780030D119F806A019F8056019F8045019F81E
:10B6880007404FEADE1707EB47078EEA0A0A07EB7F
:10B69800C7074FEA4E0EFFB25FFA8EFE87EA0E0E1C
:10B6A800574692F800A087EA0A071F7057787E402D
:10B6B8005E70967875409D70D57808F104085FFA39
:10B6C80088F86C40C445DC7002F1040203F10403FD
:10B6D800C0D8A2E71829E4D9BAF1100FE1D1DFF8F0
:10B6E80018A01AF807701AF806601AF805501AF820
:10B6F8000440D6E70101010094F000082DE9F04F5D
:10B70800A3B092F8F0301D911B920193002B00F02A
:10B71800538101461EA8FFF72CFF1B9BA74CA84D81
:10B72800A84E10330293002303939DF87C000490E5
:10B738009DF886000590205C06909DF87B00079098
:10B74800205C089004989DF881C0205C099014F84A
:10B758000C000A909DF880000B909DF885009DF8DC
:10B7680078809DF87DE09DF882A09DF887900C90E8
:10B778009DF87A00029B1C9314F80A2014F80930EB
:10B7880014F8081014F80E700D90205C0E909DF8B7
:10B798007F000F90205C10900B98205C11900C9803
:10B7A800205C12909DF8840013909DF87900149005
:10B7B8009DF87E001590205C16909DF883001790E8
:10B7C800205C18901398205C19901498205C1A90AB
:10B7D8000398013003900298DDF804B0103002900D
:10B7E8009DF80C00834536D88DF878108DF87A20AE
:10B7F80009990E9A8DF87C108DF882201199069A75
:10B808008DF880108DF87E201999169A8DF884107D
:10B818008DF886200A99189A8DF87D108DF8872062
:10B828001299109A8DF87B301B9B8DF881108DF83A
:10B8380083201A99089A1D988DF885108DF87F2015
:10B848001EA903EB0B128DF87970FFF792FE00200A
:10B8580023B0BDE8F08F15F808B082EA03008BEA40
:10B86800000016F80EB080EA0B008DF8780015F885
:10B878000E004B40434016F80A0043408DF87930DB
:10B8880081EA070315F80A10594016F8093059409B
:10B8980016F808308DF87A107A40534015F80920C8
:10B8A80053408DF87B30089A069B5340049AAA5C53
:10B8B800534016F80C2053408DF87C30DDE90832EF
:10B8C8005A4015F80C305340059AB25C53408DF835
:10B8D8007D30DDE909325A40059BEB5C5340079AFD
:10B8E800B25C53408DF87E30069B0A9A5340049A06
:10B8F800B25C5A40079BEB5C5A408DF87F200E9B48
:10B90800109A53400B9AAA5C53400C9AB25C53406D
:10B918008DF88030DDE910325A400C9BEB5C5340C7
:10B928000D9AB25C53408DF88130DDE911325A40EE
:10B938000D9BEB5C53400F9AB25C53408DF88230FC
:10B94800129A0E9B53400B9AB25C5A400F9BEB5CC9
:10B958001C995A408DF88320169B189A5340139AC5
:10B96800AA5C5340149AB25C53408DF88430DDE9E8
:10B9780018325A40149BEB5C5340159AB25C534002
:10B988008DF88530DDE919325A40159BEB5C534040
:10B99800179AB25C53408DF886301A9A169B53401A
:10B9A800139AB25C5340179AAA5C1EA853408DF8AC
:10B9B8008730FFF79DFDB8E6FF2049E794F00008BF
:10B9C80094EF000894EE000808B538B1044A054918
:10B9D8001060D82200F0B4FA002008BD0220FCE76D
:10B9E800C8190020C4F500080A4B1A6870B500236E
:10B9F80002F1180503EB03142E5D864204D11834B6
:10BA080022440A60002070BD01330B2BF2D10320C1
:10BA1800F9E700BFC81900202DE9F041CCB006466F
:10BA2800DDF8488117461C460D4631B3B8F1000FC2
:10BA380023D006A8FFF726FC204601A9FFF7D4FF6C
:10BA48000446B0B9019906A80131FFF72BFC26B1CD
:10BA58001022314606A8FFF72AFC3A46294606A8CE
:10BA6800FFF725FC06A902A8FFF78CFC029BC8F883
:10BA7800003020464CB0BDE8F0810224F9E7000010
:10BA880030B595B013A90446FFF7AEFF002830D1B2
:10BA98001B4B0C2101FB00F2D5189A5CA2422AD15B
:10BAA800139B1A7C1092DA7B0F929A7B0E925A7B28
:10BAB8000D921A7B0C92DA7A0B929A7A0A925A7A37
:10BAC80009921A7A0892DA7907929A7906925A793B
:10BAD80005921A790492DA7803929A7802925B783E
:10BAE80001930022AB6800931146064B022002F036
:10BAF80013FA15B030BD01300B28CBD1F9E700BFE0
:10BB08000CF3000894F1000810B40B2B019C03D827
:10BB1800019410BCFFF780BF032010BC704730B5FC
:10BB28000D4685B01446014668B103AA002000926C
:10BB38002A460390FFF770FF18B90398001B18BF37
:10BB4800012005B030BD0220FBE72DE9F0430D468A
:10BB5800BFB014469946804620B31BB311F00F01BD
:10BB680022D1F02201A800F0FFF920466946FFF72C
:10BB78003BFF044648B9009801AA10210130FFF79D
:10BB88003BFD2E46AF1BFFB21EB920463FB0BDE8B5
:10BB9800F08301AA09EB070108EB0700FFF7AEFDE8
:10BBA800103EEFE70224F0E70524EEE7F0B5184E63
:10BBB8003468024685B00846002304F1180103EBF7
:10BBC80003154F5D97421ED10D2A05F1190513D1B2
:10BBD8000023CDE90033CDE902330C2210216B4656
:10BBE800FFF7B3FF0446306810226946284400F086
:10BBF800A7F9204605B0F0BD01461022601900F0F3
:10BC08009FF90024F5E701330B2BD8D10324F0E783
:10BC1800C819002009B1FFF7C9BF022070471FB536
:10BC28001446A0B10C2A01D10B2912D10023CDE969
:10BC38000033CDE902330A466B461021FFF785FF32
:10BC480018B969462046FFF7B1FF04B010BD0220BD
:10BC5800FBE70320F9E7F8B51E46DDE907479DF83D
:10BC680018505BB354B34FB3212D29D819462A462F
:10BC7800204600F065F90122631C691EB018FFF721
:10BC880064FFF8B9E37ADB093B70EBB96319204626
:10BC980013F8012C13F8021C120642EA014213F8A9
:10BCA800041C0A4313F8031C012342EA0122291F3A
:10BCB800FFF735FF003818BF0120F8BD0220FCE768
:10BCC8000520FAE70720F8E70420F6E710B5044650
:10BCD80028B1044B5B6998472060002010BD022002
:10BCE800FCE700BF24F4000808B5014630B1044B56
:10BCF8000822186800F024F9002008BD0220FCE79B
:10BD0800C819002008B530B1044B0822196800F0A2
:10BD180017F9002008BD0220FCE700BFC819002061
:10BD28007FB5124E0023044602A801930D46FFF783
:10BD3800E9FF33685B6901936CB102AA082312F822
:10BD4800011B41B9013B13F0FF03F8D102A8A0473A
:10BD580002A8FFF7C9FF35B1019B23B901A8A8477D
:10BD68003368019A5A61002004B070BDC8190020D8
:10BD780008B5014638B1054B18680822104400F090
:10BD8800DFF8002008BD0220FCE700BFC81900202A
:10BD980008B538B1044B19680822114400F0D0F8EE
:10BDA800002008BD0220FCE7C8190020034B1B68CF
:10BDB80002280CBF1961596100207047C81900207A
:10BDC80049B1064B1B68D3E90423022808BF134670
:10BDD8000B60002070470220704700BFC819002080
:10BDE80030B58FB0002405460CA80994FFF78AFFE8
:10BDF8009DF8373007939DF8363006939DF8353017
:10BE080005939DF8343004939DF8333003939DF8DF
:10BE1800323002939DF8313001939DF83030009311
:10BE2800224621461E4B022002F076F80AA8FFF7A8
:10BE3800AFFF9DF82F3007939DF82E3006939DF89D
:10BE48002D3005939DF82C3004939DF82B300393E7
:10BE58009DF82A3002939DF8293001939DF82830E7
:10BE6800009322460F4B2146022002F055F809A9FB
:10BE78002846FFF7A5FF9DF8243003939DF8253049
:10BE880002939DF8263001939DF8273000932246AF
:10BE9800054B2146022002F03FF80FB030BD00BF2D
:10BEA800F0F100082EF200086CF2000808B5002036
:10BEB800FFF7E6FD0120FFF7E3FD0920FFF7E0FDAE
:10BEC8000820FFF7DDFD0020FFF78AFF002008BDEE
:10BED80010B504460B20FFF7D3FD0C20FFF7D0FD6B
:10BEE8000920FFF7CDFD0820FFF7CAFD0A20FFF75C
:10BEF800C7FD2046FFF774FF002010BD014B1860F6
:10BF0800704700BFF80000200B4A30B514680B4D8D
:10BF180043F2390305FB04331360091A6FF000423A
:10BF2800B3FBF2F2C2EBC27201319B1A93FBF1F23E
:10BF380001FB1233184430BDF80000206D4EC64195
:10BF480001380A44914200D1704711F8013B00F8CA
:10BF5800013FF7E710440A44914200D1704711F8B5
:10BF6800013B00F8013DF7E702F008BD30B530B1FC
:10BF78000A4D01444FF0FF33814201D1D84330BD0F
:10BF880010F8012B5340082243F30004013A2C40D7
:10BF980092B284EA5303002AF6D1EDE72083B8ED84
:10BFA80001207047054B4FF400529A62044B1B68FE
:10BFB80013B15B6803B11847704700BF000400481D
:10BFC800581A0020054B4FF480529A62044B1B68A4
:10BFD80013B1DB6803B11847704700BF000400487D
:10BFE800581A0020012070470120704701F03EB91F
:10BFF80001F02CB910B501F00FFE0E21044640F6F1
:10C008001F1001F023F92046012101F0EFFDBDE8E2
:10C01800104001F0CDBA000070B50C4E01EB4003A2
:10C028000D46B3654FF6FF71002304461A460846CD
:10C0380001F054FB96F85600002101F0D7FD29467F
:10C048002046BDE8704001F08BBA00BFFC19002003
:10C0580010B5044601F0A0FE01281CD101F0A4FE91
:10C0680034B11248214602F00BFB104802F0CEFA18
:10C078000F4C104B00214FF48052A1659A6194F83F
:10C08800560001F0B3FD63786BB16FF07F40BDE8F7
:10C09800104001F049BA002340F262211A460846CE
:10C0A80001F01CFBDCE7A0688001F0E7CC19002058
:10C0B800FC19002000040048002001F0B5B9000078
:10C0C80008B501F0BDF80438C0B2032896BF024B8A
:10C0D8000020185C08BD00BFEEF3000808B501F0A9
:10C0E800B0FD033008BD01F03FB901F0FFB808B555
:10C0F80001F0F6FC08BD000038B50D46144601F005
:10C1080053FB284601F088FD0E21054640F61F1016
:10C1180001F09CF828460121074D01F067FD01F068
:10C1280047FA4FF47A716143284602F0A9FA284683
:10C13800BDE8384002F06ABAE419002001F034BBC7
:10C1480008B5084B002193F8560001F04FFD002375
:10C158004FF4C0711A46084601F0C0FABDE808401D
:10C1680001F01ABAFC19002010B5044601F014FEBB
:10C1780001281CD101F018FE34B11248214602F002
:10C188007FFA104802F042FA0F4C104B00214FF48E
:10C198008052A1659A6194F8560001F027FD6378F2
:10C1A8006BB16FF07F40BDE8104001F073B9002318
:10C1B80040F262211A46084601F090FADCE7A068CE
:10C1C8008001F0E7CC190020FC1900200004004889
:10C1D80008B54FF0040001F00DF9BDE80840022051
:10C1E800F5F760BB08B500231A461946184601F052
:10C1F80075FABDE8084001F063B900001D4B73B53E
:10C208001D4D186000241D486C70C5E90144AC65DB
:10C2180001F08EFAAC8101F0F9F92146204601F0CF
:10C2280041FC21460422012001F0F2FA144E154D7A
:10C238004FF6FF7123462246084601F04FFAFFF7F2
:10C24800C7FF2246104B00944FF0FF31304602F0F2
:10C2580031F90E4B009422464FF0FF31284602F088
:10C2680029F9304602F084F9284602B0BDE870404A
:10C2780002F07EB9581A0020FC19002039D20008B3
:10C28800E4190020CC190020ADBF0008CDBF00087C
:10C298000128084805D1084BC17719700E3001F004
:10C2A8009DBB437D012B03D1034B81751970F5E7C5
:10C2B800704700BFFC190020FC0000200D4B10B592
:10C2C800044618735873012000F016F85CB1342145
:10C2D8004FF4E86000F0BAFF4421BDE8104040F296
:10C2E800417000F0B3BF14214FF4E86000F0AEFFD6
:10C2F8002421F2E7FC19002038B5114C05462070BE
:10C3080001F057FD052D04D8DFE805F0090B0317E8
:10C318001709032001F066FA0023637338BD002073
:10C32800F8E7012001F05EFA207B637B8342F5D0B9
:10C338006073BDE83840FFF7C1BF0220EAE700BFDD
:10C34800FC1900202DE9F0431E4687B0002305465E
:10C35800CDE901330C46174601F01DFD032D5BD8CE
:10C36800DFE815F07A00C1000C010400A27C082A5D
:10C3780069D8A16801A801F0D5FE2168002962D01A
:10C3880042F210729142E37C874D50D80322AA737F
:10C3980085F83820E96385F844304FF0020863686F
:10C3A800A17DDB002B820423AB74A37CDB00EB7440
:10C3B80002294FF000032B75637D02D0227D022AEB
:10C3C80046D103F10F02D2B2012A01D9012B3AD189
:10C3D800764B774A196803944FF0010903A88DF842
:10C3E800149001F0D5FC70BB287685F81790687515
:10C3F800FFF762FE4046FFF77FFF6E4801F082FAC2
:10C408006D4801F0EBFA01A800F080FF208A00F0E7
:10C4180051FFA08900F096FF384601F0FDFB624C01
:10C4280084F8560001F0BCFC666000200DE04FF077
:10C438000008E963890885F80E8085F8388085F852
:10C4480044302964ABE74FF0FF3007B0BDE8F08314
:10C45800EB7529766A75CBE72368002BF3D0A27CAD
:10C46800082AF0D8504DA16801A801F05BFE00230E
:10C4780085F838302268EA63E27C85F84420A269AE
:10C48800AB732A646268D2002A820422AA74A27C4E
:10C498002B75D200EA74A27D022A02D0237D022BDA
:10C4A8001CD1627D02F10F03DBB2012B01D9012AF5
:10C4B800C9D13E4B3E4A196803944FF0010803A8BE
:10C4C8008DF8148001F064FC0028BCD1287685F82A
:10C4D80017806875FFF7F0FD00208CE7617DE9752E
:10C4E8002A766B75F6E7304D012185F838102278E9
:10C4F80085F85020637885F85130A37885F8523054
:10C50800E3788B4202D0022B03D03BB985F8533035
:10C5180004E00B3A012A29D885F853104FF0010896
:10C5280085F80E80A388AB83A379AB77E37985F888
:10C538002030237A85F82130FFF7BEFD4046FFF70B
:10C54800DBFE1C4801F0DEF91B4801F047FA95F8BC
:10C558005130062B40F689000AD100F087FE00F022
:10C56800FB0140F6890000F071FE55E70023CDE796
:10C5780000F07CFE40F00401C9B2F2E72368013BF9
:10C58800B3F57A7FBFF45FAF0320FFF7B5FE064827
:10C59800022380F8383023688364162380F84C30EF
:10C5A800383001F0AFF937E7FC190020581A00209D
:10C5B800E4190020341A00200A1A0020F0B51E469B
:10C5C80087B00023CDE90133144607460D4601F034
:10C5D800E2FB002C724C16BF012300230026637077
:10C5E80027B1012F7AD0002007B0F0BDAB68002B2F
:10C5F80000F0D280EB68002B00F0CE80AA7F082ADA
:10C6080000F2CA80296901A801F08CFD2868003869
:10C6180018BF012000F0D6FF84F83870AB68E363D8
:10C6280095F8203084F84430686801F057FBA77308
:10C6380084F84500EB68DB002382EB7FA374AB7FB3
:10C64800DB00E37495F82130237595F82230002B30
:10C658003ED12A7D95F82410A275022995F8232049
:10C6680001D0022B36D102F10F03DBB2012B02D924
:10C67800012A40F0918000238DF81430494B4A4A32
:10C688001968049503A801F083FB002840F0848012
:10C6980001232076E3756075FFF70EFD0020FFF794
:10C6A8002BFE424801F02EF9414801F097F901A804
:10C6B80000F02CFEA88B00F0FDFD288B00F042FE58
:10C6C8004FF4FA53AA687343B3FBF2F3A3608AE703
:10C6D800FF22BFE7E27521766375DDE72B8E002B1D
:10C6E8005AD095F83230A86A012B0CBF2F7DFF274E
:10C6F800003818BF012000F065FFF0B200F06EFFAF
:10C70800012184F8381095F82C2084F8502095F8E9
:10C718002D3084F8513095F82E3084F8523095F841
:10C728002F308B4202D0022B03D03BB984F8533010
:10C7380004E00B3A012A27D884F853102B8EA383E0
:10C7480095F83230A3770126AB8E2384A673E7775A
:10C75800FFF7B2FC3046FFF7CFFD144801F0D2F8DE
:10C76800134801F03BF994F82130B34240F2367097
:10C778000CD100F07BFD00F0FB0140F2367000F0B8
:10C7880065FD4FF6FF73A1E70023CFE700F06EFDCC
:10C7980040F00401C9B2F0E74FF0FF3024E700BFD2
:10C7A800FC190020581A0020CC190020341A002047
:10C7B8000A1A00202DE9F04F85B082460E9DBDF87B
:10C7C80040809DF844709DF84890019193461E461C
:10C7D80001F0E1FABAF1010F524C54D0BAF1040F4A
:10C7E80000F09180BAF1000F3AD10B22304684F85C
:10C7F800442084F838A0E56301F070FA4FEAC803D2
:10C80800B9F1000F238241F6040363820CBF0123B0
:10C81800F223E37587F001070123237684F84500A6
:10C82800C4F840B084F80EA084F814A06775FFF728
:10C8380043FC5046FFF760FD04F1380001F062F850
:10C8480004F10E0001F0CAF8374A1068516802ABCB
:10C8580003C302A800F05AFD40F2FF1000F02AFDC1
:10C86800019801F0D9F90E2184F8560040F61F10FE
:10C8780000F0ECFC94F8560001F092FA169B636005
:10C8880005B0BDE8F08F294984F838A0EAB2895D7F
:10C8980084F8502076BB0B3D012D8CBF0025012567
:10C8A800053A012A04D8B8F10C0F38BF4FF00C082C
:10C8B8001F4B9DF83C201B7884F85350E3770125E3
:10C8C8009DF8543084F8511084F8522084F82130AF
:10C8D800A573A4F81C80A77784F82090FFF7ECFBD9
:10C8E8002846FFF709FD134801F00CF8124801F03B
:10C8F80075F8B5E7012E04D1A5F10C035D425D4141
:10C90800CEE70025CCE75046FFF7F6FC022384F873
:10C91800383004F138001623A56484F84C3000F050
:10C92800F1FF9DE7FC19002048EB000820F40008FF
:10C93800FC000020341A00200A1A00202DE9F04FCC
:10C9480087B0DFF8B4B29DF864A09DF84C900293CC
:10C9580014469DF854309DF85020BDF84880039245
:10C9680005468BF801A0BDF8446001930F4601F01D
:10C9780012FABAF1000F18BF4FF00008DFF87CA2D6
:10C98800039AB9F1000F08BFFF22012D8AF8002091
:10C9980000F0C880052D48D0002D40F0C080284602
:10C9A80000F010FE0B2238468BF844208BF83850E4
:10C9B800CBF83C4001F092F9019B8BF8450041F619
:10C9C8000402002BABF812209AF800208BF81620EE
:10C9D8000CBF0122F2228BF81720F600012289F001
:10C9E80001098BF818208BF80E50ABF810608BF803
:10C9F80014508BF81590FFF75FFB2846FFF77CFC77
:10CA08000BF1380000F07EFF0BF10E0000F0E6FF9E
:10CA18007B490868496804AA03C204A800F076FCA8
:10CA280040F2FF1000F046FC71E0012000F0CAFD62
:10CA380009224FF000098BF8442038464FF4487219
:10CA4800CBF840208BF83890CBF83C4001F046F901
:10CA58004FF48052ABF812209AF800208BF845006A
:10CA68008BF8162028460122F6008BF817208BF841
:10CA78000E90ABF81060ABF814908BF81890FFF795
:10CA88003BFC0BF1380000F03DFF0BF10E0000F00D
:10CA9800A5FF5B498868C96804AA03C204A800F016
:10CAA80035FC40F2FF1000F005FC40F6B80000F03D
:10CAB800DDFB00F0EF0140F6B80000F0C7FB0421F1
:10CAC80040F6B90000F0C2FB40F69B0000F0CEFB38
:10CAD80000F0E30141F0080140F69B0000F0B6FBCE
:10CAE80040F2D16000F0C2FB40F01801C9B240F238
:10CAF800D16000F0ABFB40F2AC6000F0B7FB00F097
:10CB08008F0141F0500140F2AC6000F09FFB4FF400
:10CB1800FA5202FB08F2B2FBF4F2CBF8082007B095
:10CB2800BDE8F08F002000F04DFD36498BF83850F5
:10CB3800E2B2C95D8BF85020002F4DD10B3C012C7F
:10CB48008CBF00240124053A012A02D80C2E38BFD4
:10CB58000C26029B9AF800208BF852308BF8534031
:10CB6800019B8BF81F2001249DF860208BF8212061
:10CB78008BF851108BF820308BF80E40ABF81C6006
:10CB88008BF81E90FFF798FA2046FFF7B5FB1E4872
:10CB980000F0B8FE1D4800F021FF5FFA88F000F0B1
:10CBA8001DFD40F6A30000F061FB00EA040140F619
:10CBB800A30000F04BFB9BF82120A24240F2367004
:10CBC80013D100F053FB00F0FB0140F2367000F087
:10CBD8003DFB4FF6FF72A0E7012F04D1A4F10C032F
:10CBE8005C425C41AFE70024ADE700F03FFB40F05A
:10CBF8000401C9B2E9E700BFFC190020FC000020CD
:10CC080048EB000820F40008341A00200A1A002013
:10CC1800F0B58BB00D46044617461E46FFF74CFA92
:10CC28000020FFF769FB204600F0BEFD0024012329
:10CC3800CDE9084303234FF4167229462046CDE96F
:10CC48000644CDE90444CDE90244CDE90053234626
:10CC5800FFF774FE2046FFF787FAFFF73FFAF4F76D
:10CC680021FE01F041FC0446204601F047FCB04299
:10CC780005D30124FFF720FA20460BB0F0BD00F0E1
:10CC88002FFF8742F0DA0024F4E70000F7B500230D
:10CC98000C4640F201211A460646084600F01EFDE1
:10CCA800644B654D4FF400529A6195F85600012186
:10CCB80000F09CFF2B78012B40F6890013D195F8E2
:10CCC8005130062B0FD100F0D1FA00F0FB0140F6ED
:10CCD800890000F0BBFA2B78042B6CD8DFE803F04E
:10CCE800524B527F090000F0C1FA40F00401C9B26A
:10CCF800EDE7524A731E1046C6F101074FF0000CCB
:10CD0800F9188C426FDC0022E7001346BA4271D151
:10CD18009A0142EAC3125B0183F020031343661CA5
:10CD28000355F6B202234648AB73AE7600F056FEC2
:10CD38000021F12000F08AFA0021F02000F086FAA4
:10CD4800AB6C642B70D17021F32000F07FFA1D21A9
:10CD5800F22000F07BFAE1008C1CF420090A00F0B4
:10CD680075FA04F0FE01F52000F070FA33486FF010
:10CD78007F4231461DE0EC77314800F02FFE00225B
:10CD8800214615E001F008F80128074625D121467B
:10CD98000DF10702304601F004F80446A0B99DF8E9
:10CDA80007302748AB7500F019FE9DF8071022469A
:10CDB800304600F065FB6968224801F061FC2148B3
:10CDC80001F024FC002006E01F4B3A460021022017
:10CDD80001F0A2F8032003B0F0BDAC75CCE7022344
:10CDE800AB73AC76C8E713F8011FC943197002F892
:10CDF80001CB85E7D1106FEA020C715C0CF0070CCF
:10CE0800013241FA0CF101F001014FEAE20C4B400A
:10CE1800D14310F80CE001F0070103FA01F141EAEF
:10CE28000E0100F80C1071E7E121F32000F00EFA72
:10CE380004218DE700040048FC1900205C1A00203A
:10CE48000A1A0020E419002090F30008F0B5BDF894
:10CE580014409DF818709DF81CE09DF8205040B1D2
:10CE6800012814D00122002398180138B0FBF2F0F1
:10CE7800F0BD87F00107E30003EBC70318330EEB9F
:10CE8800450503EBC5034FF47A714B43ECE7501F9C
:10CE9800012803F1040302D80C2C38BF0C24D1B9A3
:10CEA800A2F10B0CBCF1010F8CBF4FF0000C4FF03E
:10CEB800010C2801002F00EBCE000CBF1425002523
:10CEC800A0EB8200062A4FEA82062844A2F1020754
:10CED8000DD8354610E0012906D1A2F10C00D0F199
:10CEE800000C4CEB000CE4E74FF0000CE1E70830D5
:10CEF800BCF1000FEDD0BD000028ACBF2E182E1CD1
:10CF0800701E90FBF5F003FB0044094B062A5A5C9F
:10CF18008CBF0C340E340A2A09D8A30001334FF40D
:10CF28007A71BB404B43034951F822209CE7FFDE4E
:10CF380020F40008F4F3000808B5094B012193F820
:10CF4800560000F053FE4FF4D7602D2100F07EF913
:10CF580000F033FBBDE80840024800F07BBA00BF90
:10CF6800FC190020FFFF0F0073B5A44CB4F854302F
:10CF78000025202B8DF80350019500F01B8114D853
:10CF8800082B0DD87BB1013B072B0CD8DFE813F039
:10CF980042005B000B00CD000B000B000B00FD00F6
:10CFA800102B00F0008102B070BDB3F5807F00F057
:10CFB800988011D8402B00F01081802BF3D128469F
:10CFC80000F032FA8E4B1B68002BECD09B69002BCB
:10CFD800E9D028469847E6E7B3F5007FE3D1894BC7
:10CFE80001222946022000F097FF00F029F90428C1
:10CFF80040F08580844B85484FF400529A6201F0D6
:10D00800B7FA284600F010FA7D4B1B68002BCAD0EF
:10D018005B6814E07C4B7D484FF400529A6201F043
:10D02800A7FA002000F000FA00F0B8FE012801D1AC
:10D0380000F0BDFE724B1B68002BB4D01B68002BA0
:10D04800B1D09847AFE7704B71484FF480529A625D
:10D0580001F08EFA657895B9284600F0E5F9294679
:10D0680040F6021000F0F2F840F6441000F0FEF826
:10D0780040F00201C9B240F6441000F0E7F8FF2280
:10D088000DF1030163485E4D00F05AFD624800F05F
:10D0980071FD2B68002B86D09E68002E83D094F8F3
:10D0A8002430012B08D194F9313094F930209DF8BF
:10D0B80003105848B04776E7E06B01A900F022FE5C
:10D0C800019B9DF8031053484FF47A7203F5FA73E5
:10D0D80093FBF2F32A685BB2956894F92920A84774
:10D0E80061E7284600F0A0F9454B1B68002B3FF488
:10D0F8005AAF9B69002B3FF456AF01206AE700F056
:10D108009FF805287FF44FAF3F4B41484FF48052BA
:10D118009A6201F02DFA284600F086F9384B1B6810
:10D12800002B3FF440AFDB6889E700213B4B01222D
:10D13800022000F0F1FEA16D00293FF434AFC1F3E5
:10D14800074140F6031000F081F894F8591040F6B2
:10D15800041000F07BF894F8581040F6051000F021
:10D1680075F840F6021000F081F840F00101C9B2EC
:10D1780040F6021000F06AF8002340F262211A46D5
:10D188000846A36500F0AAFA0DE7254B0122002105
:10D19800022000F0C1FE00F0FFFD01287FF403AF7C
:10D1A80000F006FEFFE61F4B01220021022000F0DE
:10D1B800B3FEF8E6164801F0DBF9607808B900F02C
:10D1C80033F90F4B1B68002B3FF4EDAEDB68002BE7
:10D1D8003FF4E9AE9847144BE6E7144B0122294681
:10D1E800022000F099FE607808B900F01DF9044BA0
:10D1F8001B68002B3FF4D7AE1B6920E7FC19002001
:10D20800581A0020A5F3000800040048E41900207B
:10D21800CC1900205C1A0020201A0020B9F300085D
:10D22800C2F30008CCF30008D5F30008DEF30008C9
:10D23800024BA3F85400FFF797BE00BFFC1900206B
:10D24800014B1878704700BF6A1B002007B50123FF
:10D258008DF807100DF1070201460348F7F748FA61
:10D2680003B05DF804FB00BFC401002007B501232B
:10D2780001460DF107020448F7F773FA9DF8070015
:10D2880003B05DF804FB00BFC401002010B50446DC
:10D29800F5F778F801280CD140F62310FFF7E6FFE0
:10D2A80000F0F901214340F62310BDE81040FFF7D4
:10D2B800CDBF10BD10B50C4B1B7804469BB94FF47D
:10D2C800D760FFF7D3FFC4F3002100F0FE0001434D
:10D2D8004FF4D760FFF7BAFFE1B240F2B960BDE89A
:10D2E8001040FFF7B3BF10BD691B002010B51346EF
:10D2F800EFF3108472B60A4601460348F7F7F8F9C7
:10D3080084F3108810BD00BFC401002008B5014691
:10D3180008224FF4D860FFF7E9FF002008BD00009D
:10D3280007B5074B1B7840BAADF804002BB90222A9
:10D3380001A940F2BC60FFF7D9FF03B05DF804FB18
:10D34800691B002007B5074B1B7840BAADF80400ED
:10D358002BB9022201A940F2BE60FFF7C7FF03B054
:10D368005DF804FB691B002010B51346EFF3108429
:10D3780072B60A4601460348F7F7F3F984F31088B2
:10D3880010BD00BFC401002010B51346EFF3108490
:10D3980072B60A4601460348F7F7D5FA84F31088AF
:10D3A80010BD00BFC40100200A4601460020FFF757
:10D3B800EBBF000010B51346EFF3108472B60A46AF
:10D3C80001460348F7F7F2FA84F3108810BD00BF4E
:10D3D800C401002010B51346EFF3108472B60A4654
:10D3E80001460348F7F7F8F984F3108810BD00BF29
:10D3F800C401002013B504460020F4F79DFF022065
:10D40800FFF744FF04F0070401220DF1070184200F
:10D418008DF80740FFF7DEFF024B00221A7002B0BA
:10D4280010BD00BF6A1B002007B501228DF8070058
:10D438000DF107018020FFF7CDFF9DF80730002B85
:10D44800034B14BF022201221A7003B05DF804FBDB
:10D458006A1B002007B5094B8DF8060004221A70D4
:10D46800030C8DF804300322030A01A983208DF8E8
:10D478000530FFF7AFFF03B05DF804FB6A1B00201F
:10D4880010B51446FFF790FF2046BDE81040FFF79F
:10D49800E1BF000007B5094B8DF8060005221A7098
:10D4A800030C8DF804300322030A01A982208DF8A9
:10D4B8000530FFF78FFF03B05DF804FB6A1B0020FF
:10D4C80073B5002640F6E2000196FFF7CFFE00F0A4
:10D4D800FE01054640F6E200FFF7B8FE40F6E5001B
:10D4E800FFF7C4FE00F07F01044640F6E500FFF7B1
:10D4F800ADFE6FF07F40FFF7CDFF04220DEB020178
:10D5080040F61900FFF730FF3046FFF78DFF294638
:10D5180040F6E200FFF79AFE214640F6E500FFF7E5
:10D5280095FE019802B070BD13B50C4B0446052258
:10D53800972140F6AC001A70FFF788FE230C8DF88F
:10D5480004300322230A01A982208DF805308DF8C2
:10D558000640FFF73FFF02B010BD00BF6A1B002066
:10D5680007B5030C8DF80030030A8DF801300B0C59
:10D5780049BA8DF80200ADF80410062269469420D5
:10D588008DF80330FFF726FF024B06221A7003B00E
:10D598005DF804FB6A1B0020002208B51146C5206F
:10D5A800FFF718FF014B07221A7008BD6A1B0020FD
:10D5B80000221146D120FFF70DBF00221146D220CC
:10D5C800FFF708BF07B501228DF807000DF1070125
:10D5D8009F20FFF7FFFE03B05DF804FB07B50122AB
:10D5E8008DF807000DF10701A020FFF7F3FE9DF865
:10D5F80007103F2907D901F0F8010131C9B240F2FB
:10D608000670FFF723FE03B05DF804FB07B5F4F7D7
:10D61800B9FE431E584258418DF8070001220DF10A
:10D6280007019620FFF7D6FE03B05DF804FB07B5A7
:10D6380000F07F008DF8070001220DF10701892015
:10D64800FFF7C8FE03B05DF804FB0000154B9842D5
:10D6580007B51BD8144B98421BD8144B98421BD8BB
:10D66800134B98421BD8134B98428BBF6B2229222D
:10D678006F232B238DF8042001A9022298208DF80E
:10D688000530FFF7A7FE03B05DF804FBE122E923AC
:10D69800F0E7D722DB23EDE7C122C523EAE77522AD
:10D6A8008123E7E700E9A43580F8A9328044E52D15
:10D6B800000B6B1B40FC541907B58DF8062004229B
:10D6C8008DF804008DF8051095200DEB02018DF8FA
:10D6D8000730FFF77FFE03B05DF804FB07B552BAC9
:10D6E800ADF8042040BA082249BAADF80000ADF8F8
:10D6F80002105BBA69461046ADF80630FFF76AFEBD
:10D7080003B05DF804FB07B50B0C042200F007001A
:10D7180049BA8DF80400ADF8061097200DEB020108
:10D728008DF80530FFF756FE03B05DF804FB0000E6
:10D7380010B508B1194B1860F3F7B8FF0220FFF7CE
:10D74800A5FD0024164B20461C70FFF76DFEF4F76C
:10D7580017FE012817D14FF42071FFF7D4FF40F6C8
:10D7680011102146FFF772FD4FF07F00FFF75FFFB2
:10D778000E2140F61F10FFF769FDF4F7A9FD094BCC
:10D7880001221A7010BD102140F61110FFF75EFD3E
:10D79800102140F61210FFF759FDE9E75C1B002045
:10D7A800601B00206A1B002037B50C4D2B780446FF
:10D7B8001BB9FFF74BFF01232B700023084A6006B3
:10D7C800E109F3F7EDF9042200BA01900DEB02012B
:10D7D8008620FFF7FFFD03B030BD00BF601B0020AF
:10D7E8000048E80107B5094B8DF807000146187095
:10D7F80018B940F2AC60FFF729FD01220DF10701CD
:10D808008A20FFF7E7FD03B05DF804FB691B0020E1
:10D81800012873B50C46164637D10020F4F7B4FD3D
:10D82800A042B8BF44B20E2805461AD101231A46B1
:10D8380000210420FFF740FF6FF010039C42B8BF9F
:10D848001C46182140F6E700FFF700FD022201A957
:10D858008E208DF804408DF80560FFF7BBFD02B0FF
:10D8680070BD01230A28E4B21A464FF0000105D121
:10D878001846FFF721FF033464B2DDE70720C5F13E
:10D888000E05FFF719FF2C44F6E740F6D800FFF71E
:10D89800EDFC40F01E01C9B240F6D800FFF7D6FCF7
:10D8A8000120F4F771FDA042B8BF44B21428054620
:10D8B8004FF001034FF000020CD105210320FFF7C0
:10D8C800FBFE023464B26FF008039C42B8BF1C46EA
:10D8D8003821B7E7112805D103210220FFF7ECFE14
:10D8E8000534EFE70E2804D102210846FFF7E4FECD
:10D8F800E9E7C5F11605072104202544FFF7DCFEFA
:10D908006CB2E0E713B5314A0446516810686B46BB
:10D9180003C32F4B20781B78834201D0FFF762FFA7
:10D928002378032B27D8DFE803F00239283C626804
:10D93800284BB3FBF2F31A0CA1688DF800208DF880
:10D9480002301A0A237B8DF80330637B8DF801209F
:10D958008DF80430204A00234806C909F3F720F956
:10D96800030C40BA8DF80530ADF806000822694668
:10D978008B20FFF72FFD02B010BD2269154BB3FBBA
:10D98800F2F31A0C8DF800208DF802301A0A237D64
:10D998008DF801208DF803300422E8E7A36900938D
:10D9A800FAE762680B4BB3FBF2F31A0C8DF8002010
:10D9B8008DF802301A0A237B8DF80330637B8DF8CB
:10D9C80001208DF804300522D1E700BF58EB00088C
:10D9D800691B00200000093D0048E8011FB52E4AD8
:10D9E8000446D1689068127C01AB03C31A702B4BB4
:10D9F80020781B78834201D0FFF7F4FE2378032BAD
:10DA080026D8DFE803F002383302637AF12B21D1FC
:10DA18004FF6FF70FFF784FC48F20500FFF792FC11
:10DA280002236288A188ADF8061052BAE188ADF8E1
:10DA380004208DF80B30227AA37A8DF80A20ADF8ED
:10DA480008108DF80C30092201A98C20FFF7C2FCC0
:10DA580004B010BDF22BE4D141F60F50FFF760FC83
:10DA680041F22100FFF76EFC0623DAE7237B8DF8ED
:10DA780004300122E8E7E389094A5BBAADF80430CB
:10DA8800237C13708DF80630637C8DF80730638A29
:10DA9800ADF808300622D7E758EB0008691B0020CC
:10DAA800681B002007B502228DF804008DF80510C8
:10DAB8008F2001A9FFF78EFC03B05DF804FB00007E
:10DAC80010B51346EFF3108472B60A4601460348B0
:10DAD800F6F7BAFE84F3108810BD00BFC401002019
:10DAE80007B5012201A91520FFF7EAFF9DF80400F8
:10DAF8004042401003B05DF804FB000037B505460E
:10DB08000C46022201A91320FFF7DAFF0A4B1B7803
:10DB1800012B0DD1094B1B78012B09D140F2027062
:10DB2800FFF7A4FB9DF805302870237003B030BDC3
:10DB38009DF80400F6E700BF691B0020681B002061
:10DB4800F7B50D46064600240DF10701284617468D
:10DB58008DF80740FFF7D2FF2A78BA4207D89DF818
:10DB680007003146FFF726FC204603B0F0BD012030
:10DB7800FBE7000013B50322044601A91420FFF7B0
:10DB88009FFF184B1A7822704AB1012A17D0142225
:10DB98000021204600F0D0FA0F2323700DE09DF8F5
:10DBA800043023719DF80530A2605B425B10A371BD
:10DBB8009DF806305B425B10637102B010BD9DF8A2
:10DBC80004305B425B1023739DF9053002339B10D0
:10DBD80063739DF806305B425B10A373024B1B68AE
:10DBE8002361EAE7691B0020641B0020012908B5AE
:10DBF800034608460ED1012B07D10420FFF746FB48
:10DC08000220BDE80840F4F797BB022B14BF084672
:10DC18000320F6E70120F4E738B50446F4F7AEFB35
:10DC280050B102280CBF02250125284602222146B0
:10DC3800FFF7EEFD284638BD102CB4BF012502259C
:10DC4800F3E70A2070470000014B01201B681847C2
:10DC58005C1B0020014B02201B6818475C1B00203E
:10DC6800014B40201B6818475C1B002011B101299B
:10DC780004D07047044B1B6880201847024B4FF4B0
:10DC880080701B68F9E700BF5C1B0020024B4FF453
:10DC980000701B68184700BF5C1B0020014B202048
:10DCA8001B6818475C1B0020014B04201B681847A1
:10DCB8005C1B0020014B08201B6818475C1B0020D8
:10DCC800014B10201B6818475C1B0020024B4FF4C7
:10DCD80080401B68184700BF5C1B002010B568B166
:10DCE800074A002352F83340844202EBC30101D9AA
:10DCF800087910BD0133162BF4D1FEE71F20F8E791
:10DD0800B0F4000873B51D4B0193044640F60700B4
:10DD18000D46FFF7ABFAC0F3C10308336B4413F8A1
:10DD2800042C00F00703013302FA03F3144AB2FB90
:10DD3800F3F2B2FBF4F007281ED84000042834BFE1
:10DD4800042302234FF4D66002FB03F4FFF78EFA94
:10DD5800060240F2B160FFF789FA06F470663043B4
:10DD6800030544BF6FEA00506FEA1050630943434C
:10DD7800DB112B6002B070BD0123E3E704080A0C35
:10DD88000048E8014FF0FF3070474FF0FF30704710
:10DD98004FF0FF30704770470020704700207047F1
:10DDA80070474FF0FF3070474FF0FF3070477047B3
:10DDB8007047704770B5EFF3108672B6144B5C8AE3
:10DDC8001A8A944213D1C4F5806292B2904206D363
:10DDD800844218D901229A7000221C805A825A8AD9
:10DDE8000A800244C2F309025A8200200DE006D9D3
:10DDF800C4F58065ADB28542F1D88242E9E7121BCD
:10DE080092B28242EBD84FF0FF3086F3108870BD93
:10DE18006C210020EFF3108172B6034AD38A0133D4
:10DE2800D38281F3108870476C210020EFF31081B2
:10DE380072B6034AD38A013BD38281F310887047B4
:10DE48006C21002010B508481822002100F074F950
:10DE580006484FF48062002100F06EF9044B054833
:10DE68001B68BDE8104018476C2100206B1D00207E
:10DE7800D0EB0008E9DF0008014B5860704700BF8D
:10DE88006C210020014B1872704700BF6C210020E4
:10DE980073B5EFF3108572B61C4CE08A00282FD1B9
:10DEA800FFF7B8FF218A628A914227D0A378012B15
:10DEB80012D1238820805B1A9BB20221A382A17011
:10DEC80063B9A3702382238A9A428BBFD21AC3F5FF
:10DED8008063A282A38201E0002BF4D0268A0C4B37
:10DEE8001E4485F31088F3F7CBFC0A4BA18ADB6844
:10DEF8000193304602B0BDE870401847FFF796FF1F
:10DF080085F31088002002B070BD00BF6C2100208E
:10DF18006B1D0020D0EB000808B4F0B586B00023D4
:10DF2800ADF800302B4B0B9C1D7A85424CD3D8683A
:10DF380081434CD15B681BB112B1694602A898476E
:10DF48000CAB22464FF400712348019300F0F4FB18
:10DF5800FFF760FFBDF8003018440DF1020180B2F0
:10DF6800FFF728FF01302AD00023BDF80020BDF8B4
:10DF780002601A480DF1080C1F4699B216FA83F58B
:10DF88008A42ADB215D817B13244ADF80220BDF8B7
:10DF98000250019B22464FF40071284400F0CCFB4C
:10DFA800FFF744FFFFF774FF06B0BDE8F04001B08B
:10DFB80070471CF8011B415501330127DDE7FFF7C6
:10DFC80035FF6FF00200EFE76FF00400ECE76FF049
:10DFD8000500E9E76C2100206B1B00206B1D002069
:10DFE80013B5EFF3108472B6204B9A78588A022A38
:10DFF8001DBF1A8A998A5218002214BFC2F3090257
:10E008009A7090421A8228D0D98A012925D1997804
:10E01800012913D119888A1A022192B29970002114
:10E028009A82198062B99A701A821A8A90428BBFB2
:10E03800801AC2F5806298829A8201E00029F4D0A1
:10E04800188A0B4A104484F310880A4A998AD368BC
:10E05800019302B0BDE81040184784F31088F3F725
:10E0680013FC02B0BDE81040FFF7E0BE6C210020B1
:10E078006B1D0020D0EB0008024A00231360024AFF
:10E0880013607047882100208421002010B5EFF329
:10E09800108472B641B1012903D1064A13680343BB
:10E0A800136084F3108810BD024A136823EA000342
:10E0B800F6E700BF8821002010B5EFF3108472B690
:10E0C80041B1012903D1064A13680343136084F35D
:10E0D800108810BD024A136823EA0003F6E700BF60
:10E0E8008421002038B5EFF3108572B60A4B0B4C2B
:10E0F8001B6833B1236898476368984785F310888D
:10E1080038BD074B1B681BB1A3689847E368F4E761
:10E11800236998476369F0E7882100206CEB0008C1
:10E128008421002001380A44914200D1704711F837
:10E13800013B00F8013FF7E700F020BC10B5EFF312
:10E14800108472B6064A136803431360054A52F8EE
:10E158003130034342F8313084F3108810BD00BFDA
:10E16800B02100208C21002070477047B0F5803F17
:10E178003ABF000410230023B0F1807F3EBF08336C
:10E188000002DBB2B0F1805F38BF00014FEA1070C7
:10E19800054A38BF0433125C38BFDBB2C3F11F0332
:10E1A800981AC0B2704700BF60F500082DE9F84F13
:10E1B800384D394ED5F80080DFF8E0B0DFF8E0A040
:10E1C800DFF8E090D6F800C0374FDBF80010374C86
:10E1D800DAF80020D9F8003008EA0000286028683A
:10E1E80000EA020E1EEA0C0F01D019421ED04FF0B1
:10E1F800FF333B60FFF7B8FFEFF3108472B6336864
:10E20800DBF80020DAF800100B4029680B4205D132
:10E21800D9F80030134201D1F3F7C0FA84F310881B
:10E22800FFF7A3FFC5F80080BDE8F88F23682368CF
:10E238000340134062681A4204BF4FF0FF32626025
:10E2480060681840FFF792FF62683860012303FA9C
:10E2580000F022EA00026260EFF3108172B63A68B9
:10E268009340326822EA03023260226822EA0303FA
:10E27800236081F310880E4A3B6852F82330984790
:10E28800D6F800C0DBF80010DAF80020D9F8003022
:10E29800A5E700BF00010020B0210020AC2100202C
:10E2A80004010020A8210020A42100208C210020A6
:10E2B8009421002010B51146EFF3108472B6FFF7D1
:10E2C80055FF034B43F8201084F3108810BD00BF9E
:10E2D8009421002082B082B00DF1080C0CE90600F0
:10E2E800BDF8042003930B44BDF810100A4491B202
:10E2F80012B2B2F57A7FA2BFA1F57A72013312B2D7
:10E308000360828002B002B0704782B082B00DF123
:10E31800080C0CE90600BDF804200393CB1ABDF8DD
:10E328001010521A91B212B2002ABEBF01F57A72C9
:10E3380003F1FF3312B20360828002B002B070476B
:10E3480030B585B0114D6B4683E803000023029376
:10E35800ADF80C3003A82B699847009BBDF8044022
:10E368000290181ABDF80C30E41AA3B224B2002C9B
:10E37800BEBF03F57A731CB200F1FF302B689847D3
:10E38800AB682046984705B030BD00BF90EB000849
:10E3980073B5114E002305460093ADF8043001A86B
:10E3A80033699847F368009098477368044698471C
:10E3B800009B1844BDF8043023449AB21BB2B3F54D
:10E3C8007A7FA2BF0130A2F57A731BB22860284673
:10E3D800AB8002B070BD00BF90EB000837B50023DA
:10E3E8000093ADF80430074B04461B6901A8984711
:10E3F8006D46009095E8030084E80300204603B0CA
:10E4080030BD00BF90EB000837B50F4D02AB03E9F4
:10E418000300EB6898476B6804469847BDF80430DA
:10E42800009A1B1B99B21BB2002BA2EB0002BEBFC5
:10E4380001F57A7102F1FF320BB24FF47A7000FBEA
:10E44800023003B030BD00BF90EB00082DE9F04169
:10E458004FF47A75B1FBF5F5C5EB4513DFF83C8051
:10E4680005EB8303A1EBC3039CB2D8F80C30064636
:10E478009847D8F8043007469847E31999B21BB271
:10E48800B3F57A7F2844A2BFA1F57A7301301BB295
:10E498003060B3803046BDE8F08100BF90EB0008E3
:10E4A800024B00221A60024B1B681847B421002057
:10E4B800A4EB0008F8B50446174608461E467CB18A
:10E4C80073B1084B00255B6A25609847069B60601E
:10E4D8002581A572E6602361E77265612846F8BD6B
:10E4E8000120FCE7A4EB000810B5034CE36998474A
:10E4F800A36ABDE810401847A4EB000870B5064DA4
:10E50800EB69064698476B6A044630469847AB6AFB
:10E51800201ABDE870401847A4EB0008054B1B689B
:10E528000BB918467047834201D05B69F8E70120B0
:10E53800704700BFB42100202DE9F3410B4E336A28
:10E54800044698470123B7692372D4F8008005462A
:10E55800B8472844804502D2B84728442060B368A9
:10E568002068019302B0BDE8F0411847A4EB000809
:10E5780070B520B3EFF3108672B6124D2B680122E6
:10E58800827253B10022427298425C690ED10272C3
:10E598003CB120462C60FFF7CFFF86F3108800209F
:10E5A80070BD094BDB6898472C60F6E71A465B6933
:10E5B800002BF2D09842F9D143695361EDE701206D
:10E5C800EEE700BFB4210020A4EB0008084B10B50B
:10E5D8001A685369516911B95061416110BD0468E5
:10E5E80019688C4202D91A465B69F3E71946F3E7C2
:10E5F800B4210020044A13680BB100211972436149
:10E608001060FFF799BF00BFB42100202DE9F04149
:10E61800044600282DD0FFF781FF50BB657A45BB23
:10E62800EFF3108872B6144E6768336A98478742CA
:10E638002CBF27602060114FA5724FF4807323818F
:10E648003B684BB9336998472046FFF7D3FF88F3F7
:10E6580010882846BDE8F081B369984723681844B4
:10E668003B6820601B6898422046EED3FFF7AEFF58
:10E67800EDE70125EDE700BFA4EB0008B421002079
:10E6880010B5044608467CB1084B5B6A9847606041
:10E698002046FFF743FF40B12046FFF769FF2046B9
:10E6A800BDE81040FFF7B2BF012010BDA4EB000881
:10E6B8002DE9F041EFF3108772B61D4E1D4D7369B9
:10E6C80098473369044698472B684BB94FF00008C0
:10E6D8002B688BB9286828BB87F31088BDE8F081C0
:10E6E800011B241A1A688A428CBF121900221A6068
:10E6F8005B69002BF6D1E9E71C681CB1B369984740
:10E708008442E7D22C6863692B60A4F80880D4E9B6
:10E71800033098476389B3F5807FD9D12046FFF746
:10E7280075FFD5E7037A002BD6D1FFF705FFD3E7AE
:10E73800A4EB0008B42100202DE9F04F002997B080
:10E7480081461E4640F3118104464F1E1378A4EB00
:10E75800090023B90023237017B0BDE8F08FB84231
:10E76800F8DA252B05D004F8013B904608F10102A0
:10E77800ECE792F801E0AEF1300102F10108AEF1E8
:10E7880030034A424A41092B2BD8414600250A202A
:10E79800884611F8013BA3F1300CBCF1090F1BD9D5
:10E7A80098F80030692B00F09E801DD8632B29D083
:10E7B800642B00F09880582B5AD0252B1AD198F842
:10E7C8000030002B00F0938004F8013BA4EB090310
:10E7D800BB4280F28A80C9E700FB0533A3F130050C
:10E7E800D6E74FF0FF35DBE7752B7ED0782B41D08D
:10E7F800732B1CD0252304F8013BA4EB0903BB426F
:10E8080073DADCE7002D05F1FF3AD8BF4FF0000AB4
:10E8180052462046202100F0B1F8A244002D56F8B7
:10E82800043B8AF80030D8BF01252C449EE7504BA2
:10E8380056F804BBBBF1000F08BF9B465846F1F7DA
:10E8480097FC2A1A8542B8BF00228246202120461A
:10E85800019200F093F8019A00232244534502DB09
:10E8680002EB0A0482E71BF80310D1540133F5E7E1
:10E8780042F040021021DFF8FCB0DFF8FCA056F8A7
:10E8880004CB12F0400F18BFDA46BEF1300FCDF8B6
:10E8980008A0A4EB09030CBF4FF0300A4FF0200A80
:10E8A8009207A7EB03036046CDF80CA022D50028F9
:10E8B80020DA4042013D4FF02D0C05AA01920022BA
:10E8C8008246B0FBF1F001FB10AB029810F80BB0D8
:10E8D800019800F801BB5145019002F10102BAFB11
:10E8E800F1F0EDD910E042F002020A21C3E708F185
:10E8F800FF386BE7BCF1000F02D04FF0000CDCE7EB
:10E9080030228DF814200122BEF1300FA5EB02054C
:10E9180004D02020002D05F1FF350ADCBCF1000FE2
:10E9280005D02D21013B04F8011B3FF41FAF2544FE
:10E938000AE0013B04F8010BECD117E7039904F84E
:10E94800011B013B3FF412AF291B0029F6DC05A986
:10E95800114423442244A2423FF408AF11F8010DA8
:10E9680004F8010B9C42F6D100E70020F4E600BF52
:10E9780070F500089CF5000877F500080244034686
:10E98800934200D1704703F8011BF9E770B50D4DAC
:10E998000D4C641BA4100026A64209D10B4D0C4C4B
:10E9A80000F09AF8641BA4100026A64205D170BD99
:10E9B80055F8043B98470136EEE755F8043B98476D
:10E9C8000136F2E7A4F60008A4F60008A4F6000849
:10E9D800A8F60008000000002DE9F041C1F30A572D
:10E9E800A7F2FF36132E02460B460C460546804614
:10E9F80035DC002E17DA34A3D3E90023F1F7C6FB80
:10EA080000220023F1F7F6FD50B1002C57DA24F06C
:10EA180000442C430025AC422D4C08BF4FF0004465
:10EA280023462A4624E02B4F374101EA070C5CEACB
:10EA3800000C1DD024A3D3E90023F1F7A7FB002283
:10EA48000023F1F7D7FD0028EAD0002CBEBF4FF411
:10EA580080133341E41824EA07040025E0E7332E45
:10EA68000ADDB6F5806F03D1F1F790FB02460B463D
:10EA780010461946BDE8F081A7F213474FF0FF3C56
:10EA88002CFA07F70742F3D00FA3D3E90023F1F7D5
:10EA98007DFB00220023F1F7ADFD0028C0D0002C3B
:10EAA8000ADA142E01D1013406E0C6F13406012336
:10EAB800B3401D444545F6D325EA0705B0E70025D0
:10EAC8002C46ADE7AFF300809C7500883CE4377EA8
:10EAD8000000F0BFFFFF0F00F8B500BFF8BC08BC8E
:10EAE8009E467047F8B500BFF8BC08BC9E46704704
:10EAF800000000000100000002000000000000000B
:10EB08008813000010270000204E00003075000018
:10EB1800409C000050C3000060EA0000C0D401001F
:10EB280080A903000053070000EA06370000000030
:10EB38005000000040F709370000000050000000B6
:10EB4800C194C10000000000B227000000000000CE
:10EB580000000000000000000000000000000000AD
:10EB6800000000006716000855160008F115000897
:10EB780059160008ED150008791600082564732554
:10EB88003033643A0000000099190008391A000867
:10EB9800A9190008451A0008091A0008511A00089E
:10EBA80000000000B9190008711900083D19000893
:10EBB800F51800084D190008611900080119000826
:10EBC8000519000819190008C11C0008E91C0008EB
:10EBD8006D1C0008591C0008A0860100400D0300A8
:10EBE800801A060000350C0040420F0080841E0089
:10EBF80000093D0000127A000024F40000366E017E
:10EC08000048E801006CDC02000000000000000081
:10EC180000000000000000000000000000000000EC
:10EC280000000000000000000100000002000000D9
:10EC380003000000040000000100000003000000C1
:10EC480005000000010000000100000006000000AF
:10EC58000A0000002000000002000000040000007C
:10EC680008000000100000004000000080000000C4
:10EC7800000100000002000001000200040006007C
:10EC880008000A000C00100020004000800000016D
:10EC98000804020408010101010101030701000041
:10ECA8006572726F723A20526567696F6E20697378
:10ECB800206E6F7420646566696E656420696E20D5
:10ECC800746865204D573A20736574206C6F7261C3
:10ECD80077616E5F636F6E662E68206163636F7223
:10ECE80064696E676C790D0A004D4143207278544F
:10ECF800696D654F75740D0A004D41432074785451
:10ED0800696D654F75740D0A004D41432072784452
:10ED18006F6E650D0A004D4143207478446F6E652F
:10ED28000D0A00080A0C0D0E10121415181A1B1DD6
:10ED38001E21240305020501060202050000060043
:10ED48000001050404020202020202020202020297
:10ED58000202020203020202020202030403020286
:10ED68000202020405040302020202050605040366
:10ED78000202020607060504030202070707060542
:10ED88000403020707000000000000010201000060
:10ED98000000000203020100000000030403020156
:10EDA8000000000405040302010000050605040331
:10EDB8000201000607060504030201070707060506
:10EDC800040302070700000B357DF2F2F2333373B8
:10EDD80073DEDEDEDE33337373F2F2F2F20000002C
:10EDE80048E8010048E8010048E8010048E8010057
:10EDF80048E8010048E8010090D003000000000046
:10EE08000C0B0A090807073252585F2573206F6EEA
:10EE1800206672657120256420487A206174204438
:10EE2800522025640D0A005258206F6E20667265C4
:10EE38007120256420487A2061742044522025647A
:10EE48000D0A005458206F6E206672657120256483
:10EE580020487A2061742044522025640D0A00312C
:10EE68000032004D756C74695F43004D756C7469B0
:10EE78005F50000067EE000869EE000871EE0008B8
:10EE88006BEE000879EE000873EE0008A584998DF2
:10EE98000DBDB1545003A97D1962E69A459D40877E
:10EEA80015EBC90BEC67FDEABFF7965BC21CAE6AAF
:10EEB8005A41024F5CF434089373533F0C52655E19
:10EEC80028A10FB509369B3D2669CD9F1B9E742E40
:10EED8002DB2EEFBF64D61CE7B3E7197F568002CA6
:10EEE800601FC8EDBE46D94BDED4E84A6B2AE5164A
:10EEF800C5D75594CF100681F044BAE3F3FEC08A13
:10EF0800ADBC4804DFC17563301A0E6D4C14352F43
:10EF1800E1A2CC3957F28247ACE72B95A098D17F74
:10EF2800667EAB83CA29D33C79E21D763B564E1EDA
:10EF3800DB0A6CE45D6EEFA6A8A4378B324359B7A1
:10EF48008C64D2E0B4FA0725AF8EE918D5886F72C1
:10EF580024F1C751237C9C21DDDC86859042C4AA1C
:10EF6800D8050112A35FF9D0915827B93813B333E4
:10EF7800BB7089A7B622922049FF787A8FF880174C
:10EF8800DA31C6B8C3B07711CBFCD63AC6F8EEF67C
:10EF9800FFD6DE916002CE56E7B54DEC8F1F89FA99
:10EFA800EFB28EFB41B35F452353E49B75E13D4CC3
:10EFB8006C7EF5836851D1F9E2AB622A0895469DCB
:10EFC80030370A2F0E241BDFCD4E7FEA121D58342E
:10EFD80036DCB45BA476B77D52DD5E13A6B900C1FA
:10EFE80040E379B6D48D67729498B085BBC54FED70
:10EFF800869A66118AE904FEA078254BA25D8005F1
:10F008003F2170F16377AF4220E5FDBF811826C329
:10F01800BE35882E9355FC7AC8BA32E6C0199EA32D
:10F0280044543B0B8CC76B28A7BC16ADDB64741427
:10F03800920C48B89FBD43C43931D3F2D58B6EDAF0
:10F0480001B19C49D8ACF3CFCAF447106FF04A5CC1
:10F0580038577397CBA1E83E96610D0FE07C71CCD1
:10F068009006F71CC26AAE6917993A27D9EB2B228A
:10F07800D2A907332D3C15C987AA50A50359091AE7
:10F0880065D784D082295A1E7BA86D2C637C777B38
:10F09800F26B6FC53001672BFED7AB76CA82C97D8C
:10F0A800FA5947F0ADD4A2AF9CA472C0B7FD93261D
:10F0B800363FF7CC34A5E5F171D8311504C723C321
:10F0C8001896059A071280E2EB27B27509832C1A65
:10F0D8001B6E5AA0523BD6B329E32F8453D100EDBF
:10F0E80020FCB15B6ACBBE394A4C58CFD0EFAAFBA3
:10F0F800434D338545F9027F503C9FA851A3408F6B
:10F10800929D38F5BCB6DA2110FFF3D2CD0C13EC82
:10F118005F974417C4A77E3D645D197360814FDC17
:10F12800222A908846EEB814DE5E0BDBE0323A0AFB
:10F138004906245CC2D3AC629195E479E7C8376D7F
:10F148008DD54EA96C56F4EA657AAE08BA78252EA4
:10F158001CA6B4C6E8DD741F4BBD8B8A703EB5662D
:10F168004803F60E613557B986C11D9EE1F898111E
:10F1780069D98E949B1E87E9CE5528DF8CA1890D0D
:10F18800BFE6426841992D0FB054BB1623232323B1
:10F19800232320257320253032583A253032583A17
:10F1A800253032583A253032583A253032583A25E7
:10F1B8003032583A253032583A253032583A2530CC
:10F1C80032583A253032583A253032583A253032BA
:10F1D800583A253032583A253032583A2530325884
:10F1E8003A253032580D0A002323232323232044B1
:10F1F80065764555493A2020202020202530325870
:10F208003A253032583A253032583A253032583A71
:10F21800253032583A253032583A253032583A2576
:10F228003032580D0A0023232323232320417070F2
:10F238004555493A202020202020253032583A25AB
:10F248003032583A253032583A253032583A25303B
:10F2580032583A253032583A253032583A25303229
:10F26800580D0A0023232323232320446576416471
:10F2780064723A2020202020253032583A25303236
:10F28800583A253032583A253032580D0A00417024
:10F29800704B65793A2020202020004E776B4B6513
:10F2A800793A2020202020004E776B534B65793A1D
:10F2B8002020202000417070534B65793A2020208F
:10F2C80020004442496E744B65793A202020004D55
:10F2D80043526F6F744B65793A2020004D434B457C
:10F2E8004B65793A20202020004D43417070534BE4
:10F2F80065795F303A004D434E776B534B65795FC4
:10F30800303A0000000000004150505F96F20008BB
:10F31800010000004E574B5FA3F2000808000000F0
:10F328004E574B53B0F200080900000041505053AB
:10F33800BDF200080A0000004442495FCAF2000812
:10F348000B0000004D435254D7F200080C00000097
:10F358004D434B45E4F200080D0000004D434B308F
:10F36800F1F200080E0000004D415330F1F20008A0
:10F378000F0000004D4E5330FEF200081000000050
:10F388005A45524FCBF30008526164696F53656E5A
:10F3980064204F76657273697A650D0A0049525187
:10F3A8005F52585F54585F54494D454F55540D0AA4
:10F3B80000505245204F4B0D0A0053594E43204FE1
:10F3C8004B0D0A00484452204F4B0D0A0048445246
:10F3D800204B4F0D0A004952515F4352435F45523B
:10F3E800524F520D0A00020100030000841E000063
:10F3F800093D0000127A000024F4000048E80100EA
:10F4080090D0030020A1070000000000B1280000F0
:10F4180061510000C3A200000405060005C20008EF
:10F42800C9C0000801C3000845C1000819CC00087C
:10F43800EDC1000845C90008BDC70008A9BF0008FC
:10F4480055CE000895CC0008D9C10008C1C00008F5
:10F4580071C1000849C1000801C10008F7C00008CF
:10F46800F9BF0008F5BF0008F3C00008EFC00008A6
:10F4780099C20008C5C20008E5C0000871CF00089D
:10F4880059C0000821C0000841CF0008FDBF00088E
:10F49800C5C500084DC300088DDD000893DD0008D0
:10F4A800EDBF0008F1BF0008C01200001F000000F7
:10F4B800A816000017000000841C00000F000000C0
:10F4C800E42500001E000000B42D00001600000016
:10F4D800083900000E0000002C4C00001D00000040
:10F4E800685B000015000000747200000D00000049
:10F4F800589800001C00000034B7000014000000F9
:10F50800E8E400000C000000783101001B00000056
:10F51800686E01001300000034CA01000B000000EF
:10F52800286202001A00000040DB020012000000FE
:10F538003C9303000A000000C0C204001900000048
:10F5480060B3050011000000382007000900000022
:10F5580020A10700000000000403020201010101CC
:10F5680000000000000000003C4E554C4C3E0030AE
:10F5780031323334353637383961626364656667EA
:10F5880068696A6B6C6D6E6F70717273747576777B
:10F5980078797A0030313233343536373839414268
:10F5A800434445464748494A4B4C4D4E4F505152AB
:0CF5B800535455565758595A0000000093
:10F5C4000000000000000000000000000000000037
:10F5D4000000000000000000002B7E151628AED2AB
:10F5E400A6ABF7158809CF4F3C012B7E151628AE24
:10F5F400D2A6ABF7158809CF4F3C082B7E151628E9
:10F60400AED2A6ABF7158809CF4F3C092B7E151651
:10F6140028AED2A6ABF7158809CF4F3C0A000000EC
:10F62400000000000000000000000000000B0000CB
:10F6340000000000000000000000000000000C00BA
:10F644000000000000000000000000000000000DA9
:10F6540000000000000000000000000000000000A6
:10F664000E00000000000000000000000000000088
:10F67400000F000000000000000000000000000077
:10F684000000100000000000000000000000000066
:08F6940000000000000000006E
:08F69C00DC0AFF7F0100000001
:04F6A4005D010008FC
:04F6A800390100081C
:10F6AC000000000025030020C0D401000000010070
:10F6BC00000000000000000000000000040000003A
:10F6CC00401F0000A9170008D9170008F1170008FF
:10F6DC005D1800088D1E000865210008C11D00087A
:10F6EC008D21000800000000552000089120000822
:10F6FC00ED200008871D0008831D0008851D0008EB
:10F70C00591E0008891D0008951D0008B920000825
:10F71C000200000000093D00100000000000000085
:10F72C00D00500200000000000000000FF000000D9
:10F73C0000000000D00500200000000000000000C8
:10F74C00000000000000000000000000D0050020B8
:10F75C000000FF0000000000E0000000056300084E
:10F76C0035620008416200086D620008000000006C
:10F77C00000000005D6300084D620008CD660008C3
:10F78C00000000000000000000000000000000006D
:10F79C00000E0F0D0109081101000000FF00000010
:08F7AC00FFFFFFFFFFFFFFFF5D
:040000050800239D2F
:00000001FF
